:020000040800F2
:1000000000000220CD4700081348000815480008EA
:1000100017480008194800081B48000800000000A5
:100020000000000000000000000000001D48000863
:100030001F4800080000000021480008FD0D0008CE
:1000400027480008294800082B4800082D480008C8
:100050002F48000831480008334800083548000898
:1000600037480008394800083B4800083D48000868
:100070003F48000841480008434800084548000838
:1000800047480008494800084B4800084D48000808
:100090004F48000851480008534800081933000829
:1000A00057480008594800085B4800085D480008A8
:1000B000012B0008614800086348000865480008F3
:1000C00067480008694800086B4800086D48000848
:1000D0006F48000871480008310D00087548000895
:1000E00077480008794800087B4800087D480008E8
:1000F0007F480008814800088348000885480008B8
:1001000087480008654300088B4800088D480008B0
:100110008F48000891480008934800089548000857
:1001200097480008994800089B480008FD430008CC
:100130009F480008A1480008A3480008A5480008F7
:10014000A7480008A9480008AB480008AD480008C7
:10015000AF480008B1480008B3480008B548000897
:10016000B7480008B9480008BB480008BD48000867
:10017000BF480008C1480008C3480008C548000837
:10018000C7480008C948000810B5054C237833B9A2
:10019000044B13B10448AFF300800123237010BD5A
:1001A000D00000200000000030D70008084B10B538
:1001B0001BB108490848AFF300800848036803B939
:1001C00010BD074B002BFBD0BDE81040184700BF07
:1001D00000000000D400002030D70008CC00002030
:1001E00000000000154B002B08BF134B9D46A3F5E4
:1001F000803A00218B460F461348144A121A09F020
:1002000061FD0F4B002B00D098470E4B002B00D008
:1002100098470020002104000D000D48002802D05E
:100220000C48AFF3008009F0ADFC2000290002F07B
:1002300085FC09F02BF900BF000008000000022037
:100240000000000000000000D0000020683A0120FB
:10025000000000000000000040F0BF60024B40F4CE
:100260000030D860704700BF00ED00E0C27803782E
:1002700030B51AB3174A4578D168C943C1F3022192
:10028000C1F10402D2B205FA02F2D4B20F220A413D
:1002900081780A40224303F1604303F56143120170
:1002A000D2B283F8002303780122590903F01F0317
:1002B00002FA03F3084A42F8213030BD5A090121FD
:1002C00003F01F0301FA03F32032034941F82230FF
:1002D00030BD00BF00ED00E000E100E0036823F066
:1002E000010303600023036043608360C360036114
:1002F00021234361294B984217D0294B98421BD0A8
:10030000284B984220D0284B984225D0274B984222
:100310002AD0274B98422ED0264B984232D0264BDB
:10032000984236D0254B984203D13D2243F8082C01
:100330007047234B984204D14FF4746243F8202C49
:100340007047204B984204D14FF4741243F8382C74
:1003500070471D4B984204D14FF0746243F8502C03
:1003600070471A4B984203D1194A43F8642C7047DE
:10037000184B984203D1184A43F87C2C7047174B0E
:10038000984203D1164A43F8942C7047154B984273
:1003900003D14FF03D5243F8AC2C7047106002403F
:1003A0002860024040600240586002407060024095
:1003B00088600240A0600240B860024010640240C1
:1003C0002864024040640240586402407064024065
:1003D0003D00002088640240400F0020A0640240DD
:1003E00000003D20B86402400268134B10B5134072
:1003F0000C68CA6814434A6914438A691443CA6979
:1004000014430A6A14434A6A14438A6A14434A6BBF
:1004100014438A6B2243134303604369CC6A23F07D
:1004200007020B6B2343134343610B6943604B6823
:1004300083608B68C36010BD3F801CF0036811B1FE
:1004400043F0010301E023F00103036070470368F8
:1004500011B143F0200301E023F020030360704753
:100460000B0611D543694AB143F0800380294361EB
:1004700014D0036801F01E0119430EE023F080033D
:100480008029436104D17047802907D0002AF0D128
:10049000036801F01E0123EA0101016070470000BA
:1004A00010B5084A084B094CA04294BF18461046A4
:1004B00011F0005F21F0F02121F0821114BFC16022
:1004C000816010BD00640240006002400F64024081
:1004D000FFF7E6BF837910B50468002B30D01D4BC1
:1004E000196821EA04021A605A68016822EA0102C6
:1004F0005A600279016802F1804202F59E32146866
:10050000214311609A68016822EA01029A60016839
:10051000DA6822EA0102DA6042790168102A07D11A
:100520009A6811439960D96802680A43DA6010BD7D
:1005300002F1804303F59E331A681143196010BD20
:10054000037903F1804303F59E331A6822EA04021B
:100550001A6010BD003C0140054B1A685B690340FE
:1005600004D0024214BF0120002070471846704793
:10057000003C0140014B5861704700BF003C014006
:1005800010B590E80E001A43C3681A4303691A4372
:1005900043691A4383691A43C3691A43036A1A43B6
:1005A000436A1A43836A1A43C36A1A43036B1343A9
:1005B0004FF0204242F821308368082B06D10368AF
:1005C0009B0013441A6842F040021A60426B0168B3
:1005D000146893692343546843EA0413946843EA14
:1005E0000423D46843EA04431469526943EA045378
:1005F00043EA026301314FF0204242F82130C36ADE
:100600000168B3F5804F13D1826B1068936903437F
:10061000506843EA0013906843EA00231069526966
:1006200043EA005343EA0263044A42F8213010BD12
:10063000024B6FF0704243F8212010BD040100A06E
:10064000800000F1204019B1036843F0010302E08B
:100650000268024B13400360704700BFFEFF0F00AB
:10066000F0B50023012703260A6807FA03FC3CEAD9
:10067000020233D15A00056806FA02F4E443254029
:10068000056091F804E005680EFA02FE4EEA0505E1
:1006900005600D79013D012D14D885682C408460DA
:1006A00091F805E085680EFA02FE4EEA05058560C0
:1006B000446824EA0C0444608C7945689C40A4B2E8
:1006C0002C434460C46806FA02F524EA0504C460B9
:1006D000CD79C46805FA02F22243C2600133102BBF
:1006E000C2D1F0BD4FF6FF73036000230371437165
:1006F0008371C37170470369194214BF0120002040
:10070000704710B501F00703C90800EB81009B009A
:10071000046A0F21994024EA01010162016A9A40AA
:100720000A43026210BD000010B51D4A936803F031
:100730000C03042B03D0082B03D01A4B18E01A4BE0
:1007400016E05168536811F4800F03F03F035168BD
:1007500014BF154A134AB2FBF3F3114A5268C2F3AD
:100760000142C1F3881101324B435200B3FBF2F353
:100770000B4A036093680D49C3F30313CC5C036811
:10078000E34043609468C4F382240C5D23FA04F4CC
:1007900084609268C2F342328A5CD340C36010BD69
:1007A000003802400024F40000127A00000000200B
:1007B000044B1A6B09B1104301E022EA00001863F0
:1007C000704700BF00380240044B9A6B09B11043D8
:1007D00001E022EA00009863704700BF0038024041
:1007E000044B1A6C09B1104301E022EA00001864BE
:1007F000704700BF00380240044B5A6C09B11043E7
:1008000001E022EA00005864704700BF003802404F
:10081000044B5A6A09B1104301E022EA0000586211
:10082000704700BF0038024008B501214FF4006056
:10083000FFF7EEFF00214FF40060BDE80840FFF72E
:10084000E7BF00004368816810B51943C368084CCE
:1008500019430368626819430369194322F4FD438D
:1008600023F07F03027D0B431343636010BD00BF81
:10087000002C0140014B1860704700BFA08025424A
:10088000014B1860704700BF002C0140024B1868F4
:1008900000F00300704700BF002C0140094A0368C4
:1008A00010B5936081684468D3680C43C1680C43F9
:1008B000016923F4FF6323F0070321430B43D36053
:1008C00010BD00BF002C0140014B1869C0B2704739
:1008D000002C014082B000230193034B0344019399
:1008E000019B186802B07047142C014010B50949EB
:1008F00003684B6243688B62CB6A846823F0F7021B
:10090000C3681C4303694069234303431343CB6219
:1009100010BD00BF002C0140014BD3F88000704790
:10092000002C0140014B1860704700BF8C852542A8
:10093000044BDA6B09B1104301E022EA0000D863EE
:10094000704700BF002C0140014B9863704700BF07
:10095000002C0140034B5B6B034214BF01200020BD
:10096000704700BF002C0140FFF7F4BF014B9863B4
:10097000704700BF002C014010B501F0030301F0E7
:10098000FC0101F1804101F59C319B008C680F2234
:100990009A4024EA02028A608A689840104388607C
:1009A00010BD00001C4A038890429BB212D002F591
:1009B000806290420ED0B0F1804F0BD0A2F5803211
:1009C000904207D002F58062904203D002F5806227
:1009D000904203D14A8823F0700313430F4A904298
:1009E00008D002F5806290421FBF23F440730A8949
:1009F0009BB2134303804B68C3620B880385064B8D
:100A0000984203D003F58063984201D18B7A038624
:100A100001238382704700BF0000014000100040A6
:100A20004FF0FF33436000230380038143808372D0
:100A30007047038819B19BB243F0010303E023F030
:100A400001031B041B0C03807047C94389B2018258
:100A5000704783899BB20AB1194301E023EA01017F
:100A600081817047FFF7F5BF7FB5038ACA889BB2C3
:100A700023F440531343038283890E469BB223F42D
:100A8000B053898823F00C0233890B4371890B43DF
:100A90009BB213438381838AB2899BB223F4407350
:100AA0001343838204466846FFF73EFE194B9C427F
:100AB00003D003F580639C4201D1039D00E0029DB9
:100AC000A389316813F4004F4FF0190202FB05F2BD
:100AD00014BF4D008D00B2FBF5F5A2896426B5FB6D
:100AE000F6F000010109120406FB115307D5D900E5
:100AF0003231B1FBF6F202F00702104306E01A01B0
:100B00003232B2FBF6F303F00F03184380B22081B8
:100B100004B070BD001001404FF4165303600C2266
:100B200000238380C380038142818381704783894E
:100B300019B19BB243F4005303E023F400531B04A8
:100B40001B0C83817047838929B16FEA43436FEAA5
:100B500053439BB201E0C3F30E0383817047C1F39B
:100B60000801818070478088C0F308007047012326
:100B700010B5C1F342149C4201F01F0103FA01F1C8
:100B800001D10C3003E0022C0CBF1030143003688C
:100B90000AB1194301E023EA0101016010BD0123FC
:100BA00010B5C1F3421401F01F029C4203FA02F295
:100BB00001D1838903E0022C0CBF038A838A9BB294
:100BC0001340028892B243B10123090A03FA01F1EA
:100BD0000A4214BF1846002010BD184610BD090A6D
:100BE000012303FA01F1C94389B201807047000073
:100BF00070B5344B1A68824288B0064660D01860DF
:100C000002A8FFF76FFD04A8FFF786FF0121084641
:100C1000FFF7CEFD01210846FFF7CAFD01214FF481
:100C20000030FFF7DDFD072202212748FFF769FDAD
:100C3000072203212448FFF764FD02238DF80C30BE
:100C40000323002401258DF80D3002A904231E483A
:100C500002938DF80E408DF80F50FFF701FD082329
:100C60000DEB030118480293FFF7FAFC29461748D9
:100C7000FFF769FF0C2304A91448ADF81A30049655
:100C8000ADF81440ADF81640ADF81840ADF81C4072
:100C9000FFF7EAFE29460D48FFF749FF0B482A46B1
:100CA00040F22551FFF763FF262301A88DF8043099
:100CB0008DF805408DF806408DF80750FFF7D6FAFD
:100CC00008B070BD04020020000002400044004053
:100CD00030B40E490B680D4A7F2BFBD80C4B0D4DE1
:100CE0001C68611C7F291960C0B288BF002128558B
:100CF00088BF196072B613680133136062B60122AF
:100D000040F22771044830BCFFF731BF7801002062
:100D1000EC000020F40000200044004010B5441E08
:100D200014F8010F10B1FFF7D3FFF9E710BD000071
:100D300038B540F225512848FFF731FF10B340F293
:100D400025512548FFF74BFF2348FFF70CFF234BA6
:100D50001B682BB9C3B2032B02BF214B01221A60BF
:100D6000204B1A687F2A0DD81F4A204D1468C0B244
:100D7000611C28557F29116084BF002111601A6809
:100D800001321A6040F227711348FFF708FF10B3D1
:100D900040F227711048FFF722FF154B1A689AB1ED
:100DA000144A154C1168481C8028106008BF0020A8
:100DB000615C08BF10601A680748013A1A60C9B23E
:100DC000BDE83840FFF7CBBE40F227710248BDE8CE
:100DD0003840FFF7CCBE38BD004400401000002072
:100DE0007C010020F000002074010020840100201C
:100DF0007801002080010020F4000020034B1A68D5
:100E000012B11A68013A1A60704700BF583A0020C0
:100E1000064B1A68064B012A18BFB0FBF2F00130EE
:100E200018601A68002AFCD1704700BF1800002023
:100E3000583A0020044B1B685843044B18601A684A
:100E4000002AFCD1704700BF14000020583A00204F
:100E5000104A002808BF64204FF47A73B3FBF0F304
:100E600013600D4BB3FBF0F20C4B1B68B3FBF2F3BA
:100E7000B3F1807F0AD20A4A013B5360094BF0214B
:100E800083F823100023936007231360064B186038
:100E9000704700BF1400002040420F004C000020AB
:100EA00010E000E000ED00E018000020004870476E
:100EB000CBB2425008B530B903F048F800280CBF57
:100EC0000020032008BD012008BD08B528B902F0A4
:100ED0000FFC003018BF012008BD012008BD10B56F
:100EE0000C46114638B9DAB2204603F031F800302A
:100EF00018BF012010BD042010BD10B50C461146CE
:100F000038B9DAB2204603F013F9003018BF0120D7
:100F100010BD042010BD02288CBF042000207047A3
:100F200042884378007843EA022340EA032070476E
:100F30000B0A017043700B0C090E8370C17070476F
:100F4000024400F8011B9042FBD1704730B50446C3
:100F500014F8013B11F8015B5B1B151BE84201D043
:100F6000002BF5D0184630BD83690239023B994207
:100F70003DBF4389C06A01FB03000020704710B5E4
:100F800002688AB111460B4611F8014B202C09D991
:100F90003A2CF8D1511C8B4206D11278302A03D159
:100FA00001330360002010BD4FF0FF3010BD38B595
:100FB0000D46044678B103686BB11A785AB181883E
:100FC000DA88914207D15878FFF774FF10F00100DA
:100FD00001D1236801E0092000232B6038BD0138CE
:100FE0000A4411F8013B00F8013F9142F9D17047E2
:100FF000CA7E8B7E032843EA022301BF487D0A7D17
:1010000042EA002243EA024318467047C2F307232C
:101010008A76CB760378032B01BF120C0A75120A6D
:101020004A757047002370B51A4604462E25E669B6
:10103000501CB25C202A0AD0052A08BFE5220928E4
:1010400002BFCE1801337572CE18013372720B28AD
:101050000246ECD10B4400225A72E369DB7A0B7230
:10106000E0691C30FFF75CFF0860E269D07D937D8A
:1010700043EA0023CB80E269507E137E43EA0023DB
:101080008B8070BD70B5C37804460BB9002070BD6D
:1010900000F13406026B407801233146FFF72DFF43
:1010A00080B9216B636AE269E070CB1A9342EDD29A
:1010B000A378022BEAD10A44012331466078FFF776
:1010C0001CFFE3E7012070BDF8B50446FFF7DAFF27
:1010D0000546002842D12378032B37D12779012FE9
:1010E00034D104F1340601464FF400723046FFF764
:1010F00027FF552384F83232AA2384F8333252234F
:101100004122722184F8343084F83530612384F828
:10111000363084F8372084F81A2284F81B3284F899
:10112000181284F8191204F507702169FFF700FFFF
:10113000E16804F50870FFF7FBFE226A607801326F
:1011400022633B463146FFF7D8FE25710022114647
:101150006078FFF7E0FE003018BF0120F8BD70B5E1
:10116000036B8B4206460D4611D0FFF78BFF0446FA
:1011700070B92A46012306F134017078FFF7AFFEFB
:1011800000281CBF4FF0FF350124356300E0002428
:10119000204670BD002310B5C3704FF0FF330363CA
:1011A0000446FFF7DCFF18BB94F8332294F8323280
:1011B00043EA02234AF6552293421BD194F8343075
:1011C000EB2B03D01833DBB2012B15D803220B49CC
:1011D00004F16A00FFF7BAFE78B10522084904F16C
:1011E0008600FFF7B3FE002814BF0220002010BDC8
:1011F000042010BD032010BD022010BD54B800080B
:1012000058B800082DE9FF4100230B600F46154632
:10121000FFF7B5FE061EC0F226819A4B53F8264012
:10122000002C00F022813C60237805F0FE0583B19C
:101230006078FFF73FFEC1070BD4002D00F0178147
:1012400000F0040303F0FF00002B00F018810A20D7
:1012500015E10023F0B223706070FFF736FEC2077D
:1012600000F107810DB14307F1D400212046FFF7BB
:1012700091FF02281FD104F5FD75002115F8040C1B
:1012800010B12846FFF74CFE4DF82100013104292A
:1012900005F11005F2D100255DF8256036B1314623
:1012A0002046FFF777FF012801D80CE00320013525
:1012B000042DF1D1DFE0042800F0E080012801D9FD
:1012C0000D20DCE0002694F8402094F83F3043EAFB
:1012D0000223B3F5007FF3D194F84B5094F84A30D1
:1012E00053EA052504D104F15800FFF719FE05461D
:1012F00094F84470E5617B1E012BA770E0D894F848
:1013000041108BB26381002BDAD04B1E0B42D7D138
:1013100094F8468094F8453043EA082818F00F0FF7
:10132000A4F80880CCD194F8480094F8473053EAE8
:10133000002003D104F15400FFF7F2FD94F843308C
:1013400094F8422052EA0323BAD005FB07FE03EBD0
:10135000181272449042B3D3801AB0FBF1F14A489C
:101360004F1E8742ACD84FF6F570814206D840F642
:10137000F577B9428CBF0227012700E0032702312D
:1013800033443244032FA16126626362E26210D1CA
:1013900094F85F2094F85E3053EA022390D1B8F1BC
:1013A000000F8DD104F16000FFF7BAFDA062890043
:1013B00010E0B8F1000F83D0022F4FEA410018BFB0
:1013C0004018734418BF01F00101A3620CBF01462D
:1013D00001EB500101F2FF11B5EB512FFFF470AF9B
:1013E0004FF0FF332361E360032F4FF0800323713D
:1013F0002FD194F8652094F8643043EA0223012B3E
:1014000027D1711C2046FFF7AAFE10BB94F83322A7
:1014100094F83232207143EA02234AF6552293426D
:1014200017D104F13400FFF77BFD184B984210D11F
:1014300004F50670FFF774FD154B984209D104F5C9
:101440000770FFF76DFD206104F50870FFF768FD78
:10145000E060104A2770138801339BB2002013808C
:10146000E38060610BE00B2009E00C2007E02846D8
:1014700005E0032003E004287FF422AF012004B03C
:10148000BDE8F0810C020020F4FFFF0F52526141D1
:10149000727241610802002001292DE9F0470646D9
:1014A0000C4615466ED9836999426BD20378022B9C
:1014B0003BD0032B4BD0012B64D101EB510A416A85
:1014C00001EB5A21FFF74BFE074600285BD106F1DE
:1014D00034090AF10108CAF3080A14F001041FBF15
:1014E00019F80A3003F00F0343EA0513DBB208BF13
:1014F000EBB209F80A30716A0123F37001EB58214D
:101500003046FFF72CFE0746E8BBC8F3080814B1C5
:10151000C5F3071506E019F80810C5F3032521F0F7
:101520000F010D4309F8085029E0416A01EB14212D
:10153000FFF715FE074630BB640006F1340304F4E0
:10154000FF741A191D55C5F30725557017E0416A38
:1015500001EBD411FFF703FE0746A0B9A40006F182
:10156000340304F4FE741C442046FFF7D9FC25F034
:10157000704500F0704129432046FFF7D9FC012354
:10158000F37000E002273846BDE8F0870129F8B57E
:1015900005460C4652D9836999424FD20378022BF3
:1015A00029D0032B38D0012B48D101EB5106416AD9
:1015B00001EB5621FFF7D3FD10B14FF0FF30F8BD1E
:1015C000771C696AC6F308062E4401EB57212846AA
:1015D00096F83460FFF7C3FD0028EED1C7F3080783
:1015E0003D44E30795F8340046EA00204CBF00096B
:1015F000C0F30B00F8BD416A01EB1421FFF7AFFD0A
:101600000028DAD16400343504F4FF742B195878BB
:101610002B5D43EA0020F8BD416A01EBD411FFF7CE
:101620009EFD0028C9D1A40005F1340004F4FE7425
:101630002044FFF775FC20F07040F8BD0120F8BD94
:10164000B1F5001FF8B505460C4601D30220F8BDE0
:10165000CA06FBD106682961826862B93378022B19
:1016600001D9B36A33B93389B3EB541FEED9B36AE6
:10167000AB6116E01A4677897F02BC4211460CD353
:101680002868FFF783FF431C024618D00128DDD9E4
:10169000B3699842DAD2E41BEFE73046FFF764FC07
:1016A000A861AB696A61002BD0D003EB54233436B8
:1016B000C4F308043444AB61EC610020F8BD0120A0
:1016C000F8BD2DE9F041804605680F4631B9EE6856
:1016D000A6B1AB699E4228BF012610E02846FFF75D
:1016E00055FF012861D9421C03D14FF0FF30BDE8FE
:1016F000F081AB69984259D33E4600E001262B6940
:1017000013B90020BDE8F081BE4217D1AB69D8F80B
:101710000000741C9C4228BF02242146FFF736FFBC
:10172000012842D0431CE0D038B1EB68012B05D929
:10173000AA69934238BF1E4600E0A4B93446AB699B
:1017400001349C4202D3012EDBD902242146D8F871
:101750000000FFF71BFF30B1012826D00130C4D0B4
:10176000B442ECD1CDE74FF0FF3221462846FFF7D7
:1017700093FEC0B947B9AA692B69EC60023A93425B
:101780000AD8013B2B6107E0224639462846FFF77D
:1017900083FE0028EFD006E02B7943F001032B7184
:1017A0002046BDE8F08101289FD00120BDE8F081EE
:1017B000F8B50D46012D0746114601D80220F8BDA7
:1017C0000468A3699D42F9D22AB14FF0FF32204646
:1017D000FFF762FE08BB29463868FFF7D7FE0646CA
:1017E00008B90020F8BD0128E8D0431C14D000221D
:1017F00029462046FFF750FE78B9A2692369911E59
:101800008B4205D201332361237943F00103237115
:1018100096423546DFD3E4E70120F8BDF8B505462A
:101820000E46FFF72FFC0446F8B931462846FFF76D
:101830009BFB05F13406074628634FF400722146EE
:101840003046FFF77DFB6B899C4204D36889001BFF
:1018500018BF0120F8BD01233A1931466878FFF717
:101860004CFB0028F2D10134EDE70120F8BD2DE951
:10187000F843836904468946002B4BD0076920371B
:10188000B7F5001F46D2C7F308080668B8F1000F85
:1018900039D141690133836131B93389B3EB571FC2
:1018A00031D80023A36135E07389013B13EA572344
:1018B00029D13046FFF76AFE0128054602D80220EA
:1018C000BDE8F883421C02D10120BDE8F883B3696A
:1018D000984212D3B9F1000FE3D061692046FFF7B7
:1018E000F0FE0546C8B10128E9D0431CECD0014602
:1018F0003046FFF793FF0028E6D165612946304660
:10190000FFF732FBA061343646442761E6610020D0
:10191000BDE8F8830420BDE8F8830720BDE8F8831C
:101920002DE9F0470B7807682F2B04460E4601D0AF
:101930005C2B01D1324601E07B6908E013782F2B44
:10194000164602F10102F9D05C2BF7D00023A36008
:1019500033781F2B04D904F12008DFF8AC913FE065
:10196000802384F82B3020460021BDE8F047FFF7A4
:1019700067BE04F11F00002113F8012F2E2A01F188
:1019800001013CD02F2A3FD1202A0E448CBF2023B6
:10199000242384F82B3000212046D4F800A0FFF740
:1019A0004FFE054630B9A1695046FFF7D8FB054602
:1019B000002873D094F82B30002D40F087805A0710
:1019C00000F19E80A379DB0640F19380236938788B
:1019D000C3F3080307F134011944FFF709FBA060C2
:1019E0000B2220214046FFF7ABFA334613F80129BA
:1019F0002E2ABED000211A46084608252AE00329CF
:101A00004AD000F8012FB7E75C2ABDD0202ABBD905
:101A100042E02F2B25D05C2B23D02E2B6BD08D4278
:101A20003AD913F0800F18BF03F07F03DFF8DCC052
:101A300018BF19F803301CF801EFBEF1000F1AD1DE
:101A4000A3F1610EBEF1190F01D8203BDBB208F8FB
:101A50000130013112F8013F202B00F10100D8D8EC
:101A60000CE0321801E05C2D08D1901B12F8015BEC
:101A70002F2DF8D1F9E77345DDD10DE061B194F870
:101A80002020E52A04BF052284F82020202B8CBFCB
:101A90000023042306447CE7062531E0E06903784F
:101AA00093B1C37A03F03F03A371C37A190706D435
:101AB0000B224146FFF74AFA00283FF47BAF002192
:101AC0002046FFF7D4FE6CE7042573E7042D17D1F9
:101AD00013F0200F03F0040306D0002B80D08023E6
:101AE00084F82B3000250BE0002B14BF04250525BE
:101AF00006E0052504E00B2DCED008210B25A9E733
:101B00002846BDE8F08700BFA1B800085DB800080E
:101B100070B5044605680E460420A16909B328463D
:101B2000FFF71DFBF8B9E3691A78FAB1DB7AE52A09
:101B300003F03F03A3710DD02E2A0BD00F2B09D039
:101B400023F02003A3F1080253425341B34201D1D1
:101B5000002070BD00212046FFF789FE0028DCD060
:101B600001E00028F4D00023A36170BD0420FAE74F
:101B700038B5002104460568FFF762FD70B9A16918
:101B80002846FFF7ECFA48B9E3691B78E52B08D043
:101B90003BB101212046FFF76AFEEFE7042808BFAA
:101BA000072038BD70B505460668FFF7E1FF04461B
:101BB00090B9A9693046FFF7D2FA044660B90146E8
:101BC0002022E869FFF7BCF90B2205F12001E86942
:101BD000FFF705FA0123F370204670BD1FB5019091
:101BE00004A8009140F8041D1446FFF7C8F9002826
:101BF00013DB0C4B53F820200AB100211170019A1D
:101C00000AB100211170019A43F820203CB1002252
:101C100001A96846FFF7F6FA02E00B2000E0204633
:101C200004B010BD0C0200202DE9F04391B017461E
:101C300001910446002800F0C18002F03F052A46C9
:101C400003A901A8FFF7DEFA0646002840F0C48089
:101C50000DF14008039B48F8303D01994046FFF7DD
:101C60005FFE20B99DF93B30002BB8BF062017F06E
:101C70001C0F47D040B1042802D14046FFF792FF25
:101C800045F0080548B1A0E09DF8163013F0110F9B
:101C900040F09A80780700F19380290740D5039B94
:101CA000DDF82C9018784946FFF7A2F90746FFF7B0
:101CB000FDF8014609F10E00FFF73AF90B9B039876
:101CC0002022DA720B990022FFF7A0F90B9B002269
:101CD0001A775A779A77DA77039B0121D970EFB197
:101CE000039B39464046D3F83090FFF761FD00284A
:101CF0006BD149460398FFF732FA039B791ED960EE
:101D000050B162E0002860D19DF81630DA0659D44F
:101D1000BF0701D5D80757D4290701D545F040059D
:101D2000039FDDF82C803B6B2362C4F82480387855
:101D30004146FFF75DF9A06008F11C00FFF7F0F8DD
:101D40002760E060FB88A380002104F128074FF49E
:101D5000007225746174E16161613846FFF7F0F843
:101D6000AA0634D5E56895B3039B6561B3F80A808C
:101D7000A1684FEA4828A8450CD22068FFF706FC66
:101D800001280146C8EB050503D9431CF3D1012600
:101D900000E00226A161FEB9C5F30803BBB1039EB2
:101DA0003046FFF7E1F8A0B100EB5522E2610123D4
:101DB00039467078FFF793F868B908E009200EE01B
:101DC000082002E0042000E00720064604E000208E
:101DD00005E0022600E0012600232360304611B012
:101DE000BDE8F0832DE9F04F984685B000230F46FB
:101DF000C8F8003003A905461446FFF7D8F80028B4
:101E000040F09980687C002840F095802B7CD907B1
:101E100040F19080EB686869181A844228BF044634
:101E200005F12809002C00F083806A69C2F30803D9
:101E3000002B65D1039B5B89013B13EA522312D12E
:101E40000AB9A86805E0A96928680193FFF79EFB15
:101E5000019B012801D8022002E0421C02D101208E
:101E6000687468E0A861DDF80CB0A9690193584670
:101E7000FFF77AF80028EED0019B660A03EB000A10
:101E800020D0BBF80A209BF801009919914288BF25
:101E9000D61A334652463946FFF721F80028DED1DC
:101EA00095F91030002B0BDAE869CAEB0000864286
:101EB00006D94FF40072494607EB4020FFF78FF830
:101EC00076022AE0EA69924518D095F91030002B85
:101ED0000BDA012349469BF80100FFF70EF80028B2
:101EE000BDD12B7C03F07F032B7403980123524652
:101EF00049464078FEF7F3FF0028B0D1C5F81CA092
:101F00006969C1F30801C1F50076A64228BF2646DB
:101F1000324649443846FFF762F8D8F80030334477
:101F2000C8F800306B69A41B37441E446E6179E722
:101F3000204600E0072005B0BDE8F08F2DE9F04F06
:101F40009B4685B000238846CBF8003003A90446A1
:101F50001646FFF72CF8002840F0AB80607C002884
:101F600040F0A780237C9A0740F1A2806369F34286
:101F700028BFDE4304F12809AEB16369C3F3080248
:101F8000002A74D1039A5289013A12EA532201922B
:101F90001CD11BB9A06860B9014600E0A1692046C8
:101FA000FFF78FFB28B9237C43F040032374002004
:101FB0007FE0012801D1022002E0431C02D1012070
:101FC000607476E0A368A06103B9A06094F9103052
:101FD000002B0CDA0398E269407801234946FEF7AA
:101FE0008CFF0028EBD1237C03F07F032374DDF802
:101FF0000CA0A1695046FEF7B7FF0028DBD0019B7B
:10200000750A03EB000721D0019ABAF80A309AF852
:1020100001002A449A4284BF019A9D1A2B463A46EF
:102020004146FEF76AFF0028C9D1E169C91B8D420C
:102030000AD94FF4007208EB41214846FEF7CFFF62
:10204000237C03F07F0323746D0221E0E3699F4248
:102050000CD06269E3689A4208D201233A464946A5
:102060009AF80100FEF73BFF0028A8D1E7616069FC
:10207000C0F30800C0F50075B54228BF35462A46B2
:1020800041464844FEF7ABFF237C63F07F03237493
:10209000DBF800302B44CBF800306369761BA84492
:1020A0001D44E3686561AB422CBFE360E56063E714
:1020B000072005B0BDE8F08FF7B501A90546FEF78A
:1020C00076FF002840D12B7C03F0400202F0FF0095
:1020D000002A39D01B060CD50198EA694078012303
:1020E00005F12801FEF709FF68BB2B7C03F07F0395
:1020F0002B74FEF7DBFE296A07460198FFF72FF8DD
:10210000044608BB6E6AF37A43F02003F372AA68B0
:1021100028683146FEF77AFFE96806F11C00FEF7F1
:1021200007FF394606F11600FEF702FF019BB47463
:102130000122F474DA700198FEF7C6FF2B7C23F0BD
:1021400040032B7400E0012003B0F0BD13B504463A
:10215000FFF7B2FF28B901A92046FEF728FF00B912
:10216000206002B010BD73B50D4601A90446FEF70C
:102170001EFF002840F09580607C002840F0918090
:10218000E368AB4204D2227C12F0020F08BF1D4666
:10219000002263696261002D00F08180019A5689F6
:1021A00076026BB1013B6A1EB3FBF6F1B2FBF6F2AD
:1021B0008A4205D3724213406361ED1AA16910E0AF
:1021C000A16869B92046FFF77CFA0128014601D1D0
:1021D000022002E0013002D10120607461E0A160C0
:1021E000A161B9B900262CE0636933446361237CA3
:1021F0009A07A5EB060510D52046FFF762FA0146BF
:1022000080B14B1CE8D00129E2D9019B9B6999421E
:10221000DED2A161B542E7D805E02068FFF7B6F944
:102220000146EEE7054663692B446361C5F3080385
:10223000002BD7D00198FEF797FE0028C8D000EBFE
:102240005526E36865699D4281BF237CE56043F0C4
:1022500040032374C5F3080018B3E269B2421CD0EE
:1022600094F91030002B04F128050BDA01980123B2
:1022700029464078FEF741FE0028ADD1237C03F0CB
:102280007F03237401980123324629464078FEF7E4
:1022900026FE0028A0D1E66103E0002001E02E46E2
:1022A000D8E702B070BD1FB50446019138B30022D3
:1022B00003A901A8FEF7A6FFF0B9039B23600199CB
:1022C0002046FFF72DFB00BB94F92B30002B08DBD9
:1022D000A379DB060FD5039BE1691878FEF788FE2A
:1022E000A060039BDB88A38000212046FFF7A8F9AC
:1022F0000428034605D105200023236008E00920B7
:1023000006E0002BF8D1184602E00428F3D0F3E7EA
:1023100004B010BD13B501A90446FEF748FE00B98C
:10232000206002B010BD37B50D4601A90446FEF786
:102330003EFEC0B90146204615B9FFF781F912E00B
:10234000FFF7E6FB10F0FB030DD16B72A3691BB125
:1023500029462046FEF766FE00212046FFF787FA51
:10236000042808BF002003B030BD000008B9014BAD
:1023700018607047100200202DE9F047984601F1DF
:102380000C03B3F5F07F0F46154629D202F108037E
:10239000B3F5487F24D2134EDFF84C9000EB400099
:1023A000002406EB80063B191A46E91D284616F85C
:1023B00004A002F071FFBDF82010072301201FFACE
:1023C00088F200FA03FE1EEA0A0F14BFA9F80020E3
:1023D000A9F8001013F1FF33F3D201340C2CE2D131
:1023E000BDE8F08721B90008000008602DE9F3413D
:1023F000089E0F4614469846451E15F8010F38B141
:102400002246009643463946FFF7B6FF0834F4E704
:1024100002B0BDE8F08108B507F032F84FF4FA6376
:10242000036008BD38B502460D46374C30B103781D
:1024300023B123683549D86807F050FA132D5BD8CB
:10244000DFE805F00A0E12161A1E22262A2E323650
:102450003A3E42464A4E525623682D48D9684EE0CD
:1024600023682C48D9684AE023682B48D96846E09D
:1024700023682A48D96842E023682948D9683EE0A1
:1024800023682848D9683AE023682748D96836E0A5
:1024900023682648D96832E023682548D9682EE0A9
:1024A00023682448D9682AE023682348D96826E0AD
:1024B00023682248D96822E023682148D9681EE0B1
:1024C00023682048D9681AE023681F48D96816E0B5
:1024D00023681E48D96812E023681D48D9680EE0B9
:1024E00023681C48D9680AE023681B48D96806E0BD
:1024F00023681A48D96802E023681948D968BDE8FA
:10250000384007F06FBA00BFBC00002021C50008AA
:1025100026C5000831C5000868C500087AC500084E
:1025200096C50008A4C50008BFC50008DCC50008A2
:1025300016C600083EC6000860C6000883C600082C
:10254000A4C60008BDC60008DBC6000800C7000816
:1025500042C700087EC70008A9C70008CCC700080A
:10256000E8C700080EB478B5059B03F00302012A02
:10257000014605D0022A16D0002A46D1012224E0C5
:1025800013F4007F03F4806203D0002A08BF1222F4
:1025900002E0002A08BF022218BF0A2213F0080F27
:1025A00018BF322211E013F4007F03F4806203D0DD
:1025B000002A08BF132202E0002A08BF032218BF26
:1025C0000B2213F0080F18BF3322134B00244FF4D3
:1025D0000B7000FB0435D5F82862F60707D50134E7
:1025E000082CF6D106F04CFF172303600DE02846B7
:1025F000FFF71AFB38B9D5F8283243F00103C5F8C4
:102600002832E01C03E0FFF706FF4FF0FF30BDE883
:10261000784003B0704700BF18020020022810B5B0
:1026200016DD0338072813DC0D4B4FF40B7404FB45
:102630000034D4F82832DB070AD52046FFF786FDA0
:10264000D4F8283223F00103C4F82832002010BD4A
:1026500006F016FF092303604FF0FF3010BD00BFE6
:10266000180200200228F7B50F46164633DD03385E
:1026700007282CDC1A4B4FF40B7505FB0035D5F8F9
:102680002832DB0723D50024B6F5007F0FDD01AB30
:102690004FF4007239462846FFF7A4FB80B9019B2E
:1026A000B3F5007F1F441C440FD3F61AECE7002E4D
:1026B0000BDD01AB324639462846FFF793FB10B1DC
:1026C000FFF7A9FE07E0019B1C44204605E006F049
:1026D000D7FE092303604FF0FF3003B0F0BD00BF09
:1026E000180200200128F7B50E46174606D13B4BCD
:1026F0001868002802DA3446394D13E0022803D165
:10270000384B186800281ADB002863D0012814D140
:10271000F1E723780A2B09D02078FEF7D9FA14F8CC
:10272000013B2B60A31B9F42F3DC0DE02B680D2BBC
:10273000F2D00D20FEF7CCFAEEE7022816D12A4D92
:102740003446A31BBB4201DB384645E023780A2B05
:1027500005D12B680D2B02D00D20FEF7B9FA207899
:10276000FEF7B6FA14F8013B2B60EAE703380728B6
:102770002CDC1E4B4FF40B7404FB0034D4F82832CD
:10278000DB0723D50025B7F5007F0FDD01AB4FF444
:10279000007231462046FFF7D1FB80B9019BB3F5AB
:1027A000007F1E441D440FD3FF1AECE7002F0BDD02
:1027B00001AB3A4631462046FFF7C0FB10B1FFF7A8
:1027C0002AFE07E0019B1D44284605E006F058FE5E
:1027D000092303604FF0FF3003B0F0BD1C00002060
:1027E000781300202000002014020020180200208E
:1027F000022838B50B461BDD0338072818DC0F4CC0
:102800004FF40B7505FB0040D0F82842E4070FD5C4
:10281000012A03D0022A03D072B903E0416900E023
:10282000C1681944FFF79FFC30B1FFF7F4FD03E0E6
:1028300006F026FE09230360002038BD18020020A0
:10284000012804D1084B1B68002B08DB184602281E
:1028500005D1064B1B6810EA230038BF1846022832
:102860008CBF0020012070471C00002020000020A9
:102870007F4AFF2310F4807F10B513705370134606
:1028800027D0B0F5B97F1CD007D8B0F58A7F0CD01F
:1028900040F26B1398420BD010BDB0F5BA7F0BD04D
:1028A00040F27513984210D010BD7123137010BD03
:1028B00000231370342302E000231370422353706B
:1028C00010BD002313704423F9E700231370432342
:1028D000F5E77F2800F2CB80664A127841000AB102
:1028E000654C00E0654C14F810202144D407497869
:1028F00001D5002205E002F0020202F0FF042AB135
:102900007122FF291A7006D0012202E0FF2903D0AC
:102910002246995410BD10BD6938142800F2A780D2
:10292000DFE800F05DA5430BA5A5A596A56D6D4F4D
:102930001CA5A5A5A57DA5A52B00514A1278032AA3
:1029400000F29580DFE802F00204060834221DE060
:1029500044221FE0302221E0812223E0484A1278FD
:10296000032A00F28480DFE802F0340204064122E8
:102970007BE0332279E0832277E0414A1278032A10
:1029800075D8DFE802F002060A0E42221A704322CE
:102990005CE043221A70412258E031221A7033223F
:1029A00054E080221A70832250E0354A1278032ABC
:1029B0005DD8DFE802F0572C0204302255E0812276
:1029C00053E02F4A1278032A51D8DFE802F022029E
:1029D0000406432249E0312247E0802245E0284AAC
:1029E0001278032A43D8DFE802F0020406083422F2
:1029F0001EE0442220E0302222E0812224E0204A0E
:102A00001278032A33D8DFE802F0020406084422D1
:102A10002BE0422229E0322227E0822225E0184AD8
:102A20001278032A23D8DFE802F0020A060E4222B7
:102A30001A7044220AE043221A70422206E0312230
:102A40001A70322202E080221A7082225A7010BD5F
:102A50000B4A1278032A0AD8DFE802F002020406C1
:102A6000402202E0342200E084221A7010BD10BD22
:102A70007C1300207E13002010C800085AC90008EB
:102A800024000020820510B517D5C0F3080059288E
:102A900004D1002004F0EAFD002211E0164CFFF7FB
:102AA000E7FE2078FF2826D004F0E0FD6078FF28BC
:102AB00021D0BDE8104004F0D9BD592803D101222E
:102AC0000E4B1A7010BD0D2806D1012000F082FCBB
:102AD000BDE8104004F0A4BD074CFFF7C9FE207804
:102AE000FF2808D004F0A8FD6078FF2803D0BDE8D7
:102AF000104004F0A1BD10BD7C1300207E13002007
:102B000008B501214FF08040FDF79FFF084A136888
:102B100001331360074A13680133C82B03BF002336
:102B20001360054B136004BF01221A6008BD00BF8B
:102B3000603A0020B81500205C3A00207FB501F013
:102B4000C9FE01F051FF0520FEF782F901A8FDF74B
:102B500067FF01210846FDF743FE0023ADF80C3066
:102B6000ADF806300723029301A940F219434FF054
:102B70008040ADF80430FDF715FF012211464FF0FB
:102B80008040FDF76FFF1C2301248DF8003068465C
:102B90000F238DF801308DF802308DF80340FDF7DA
:102BA00065FB21464FF08040FDF743FF4FF4E130D5
:102BB000FEF71EF800F02EFD1B48FEF7AFF81B4B8A
:102BC0001C681D464CB11A4807F0FAFC1BE00A20AD
:102BD0000134FEF72FF90A2C08D0012215491648B6
:102BE000FEF7FCFF0328064605D1F0E731461348FF
:102BF000FFF718FC07E00028F8D12146104807F03D
:102C000037FC01232B6002F087FB052001F0B2FCAA
:102C1000002002F067FB00F0EBFB00F073FB06F016
:102C20001FFC002004B070BD5ACA000880130020A9
:102C300070CA00086FCA000884130020ABCA0008DD
:102C400088CA000807F015BF70B5824204469DF897
:102C5000106008D04FF6FF704FF6E072012B0CBFEA
:102C60001546054601E04FF478450B46084A0948E9
:102C7000152107F05BFE04FB06F1002304934FF4DB
:102C800016722B4620310348BDE87040FFF7AEBBFB
:102C9000B1CA0008BC1500202DE9F3410C4EDFF845
:102CA0003480054600240F1A3368611999420CD20A
:102CB000142C0AD014230093204600233A4608EB34
:102CC0000111FFF7C1FF0134EEE702B0BDE8F0816A
:102CD000D8150020F41500202DE9F0438FB0002412
:102CE0002146074600944FF4167040F2DF1340F27D
:102CF0001F32494D02F0DEFA48492C6002A8FFF766
:102D0000D2FA60BB464EA94606F10908444902A81A
:102D1000FFF709FB00BB737AF3B1424808F0A2F851
:102D2000C0B20428F2D9043808EB00040FB13E49C0
:102D30000CE03E49204607F06FFE002850D03C4989
:102D4000204607F069FE00284AD03A49204607F09D
:102D500063FE002844D0D9E702A8FFF7DBFA296810
:102D6000012904D9344B3548102207F06BFC0021AF
:102D70000846FFF791FF0026344640F2751800F030
:102D80002FFB76282AD05A2824D002D8292821D0EF
:102D9000F5E7B0F5B97F02D0404510D0EFE72B68DA
:102DA000013BA342EBD9671CBB1B132B88BFA4F1CB
:102DB000120639463046FFF76FFF3C46DFE7002C2E
:102DC000DDD0013CA64228BF264621463046FFF70B
:102DD00063FFD4E7194B03EB04140EE000240CE06E
:102DE0002C683F2C92D815480E4900EB0410013492
:102DF00007F049FEC9F8004088E70021009140F241
:102E0000DF1340F21F324FF4167002F053FA2046DF
:102E10000FB0BDE8F08300BFD8150020B7CA000886
:102E2000DC150020E5150020EBCE0008B9CA00082B
:102E3000BECA0008C3CA0008452C0008F4150020CB
:102E400073B5224B04462025187800950E4620497C
:102E5000002351F8201022461846FFF7F5FE002304
:102E600022461C4900950120FFF7EEFE0023224672
:102E7000194900950220FFF7E7FE0095002322463E
:102E800016490320FFF7E0FE00951EB101232246FC
:102E9000134902E013493346224620250420FFF758
:102EA000D3FE2246009500230F490520FFF7CCFEF4
:102EB0000E4B0F491878009551F820100023224638
:102EC0000620FFF7C1FE02B070BD00BF2400002045
:102ED00028000020C8CA0008CECA0008D2CA0008CC
:102EE000D7CA0008E3CA0008E8CA0008500000205A
:102EF00028CB000873B5134C00264FF6FF734FF430
:102F00001672342120460096FFF770FA204607F02B
:102F1000A9FF0D4CC5004FF47843009305F51672D8
:102F200020464FF6FF733421FFF760FA00964FF604
:102F3000FF7305F5187234212046FFF757FA02B0E7
:102F400070BD00BFF41900209FB80008F7B5002439
:102F50000646009440F2DF1340F21F3221464FF440
:102F6000167002F0A7F93EB100944FF6FF734FF4CC
:102F700016722021984806E0984800964FF6FF7395
:102F80004FF416722021964D0024FFF72FFA2C7073
:102F9000FFF7B0FF274600F023FA762800F00B81F8
:102FA00015385128F7D801A353F820F02D31000827
:102FB00059310008972F0008972F0008972F000815
:102FC0005131000835310008A331000845310008AF
:102FD0005D310008972F0008972F0008BB310008CB
:102FE00049310008F9300008FD300008653100085B
:102FF00061310008972F0008972F0008972F0008CD
:103000004131000801310008393100083131000830
:1030100069310008972F0008972F00082131000818
:10302000F530000809310008053100084D3100086D
:103030006D310008972F0008972F0008972F000880
:103040001D310008113100083D31000871310008C0
:1030500075310008972F0008972F0008972F000858
:10306000153100080D3100082531000855310008E0
:1030700079310008972F0008972F0008972F000834
:103080007D31000819310008972F00082931000808
:10309000972F0008972F0008972F0008972F0008F8
:1030A000972F0008972F0008972F0008972F0008E8
:1030B000972F0008972F0008972F0008972F0008D8
:1030C0008B310008972F0008972F0008972F0008D2
:1030D000972F0008972F0008972F0008972F0008B8
:1030E000972F0008972F0008972F0008972F0008A8
:1030F00081310008622355E0642353E0652351E0E9
:1031000066234FE067234DE068234BE0692349E0E5
:103110006A2347E06B2345E06C2343E06D2341E0E5
:103120006E233FE06F233DE070233BE0712339E0E5
:10313000722337E0732335E0742333E0752331E0E5
:1031400076232FE077232DE078232BE0792329E0E5
:103150007A2327E0302325E0312323E0322321E0C6
:1031600033231FE034231DE035231BE0362319E011
:10317000372317E0382315E0392313E02D2311E01E
:10318000002C3FF408AF013C11E0002C3FF403AFEA
:103190000EB1144900E014491148114C07F05AFCD3
:1031A0000DE06123062C3FF6F6AE2B5501342F556A
:1031B000FFF7A0FEEFE6002401E06323F2E7002121
:1031C000009140F2DF1340F21F324FF4167002F00C
:1031D00071F8204603B0F0BDF1CA0008FBCA000830
:1031E000F4190020C3CA0008BECA00082DE9F8433C
:1031F000414CDFF80C812168404E0020FFF720FE93
:103200000025274600F0ECF876286BD05A2815D018
:1032100002D8292812D0F5E7B0F5B97F04D040F2E2
:103220007513984204D0EDE7052DEBD8013502E087
:10323000002DE7D0013D2168284650E0062DE1D859
:10324000DFE805F004191C2630440E0033782168AD
:103250000133DBB2042B08BF0023337000203EE0B3
:1032600098F800300BB1002000E0012004F0DEF9F6
:103270002168062033E004F0A1F933E00120FFF7D4
:103280002BFD10B104F0DEFA2CE02168022026E0CC
:103290000020FFF721FD10B104F084FA22E021683C
:1032A00003201CE02068DFF8509018B104F0ECFA1D
:1032B000002305E0FFF74AFE28B104F0F1FA0123EC
:1032C000C9F800300EE03968042008E00120FFF75B
:1032D0003DFE10B104F0CAFA04E021680520FFF7B2
:1032E000AFFD8FE72168FF20FFF7AAFD0020BDE8B2
:1032F000F84300F06FB800BFD41500202400002070
:103300005000002008B50520FFF730F80021FF200D
:10331000BDE80840FFF794BD38B58020FDF71CF9E3
:10332000002848D08020FDF725F980212248FDF7AC
:10333000E2F900283FD100F18040402100F5013042
:10334000FDF7D9F91D490B785A1E072A08D81C4CDD
:10335000227801284FEA520208BF62F07F022270F1
:103360000133DBB20A2B01D80B7038BD00230B7080
:10337000134B144C1878F0281D4603D1236843F4EE
:10338000007315E0E02803D1236843F480730FE055
:10339000238818430C4B1A88824208D018800B4BA4
:1033A0001B6813B9FFF76EFB01E0094B186000239F
:1033B000236000232B7038BD00040240081A00204F
:1033C000141A0020101A00200A1A00200C1A0020DB
:1033D000041A0020014B1860704700BF0C1A00202F
:1033E000024B002218681A60704700BF041A0020C0
:1033F00070B5012186B00220FDF7DAF91E4E06A94C
:103400008025002441F8105D30468DF80C408DF881
:103410000F40FDF725F901214FF48040FDF7ECF94D
:1034200007210120FDF7A8FA04950C23012504A823
:103430008DF815308DF814408DF81650FDF74AF8C8
:10344000172301A88DF804308DF805508DF806502B
:103450008DF80750FCF70AFF29460220FDF7A8F96E
:10346000402304A930468DF814408DF8174004938A
:10347000FDF7F6F806B070BD0004024010B50D4B24
:10348000586B10F0450FFBD0430704D50420FDF71F
:103490005BFA032010BD10F0010404D00120FDF7F9
:1034A00053FA012010BD40F2FF50FDF74DFA2046BF
:1034B00010BD00BF002C014038B5394B0546586B94
:1034C00010F0450FFBD0410704D50420FDF73CFA6E
:1034D000032038BD10F0010404D00120FDF734FAB8
:1034E000012038BDFDF7F0F9A84201D0102038BD09
:1034F00040F2FF50FDF728FA2046FDF7EBF9294B83
:1035000003404BB3002829DB420029D4830029D48F
:10351000C50029D4040129D4410129D4C20129D4E8
:10352000030229D44502E1D4840227D4C10227D45E
:10353000020327D4430327D4850327D4C40327D405
:10354000010427D4420427D4830427D410F0080FA1
:103550000CBF00201A2038BD184638BD1C2038BDCD
:10356000092038BD0A2038BD0B2038BD0C2038BDDD
:103570000D2038BD0E2038BD0F2038BD112038BDBC
:10358000122038BD132038BD142038BD152038BD99
:10359000162038BD172038BD182038BD192038BD79
:1035A000002C014008E0FFFD10B5094800230C2461
:1035B00080E81800C36040224FF48063826003619A
:1035C000FDF76CF92046BDE81040FFF775BF00BF5E
:1035D000D01A002010B50D4B0D481B681B0403606A
:1035E000402383600023C3600D244FF48063446054
:1035F0000361FDF753F92046FFF75EFF20B9FDF7A1
:1036000069F9C0F3432010BDFF2010BDCC1A002083
:10361000D01A0020F7B54FF4C060FCF71DFE01255D
:10362000002631236846304C8DF800308DF801605B
:103630008DF802608DF80350FCF718FE3B236846B6
:103640008DF800308DF80150FCF710FE29460C2053
:10365000FDF7AEF820460C220821FDF752F820466F
:103660000C220921FDF74DF820460C220A21FDF716
:1036700048F820460C220B21FDF743F81B4F0C2283
:1036800011462046FDF73DF80C2238460221FDF791
:1036900038F84FF4706300936946022320468DF892
:1036A00005308DF804308DF806608DF80750FCF772
:1036B000D7FF0423694638460093FCF7D1FF4FF447
:1036C00080536946204600938DF80760FCF7C8FFD9
:1036D00029464FF40060FDF78FF829464FF480002B
:1036E000FDF766F803B0F0BD00080240000C024090
:1036F0002DE9F04F9C4D9D4C87B0FDF795F80026C5
:10370000762328462B752E606E60AE60EE602E61CB
:10371000FDF798F80320FDF7B3F80120FDF7AAF8AC
:103720004FF480632046236126606660A660E660F1
:10373000FDF7B4F84FF480330293029BCBB9029BA0
:10374000002B00F0E08240F2FF50FDF7FDF800266C
:103750004FF4D5700821402384E84B004FF4806378
:1037600082482361FDF79AF84FF480330393804A2F
:103770000CE08020FDF7F8F80028E0D1029B013B27
:10378000DAE7039931B1039B013B0393536B13F0C9
:10379000450FF6D0039A0AB15A0714D50420FDF755
:1037A000D3F8402300263727A3607048E6604FF423
:1037B0008063236184E8C000FDF770F83846FFF7A6
:1037C0007BFEB04609E05F0602D54020FDF7BCF85D
:1037D000684B01221A604FF080480023372684E8A6
:1037E00048004022E3606148A2604FF48063236197
:1037F000FDF754F83046FFF75FFE002840F0838263
:10380000DFF86C91DFF864B10746CA463723002120
:103810004022564801934FF4806684E80A00A26073
:103820000092E1602661FDF739F8019B1846FFF729
:1038300043FE002840F0678248F0004343F48013C1
:10384000CBF80030009ACBF80C0029234748CBF87E
:103850000430CBF80820CBF81060FDF71FF8D9F83A
:10386000343013F0450F02D1DAF83430F9E713F0B1
:10387000040637D140F2FF50FDF766F83046FDF7F9
:1038800029F8002807F101074FF6FF7302DB9F427A
:10389000BCD138E29F4200F03682460002D5354B5B
:1038A00002221A60FCF7F2FF002800F02C82314E51
:1038B0003368042B1FD13368022B3FD80023032227
:1038C00023606260E36040224FF4806327482361F5
:1038D000A260FCF7E3FF264B586B10F0450FFBD0BE
:1038E000420701D5042003E010F0010729D0012090
:1038F000FDF72AF807E20023022223606260E360FA
:10390000C0224FF480631948A2602361FCF7C6FF10
:10391000FFF7B4FD002840F0F681FCF7DBFF164FFF
:1039200038600420FCF7D6FF78600820FCF7D2FF4F
:10393000B8600C20FCF7CEFFF860BCE7062B1DD169
:10394000BCE7FCF7C1FF032840F0DD8140F2FF50E7
:10395000FCF7FAFF3846FCF7BDFF10F4604F40F06B
:10396000D281000C0BE000BFB01A0020D01A00205A
:10397000002C0140981A00209C1A00200120336876
:10398000E24F042B28D009236360C0233860A36072
:10399000000400232060E360DD484FF4806323616E
:1039A000FCF77CFFFFF76AFD002840F0AC81FCF7D4
:1039B00091FFDFF86C83C8F800000420FCF78AFF51
:1039C000C8F804000820FCF785FFC8F808000C20A0
:1039D000FCF780FFC8F80C00DFF84483CD484FF0B7
:1039E000000A85F814A0C5F800A0C5F804A0C5F821
:1039F00008A0C5F80CA0C5F810A0FCF723FFD8F864
:103A00000020C54B3068D7F8009083F856004FEA85
:103A1000126E5FFA8EF14FEA911CCEF3830E01F025
:103A2000030183F800C083F801E09970C2F30741F5
:103A3000D970C2F30721D2B219715A71D8F8042093
:103A4000A3F85490110E0901D980D988C2F3074E0A
:103A500089B241EA1E11D980110A0EF00F0E5FFAE9
:103A600081FC83F808E04FEADC1E83F809E0C1F32B
:103A7000801E83F80AE0C1F3401E83F80BE00128A2
:103A8000C1F3001E83F80CE083F80DA09E4600F2FF
:103A90004981890201F44061CEF81010DEF810303F
:103AA000D8F80810920002F47F721A43CEF8102062
:103AB000DEF810000A0ED3B240EA9310C2F3C2023D
:103AC00003F00703CEF810008EF814208EF815309E
:103AD0000B0CC3F342128EF81620C3F382025B0074
:103AE00003F006038EF817208EF818309EF8183071
:103AF000C1F3072C43EADC138EF81830DEF810B05F
:103B00009EF818209EF808A00123023203FA0AFA50
:103B100003FA02F2D1170BF1010BA2FB0A230AFBF5
:103B20000133A2FB0B010BFB0311CEE91201CEF80E
:103B300050A0CCF380134FEA4C0C0CF07E0C8EF8A6
:103B400019308EF81AC09EF81A2098F80830D8F864
:103B50000C10DFF8BC8142EAD31203F07F038EF829
:103B60001A208EF81B300B0EDA098EF81C20C3F3D6
:103B700041128EF81D20C3F382029B0003F00C0358
:103B80008EF81E208EF81F309EF81F000A0CD3B24C
:103B900040EA9310C2F340128EF81F0003F00103B5
:103BA0008EF8202000228EF821208EF822300B0A79
:103BB000D8B24FEAD01C8EF823C0C3F3801C8EF815
:103BC00024C0C3F3401C8EF825C000F00300C3F3EB
:103BD000001CC1F34601C3F381038EF826C08EF8A2
:103BE00027308EF828008EF829104C490B684FF0CA
:103BF000010A180E8EF82AA08EF82C00C3F3074095
:103C00000002AEF82E00BEF82E001FFA80FCC3F3AF
:103C100007204CEA00001B06AEF82E00CEF830302C
:103C20004B68DEF830004FEA136C40EA0C40CEF8E7
:103C300030004FEA132CDEF83000E2600CF47F4CC9
:103C40004CEA0000CEF83000DEF83000C3F3072C59
:103C50004CEA0000DBB2CEF830008EF834308B68CE
:103C6000180E8EF83500180C0006CEF83800DEF875
:103C700038004FEA032C0CF47F0C4CEA0000CEF81D
:103C80003800DEF838001B0203F47F430343CEF80C
:103C90003830CB68DEF8381041EA1361CEF83810BE
:103CA0009EF83CC0190CC1F3031009024CEA000055
:103CB00001F470618EF83C00AEF83E10BEF83E1084
:103CC00088B2C3F307210143C3F34603AEF83E10A5
:103CD0008EF840304FEA09432360404607234FF0F7
:103CE000400B4FF48069636000938EF841A0C4F8E4
:103CF00008B0C4F81090FCF7D1FD009B1846FFF700
:103D0000DBFB00283CD04FF0FF3014E1CC1A002040
:103D1000D01A0020B01A0020181A00209C1A002087
:103D2000701A002002287FF404AF120402F47C12FF
:103D3000CEF81020D8F80830DEF81020190E42EA2C
:103D40000122CEF81020DEF81020C3F307410A4309
:103D5000CEF81020DEF81020C3F3072C01324FF00C
:103D6000000343F10003DB0443EA5233CEF84C3046
:103D7000D2044FF40073CEF84820CEF85030D8E685
:103D80003368032BBFD0022B00F2D480FCF7A2FDD6
:103D900010F00073B7D11022404608260493059313
:103DA000C8F80C300093C8F804200192C8F80060ED
:103DB000C8F808B0C8F81090FCF770FD019A1046DA
:103DC000FFF77AFB009B002872D13B68C8F80C0013
:103DD0001B04C8F80030009037234046C8F8043070
:103DE0000193C8F808B0C8F81090FCF757FD019B84
:103DF0001846FFF761FB009A034600285AD14F4846
:103E000000934FF0FF3280E84400302282600222AB
:103E1000C2600361C0F814A03326FCF767FD009B65
:103E2000C8F800304046C8F80C30C8F80460C8F83C
:103E300008B0C8F81090FCF731FD3046FFF73CFBA6
:103E4000009BD0BBDFF8FC8003AED8F8342040F2F2
:103E50002A63134053B94FF40010FCF785FD002886
:103E6000F3D0FCF759FD46F8040FEEE70820FCF705
:103E70007BFD08B108203BE50220FCF775FD08B189
:103E8000022035E52020FCF76FFD08B120202FE54A
:103E90004FF40070FCF768FD064610B14FF4007057
:103EA00026E540F2FF50FCF74FFD049B1BBA08E0EB
:103EB000064603E00646134600E00646002E7FF461
:103EC00022AF5B037FF51FAF3B68DFF87C80E660C5
:103ED0001B044FF0370A40464FF040094FF480670B
:103EE0002360C4F804A0C4F808902761FCF7D6FC4E
:103EF0005046FFF7E1FA78B902230624404688E8E5
:103F00001800C8F80890C8F80C60C8F81070FCF7E2
:103F1000C5FC2046FFF7D0FA00287FF4F4AE2875E0
:103F200028606860A8604FF4006328610448EB6073
:103F3000FCF788FC002007B0BDE8F08F801A002055
:103F4000B01A0020002C0140D01A00200020704739
:103F50002DE9F04F6C4BDFF8D4A16C4D6C4F002471
:103F6000012691B02C708146CAF800404FEA4128E2
:103F70003E603146DC6240F22A30FCF7D9FC4FF05B
:103F8000FA516448FCF7A4FA21466248FCF756FA55
:103F90006048FCF7A3F94FF0006301935E4B029376
:103FA0004FF4806307934FF4805308934FF480439A
:103FB00009934FF440330B9304230C9303230D9385
:103FC0004FF40003CDF80C900E934FF400794FF4AA
:103FD000001301A94F480F930494CDF81490069450
:103FE0000A94FCF701FA324610214A484B4CFCF780
:103FF00037FA20214748FCF72AFA31464548FCF7B2
:104000001DFA3046FCF78EFC454BC4F800901B6847
:104010004FF0100B022B20464FF0000356464FF492
:1040200080694FF0400A08BF4FEA5828C4F804B02E
:10403000E360C4F808A0C4F81090FCF72FFC5846C1
:10404000FFF73AFA834610BB36484FF0FF314FF086
:10405000900C4FF0020E4FF4007380E80A500123D9
:104060004361C0F810B0FCF741FCC4F80080204662
:104070004FF01208C4F80480C4F808A0C4F80CB0CB
:10408000C4F81090FCF70AFC4046FFF715FA264AE0
:104090004FF0FF33116831B9316821B9297811B96E
:1040A0000BB1013BF6E7204B00221A60164B4FF094
:1040B000FF365A6B920402D50EB1013EF9E73B6818
:1040C000012B16D1FFF770FA114B002204461A603B
:1040D0000EB900B9042440F2FF50FCF735FC2B78F0
:1040E00013B10A4B1C78E4B2FFF774FA0428FBD131
:1040F00003E0002EEED00024EDE7201C18BF0120C5
:10410000404211B0BDE8F08F002C0140151A00208C
:10411000E41A002058640240802C0140D01A00208C
:10412000981A0020801A0020C81A0020AC1A00201B
:104130002DE9F04F804BDFF828A2804D804F0024FE
:10414000012693B02C708046CAF800404FEA4129FE
:104150003E603146DC6240F22A30FCF7E9FB4FF06A
:10416000FA517848FCF7B4F921467648FCF766F92D
:104170007448FCF7B3F84FF000630393724B049359
:10418000402306934FF4806309934FF480530A93BE
:104190004FF480430B934FF440330D9304230E935D
:1041A00003230F934FF40003CDF8148010934FF4C2
:1041B00000784FF4001303A962481193CDF81C80D6
:1041C00008940C94FCF710F9324610215D485F4CBE
:1041D000FCF746F920215B48FCF739F9314659488C
:1041E000FCF72CF93046FCF79DFB594BC4F80080D6
:1041F0001B682046022B56464FF000034FF0100A72
:104200004FF0400B4FF4806808BF4FEA5929C4F8BB
:1042100004A0C4F808B0E360C4F81080FCF73EFBCB
:104220005046FFF749F9002849D14A4BE0601B6826
:10423000C4F808B003FA0AF320464FF0370A2360A7
:10424000C4F804A0C4F81080FCF728FB5046FFF720
:1042500033F9A0BB1723E0604FF0010A20466360EA
:104260000193C4F800A0C4F808B0C4F81080FCF7AB
:1042700015FB019B1846FFF71FF900BBC4F800901F
:10428000E0604FF019092046C4F80490C4F808B063
:10429000C4F81080FCF702FB4846FFF70DF970B92F
:1042A0002D4B4FF0FF314FF400729024D86018610D
:1042B000184683E81600C3F814A0FCF717FB274A3A
:1042C0004FF0FF33116831B9316821B9297811B93C
:1042D0000BB1013BF6E7214B00221A60164B4FF061
:1042E000FF365A6BD20402D50EB1013EF9E73B68A6
:1042F000012B16D1FFF758F9114B002204461A6022
:104300000EB900B9042440F2FF50FCF71DFB2B78D6
:1043100013B10A4B1C78E4B2FFF75CF90428FBD117
:1043200003E0002EEED00024EDE7201C18BF012092
:10433000404213B0BDE8F08F002C0140151A002058
:10434000E41A002058640240802C0140D01A00205A
:10435000981A0020CC1A0020801A0020C81A0020C9
:10436000AC1A002010B54FF48070FCF7F3FA214C22
:1043700048B100234FF480702370FCF7F7FA1E4B0E
:1043800001221A602EE00220FCF7E4FA20B102209C
:10439000FCF7ECFA022324E00820FCF7DBFA20B15A
:1043A0000820FCF7E3FA04231BE02020FCF7D2FAF4
:1043B00020B12020FCF7DAFA062312E01020FCF7E7
:1043C000C9FA20B11020FCF7D1FA052309E04FF417
:1043D0000070FCF7BFFA28B14FF40070FCF7C6FA82
:1043E0000723237000214CF23A30FCF7A1FA23781E
:1043F00010BD00BF151A0020AC1A0020064B1B6828
:1044000013F0C05F07D0054B054801224FF0C251A1
:104410001A60FCF75DB8704700640240C81A0020BB
:10442000586402400C4B1A6812F0010F14BF0023AD
:104430000823910748BF43F0020352074FF0C042E0
:104440004FF03601118048BF43F0010302F500220E
:104450009BB21380704700BF380000204FF0C0436C
:1044600001221A800520FCF7E5BC4FF0C0432A2248
:104470001A8003F50023C0F30F221A80C0B2C1F3E3
:104480000F22C9B218801A80198070474FF0C043BC
:104490002B221A8003F50023C0F30F221A80C0B22A
:1044A000C1F30F22C9B218801A80198070474FF0EB
:1044B000C0432C221A80704730B54FF0C044B0255D
:1044C000258004F5002489B280B220802180C2F3C7
:1044D0000F21D2B221802280C3F30F22DBB22280CF
:1044E0002380BDF80C30238030BD30B54FF0C04480
:1044F000B425258004F50024C0F30F25C0B2258023
:1045000092B22080C1F30F20C9B220802180228086
:10451000C3F30F22DBB222802380BDF80C3023804E
:1045200030BD30B54FF0C044B625258004F50024D9
:10453000C0F30F25C0B2258092B22080C1F30F20B6
:10454000C9B2208021802280C3F30F22DBB22280F7
:10455000238030BD4FF0C043E6221A8003F50023CC
:10456000C0F307421A80C0F30722C0B21A80188035
:1045700070470000014B1860FFF754BF380000205F
:104580002DE9F0438D4D8E4E99B001211820002465
:10459000FCF70EF903274FF2B37309A928460993D4
:1045A0004FF680798DF828408DF82B408DF82970D2
:1045B000FCF756F809A93046CDF82490FCF750F8DE
:1045C00001217820FCF7F4F84FF002084CF2337325
:1045D00009A9284609938DF828808DF829708DF84F
:1045E0002A408DF82B40FCF73BF8214628460C2248
:1045F000FCF787F828460C220121FCF782F82846B0
:104600000C220421FCF77DF828460C220521FCF73A
:1046100078F828460C220821FCF773F828460C226B
:104620000921FCF76EF828460C220A21FCF769F8EC
:1046300028460C220E21FCF764F80C2228460F2194
:10464000FCF75FF809A93046CDF82490FCF708F88C
:1046500030460C220721FCF754F830460C22082182
:10466000FCF74FF830460C220921FCF74AF8304697
:104670000C220A21FCF745F830460C220B21FCF7EE
:1046800040F80C2211463046FCF73BF830460C222D
:104690000D21FCF736F830460C220E21FCF731F8DC
:1046A0000C2230460F21FCF72CF84FF4005309A9D7
:1046B00028460993FBF7D4FF0C2228460D21FCF76E
:1046C00020F8802309A928460993FBF7C9FF0C228B
:1046D00028460721FCF715F801210846FCF774F875
:1046E0000F2302930D23049310230C934FF4805354
:1046F000129309A802AB4FF0C04616931793039488
:10470000059406940794089409940A940B940D94C4
:104710000E940F9410941194139414941594FBF721
:104720002FFF01212046274DFBF78AFFFFF796FE5A
:10473000E223338023232B804FF0E009A5F800808B
:1047400004234FF001082B806420A6F80090A5F800
:104750000080FCF75DFBA6F800901B482F80FFF758
:10476000F9FE21462046009440F2DF1340F21F324A
:10477000FFF7A2FE3B460094082233214FF47A70E3
:10478000FFF7B3FE3A46182140F212201723FFF735
:10479000C8FEF023338029232F803380FFF742FEA9
:1047A000BE23338006232B80FF232B80A5F80080B7
:1047B0002B802C802C8019B0BDE8F083000C0240C7
:1047C0000010024000000860E09304000649074A18
:1047D000074B9A42BEBF51F8040B42F8040BF8E7AE
:1047E00004488047044800473CD7000800000020E8
:1047F000CC000020D5480008E50100083349344AC0
:10480000002301E041F8043B9142FBD3FEF796F907
:10481000FEE7FEE7FEE7FEE7FEE7FEE7FEE7FEE770
:10482000FEE7FEE7FEE7FEE7FEE7FEE7FEE7FEE760
:10483000FEE7FEE7FEE7FEE7FEE7FEE7FEE7FEE750
:10484000FEE7FEE7FEE7FEE7FEE7FEE7FEE7FEE740
:10485000FEE7FEE7FEE7FEE7FEE7FEE7FEE7FEE730
:10486000FEE7FEE7FEE7FEE7FEE7FEE7FEE7FEE720
:10487000FEE7FEE7FEE7FEE7FEE7FEE7FEE7FEE710
:10488000FEE7FEE7FEE7FEE7FEE7FEE7FEE7FEE700
:10489000FEE7FEE7FEE7FEE7FEE7FEE7FEE7FEE7F0
:1048A000FEE7FEE7FEE7FEE7FEE7FEE7FEE7FEE7E0
:1048B000FEE7FEE7FEE7FEE7FEE7FEE7FEE7FEE7D0
:1048C000FEE7FEE7FEE7FEE7FEE70000D00000207F
:1048D000683A01203E4AD2F8883043F47003C2F8A7
:1048E00088303C4B1A68002142F001021A6099603E
:1048F0001A6822F0847222F480321A60364A5A60B2
:104900001A6882B022F480221A60D9600091019165
:104910001A6842F480321A601A6802F40032019276
:10492000009A01320092019A1AB9009AB2F5C06F4A
:10493000F2D1284B1B6813F4003318BF01230193F5
:10494000019B012B3DD1234B24491A6C42F080522C
:104950001A640A6842F480420A609A689A609A6807
:1049600042F400429A609A6842F4A0529A601A682F
:1049700022F080721A601968164A8801FBD4184B1D
:104980005360136843F0807313601168114B890101
:10499000FBD5144A40F205711160126802F007025B
:1049A000052A00D0FEE79A6822F003029A609A680E
:1049B00042F002029A609A6802F00C02082AFAD1C8
:1049C00000E0FEE7024B4FF000629A6002B07047D1
:1049D00000ED00E00038024010300024007000407C
:1049E000042A4007003C0240174A1849936803F024
:1049F0000C03042B03D0082B03D0154B18E0154BE8
:104A000016E05068536810F4800F03F03F035068BD
:104A100014BF104A0E4AB2FBF3F30B4A5268C2F3BA
:104A20000142C0F38810013243435200B3FBF2F35A
:104A30000B60054B084A9B68C3F30313D25C0B68F9
:104A4000D3400B60704700BF003802404C0000208C
:104A50000024F40000127A003C000020F8B54368FE
:104A6000013B002B04460E46436008DA154F014611
:104A7000386805F01FFF421C054616D003E00368A6
:104A80005A1C02601D786368013B002B636007DAE3
:104A90000C4F2146386805F00DFF431C05D00BE094
:104AA00023685A1C2260187806E03B680648D968DB
:104AB00004F098FF0020F8BD45EA0025358001206C
:104AC000F8BD00BFBC00002030CB00089368013B5C
:104AD000002B10B4936009DA9469A34202DBCBB2D5
:104AE0000A2B03D15DF8044B06F0B2BA1368581CC8
:104AF00010601970C8B25DF8044B704770B5436818
:104B0000013B002B04460E46436007DA0C4D01467C
:104B1000286805F0CFFE431C07D003E003685A1C49
:104B2000026018783070012070BD2B680548D96884
:104B300004F058FF204604F00FFD002070BD00BFB8
:104B4000BC0000204ECB00082DE9F04F85B0884610
:104B50000DF10E01064692469B469DF83890FFF7F0
:104B6000CDFF0446002800F092800F9F9DF80E5064
:104B7000023F002D49D1B9F1000F01D12A4624E0AE
:104B8000A8461FFA88F39F4279D90DF10F013046EC
:104B9000FFF7B4FF08F101080446002877D09DF81C
:104BA0000F305D40EDE70DF10F0130468DE80C0050
:104BB000FFF7A4FF9DE80C000446002867D053458A
:104BC0009DF80F3009D35D40013293B208EB030921
:104BD0009F421FFA89F9E6D809E0BBF1000FF2D035
:104BE000B9F5804F24BF3A4901F80930EBE7384B5B
:104BF00013F808208ABB374A127872BB9844802386
:104C000088F80D2088F80E3027E0B9F1000F01D1A7
:104C1000C84630E0002293B203EB08099F421FFA16
:104C200089F91AD90DF10F01304601920093FFF76F
:104C300065FF009B019A044648B353459DF80F3029
:104C400008D2BBF1000F05D0B9F5804F24BF204931
:104C500001F809305D400132DDE7012710E00DF178
:104C60000F013046FFF74AFF08F10108044670B112
:104C70009DF80F305D401FFA88F39F42EFD8002760
:104C80000DF10F013046FFF739FF044650B9124DC0
:104C900012482B68D96804F0A5FE2B68D86804F088
:104CA00015FD10E09DF80F30AB420BD00A4C0C48BC
:104CB0002368D96804F096FE2368D86804F006FDDE
:104CC000002400E03C46204605B0BDE8F08F00BF60
:104CD000643A002050000020BC0000206CCB00088B
:104CE00090CB00082DE9F04FAD4E8BB034689DF8A5
:104CF00050909DF854A00D4617469846002C35D18B
:104D0000A84904F0E3FD8346306008B9002422E29C
:104D1000022D32D107AB19195846FFF7EFFE50B9F3
:104D2000A14CA2482368D96804F05CFE2368D868C7
:104D300004F0CCFCEAE701340A2CEBD107229C49B1
:104D400007A804F0A5FF30B1974B9A481B68D968B3
:104D500004F048FEDAE79DF823201A2A0AD0924B85
:104D600095491B68D86804F0B9FDCFE7012906D042
:104D70000229CBD100248C4D46E0012DC6D13568E7
:104D800007A92846FFF76AFE044650B9864D8B48AE
:104D90002B68D96804F026FE2B68D86804F096FCCE
:104DA000D9E1BDF81C300193CDF800A04B46424636
:104DB00039462846FFF7C8FE0446CCE12868DFF8EC
:104DC000E8B105F077FD0246013000F0A781142A12
:104DD00000F0FC8023DC112A45D0122A00F0CF809D
:104DE000102A40F08B81D6F800B007A95846FFF78B
:104DF00035FE044628BB2B687048D96804F0F2FDE4
:104E00002B68D86804F062FC31684B68013B002BCA
:104E10004B60D3DB0B685A1C0A601A78D7E7212A4B
:104E200000F0328103DC202A00F0218166E1222A91
:104E300000F08781302A40F0618134680DF11A0159
:104E400053E10DF11A015846FFF708FE0446002809
:104E5000D1D0BDF81A300193CDF800A04B464246A0
:104E60003946584684E0346807A92046FFF7F6FD26
:104E7000002800F06E8107A92046FFF7EFFD00280B
:104E800000F0678107A92046FFF7E8FD002800F041
:104E9000608107A92046FFF7E1FD002800F0598155
:104EA00007A92046FFF7DAFD002800F0528107A984
:104EB0002046FFF7D3FD002800F04B810DF11A01C9
:104EC0002046FFF71BFE002800F0438107A920467B
:104ED000FFF7C4FD002800F03C816368013B002B14
:104EE000636008DA2146286805F0E4FCB0F1FF3F72
:104EF000834605D128E023685A1C226093F800B04D
:104F00006368013B002B636007DA2146286805F0DF
:104F1000D1FC411C024604D116E023685A1C2260D1
:104F20001A786368013B002B636008DA2146286821
:104F3000039205F0BFFC431C039A0ED104E02368E2
:104F4000591C2160187808E02B681D48D96804F0C6
:104F500049FD2B681B48D968F5E04BEA022B4BEA68
:104F600000400190CDF800A04B464246394620460D
:104F7000FFF7EAFD012804467FF446AFE1E034681C
:104F800007A92046FFF76AFD30B107A92046FFF7C1
:104F900065FD002840F0DD802B680B48D968D2E021
:104FA000E81A0020B4CB0008BC000020B7CB0008F2
:104FB000D8CB0008E0CB0008F7CB00081ECC0008D7
:104FC00030CB000802CD000841CC0008346806A9A7
:104FD0002046FFF743FD90B10DF11A012046FFF77F
:104FE0003DFD60B10DF116012046FFF787FD002859
:104FF00000F0AF8007A92046FFF730FD18B92B68F5
:105000005748D9689FE00DF115012046FFF776FD5E
:10501000002800F09E800DF1150120469DF815B086
:10502000FFF76CFD00B39DF8153003930DF11501EA
:105030002046FFF763FD002800F08B80039B9DF85E
:1050400015201B0243EA024343EA0B0B00239AB2EA
:105050005A4509D20DF1170120460393FFF74EFD83
:10506000039B01330028F2D12B6898686FE007A9F1
:105070003068FFF7F3FC28B1BDF81C10394805F083
:10508000F7F95EE00446BFE6D6F800B00DF11A016C
:105090005846FFF733FD00285BD09DF81A103248C0
:1050A00005F0E6F900249DF81A20E3B29A420DD9E2
:1050B00007A95846FFF722FD0134002849D0286887
:1050C0009DF81C108268FFF701FDECE7274B18687C
:1050D0000A218268FFF7FAFC33E09DF81A305A1E65
:1050E0008DF81A20002B34D007A92046FFF706FDC3
:1050F0000028F2D12B681E48D96824E01B4C1D49BA
:105100002368D86804F0EAFB2368D86804F0DEFA64
:105110000024306804F020FA34601CE0DBF8002042
:105120001548D16804F05EFCDBF80030D86804F064
:10513000CDFA124B186804F00FFA104A00231360DE
:1051400009E0012407E004F04DFC2B68D86804F066
:10515000BDFA002458E620460BB0BDE8F08F00BF32
:1051600064CC000887CC000893CC0008BC00002069
:10517000A7CC0008C5CC0008EACC0008E81A00203B
:105180002DE9F047334D98462B680F469146B3B949
:10519000314904F09BFB04462860002857D00146A3
:1051A0002E4804F01FFC21461A2004F0CDFB2146B6
:1051B000012004F0C9FB2146102004F0C5FB284C57
:1051C0002A6820681021FFF781FC2E68206832468B
:1051D000E82109F1020AFFF779FC32460321206831
:1051E000FFF774FC5FFA8AF132462068FFF76EFC25
:1051F000B8F1000F14BF4FF0FF084FF00008CAF3DA
:10520000072132462068DFF85CA0FFF75FFC3246DA
:1052100041462068FFF75AFCB9441FFA89F9B9459D
:105220000AD01AF8071020683246013781EA0808C8
:10523000BFB2FFF74BFCF2E7324641462068FFF76A
:1052400045FC286804F042FA0120BDE8F087BDE87B
:10525000F08700BFEC1A002025CD0008D8CB00084D
:10526000BC000020643A002010B5044C206818B13E
:1052700004F072F90023236010BD00BFE81A00207B
:1052800010B5044C206818B104F066F900232360BF
:1052900010BD00BFEC1A002038B514461D46FFF7BC
:1052A000E4F829462046FFF7F1F8BDE83840FFF75B
:1052B000FEB8000070B50E469D1B1146141A6A1CFC
:1052C00004FB02243246FFF7E7FFBDF81020044933
:1052D0000023A34202D00A800133FAE770BD00BF69
:1052E00000000860002210B540F2DF13044640F2CF
:1052F0001F311046FFF7D0FF06484FF44872A4B2A2
:105300004FF4F0732146013B0180FCD1013AF7D103
:1053100010BD00BF00000860FFF732B9431C044A0B
:105320009BB2D15C135C03EB012080B2704700BFDD
:10533000643A00200648074903885A1C02339BB28E
:1053400092B203808A5CC85C02EB002080B2704796
:1053500022370020643A0020034A138801339BB2AD
:105360001380024AD05C704722370020643A002044
:10537000034A138801339BB21380024AD056704708
:1053800022370020643A002010B50649064C0B88ED
:105390005A1C92B2A05CE25C02330B8042EA00200D
:1053A00010BD00BFFE1A0020643A002010B50B4A61
:1053B0000B49136811F810400633136042000132A4
:1053C0008B5C43EA0423013B9BB21C0A01F81040AA
:1053D0008B54044A13880133138010BD0C1B00202A
:1053E000F01A002022370020054A136808331360A2
:1053F000044B01221A70044A13880133138070474A
:105400000C1B00202537002022370020054A136896
:1054100008331360044B00221A70044A13880133C6
:10542000138070470C1B00202537002022370020F6
:10543000054A136808331360044B02221A70044AA9
:1054400013880133138070470C1B00202537002080
:105450002237002010B50B4A0B49136811F8104091
:1054600006331360420001328B5C43EA04230133AC
:105470009BB21C0A01F810408B54044A1388013374
:10548000138010BD0C1B0020F01A002022370020D2
:1054900070B50F4C0546FFF76BFF238801339AB2B6
:1054A0000C4B9E79012303FA01F13140234615B1DB
:1054B000B1FA81F14909084C21B121680C31216010
:1054C000024402E02168073121601A8070BD00BFEC
:1054D00022370020F01A00200C1B002010B50A4BC8
:1054E0001A6814321A600446FFF724FFFFF716FF0C
:1054F000064B020A03F8142003EB4403044A5870D5
:1055000013880133138010BD0C1B0020F01A0020FB
:105510002237002010B5FFF70DFF134B134C1A78FC
:10552000134B42B11A6814321A60FFF7F7FE030AF0
:105530002372607213E00F4A127842B11A68143273
:105540001A60FFF7EBFE030AA372E07207E01A6825
:1055500010321A60FFF7E2FE030A23716071064AF7
:1055600013880133138010BD3C370020F01A00204F
:105570000C1B0020021B00202237002010B5094B15
:105580001A680A3204461A60FFF7D4FE064B020A74
:1055900003F8142003EB4403044A587013880133C2
:1055A000138010BD0C1B0020F01A002022370020B1
:1055B00008B5134B1B78014643B1031F012B16D8C6
:1055C000104A13680B33136004310AE00E4B1B784A
:1055D0004BB1031F012B0AD80A4A13680B3313601F
:1055E0000631C9B203E0074A136807331360FFF7B7
:1055F000B3FE064B064A585413880133138008BD86
:105600003C3700200C1B0020021B0020F01A002059
:1056100022370020184B1A78184B72B11A680832DA
:105620001A60031F012B98BF0430A1F1040398BF37
:10563000C0B2012B17D8043110E0114A12787AB1A8
:105640001A6808321A60031F012B98BF0630A1F1B7
:10565000040398BFC0B2012B05D80631C9B202E0DD
:105660001A6804321A60074B5A5C1A54064A1388A7
:1056700001331380704700BF3C3700200C1B002013
:10568000021B0020F01A00202237002010B5164B14
:10569000164C1A78164B01463AB11A6813321A6042
:1056A000FFF766FE227A637A09E0124A12785AB14D
:1056B0001A6813321A60FFF75BFEA27AE37A43EAB4
:1056C0000223184480B206E01A68207907321A6073
:1056D000637943EA0020084B084A1B5C6354138833
:1056E0000133138010BD00BF3C370020F01A0020AA
:1056F0000C1B0020021B0020643A002022370020EF
:10570000094A136807331360084B13F8101003EBB2
:105710004000427842EA012205498A5CDA71054A72
:1057200013880133138070470C1B0020F01A0020EF
:10573000643A002022370020044A136809331360BA
:10574000034A138801331380704700BF0C1B0020ED
:105750002237002010B5094B1A680A3204461A6035
:10576000FFF712FE064B020A03F8142003EB440372
:10577000044A587013880133138010BD0C1B00209D
:10578000F01A00202237002008B5044A13680E33AF
:105790001360FFF7F9FD024B188008BD0C1B0020B9
:1057A0002237002010B54368013B002B0C464360B4
:1057B00007DA084B0146186805F07CF8431C07D04F
:1057C00003E003685A1C026018782070012010BDA5
:1057D000002010BDBC00002037B50C460DF10601BD
:1057E0000546FFF7DFFF08B900200EE00DF10701C5
:1057F0002846FFF7D7FF0028F6D09DF807209DF830
:10580000063043EA02232380012003B030BD0000AC
:105810002DE9F0411549164804F058F80446F8B14E
:10582000144FDFF8588000256368013B002BAEB2AF
:10583000636009DA2146386805F03CF8431C08D05B
:1058400008F806000135EFE723685A1C2260187833
:10585000F6E7094B1E802046BDE8F04103F07CBE10
:105860000348BDE8F04104F0FBBD00BFB4CB000825
:105870004A390020BC00002028370020643A00206C
:1058800038B50C4605460146E0B204F05DF82946FD
:10589000200ABDE8384004F057B8000070B506464D
:1058A0000C464FF6FF711546FFF7EAFF20463146DA
:1058B00004F04AF8054B00241D44285D31460134AC
:1058C00004F042F8B4F5804FF7D170BD643A00207F
:1058D000FE292AD1C043C3B2D8074ABF164AFF20C7
:1058E0001078990742BF144A527810405A0742BFB5
:1058F000114A92781040190742BF0F4AD2781040DF
:10590000DA0642BF0C4A12791040990642BF0A4A91
:10591000527910405A0642BF074A927910401B063E
:1059200009D5054BDB79184070471F2902D1034B7D
:1059300018787047FF207047530000204839002036
:10594000024A937943F0100393717047F01A0020D4
:10595000C1F30B010A44C0F30B000244D30401D588
:10596000FFF7EEBF024A937923F01003937170475B
:10597000F01A002000F00F0001F00F01401A821A07
:10598000D30601D5FFF7DCBF024A937923F0100359
:1059900093717047F01A002001F00F010A4400F0E3
:1059A0000F000244D30601D5FFF7CABF024A93791C
:1059B00023F0100393717047F01A00204A40D30B74
:1059C000064B9A7905D14840010402D542F0040201
:1059D00001E022F004029A71704700BFF01A002023
:1059E000054B9A7910F4803F14BF42F0010222F077
:1059F00001029A71704700BFF01A002070B5224C66
:105A000014F8101004EB4000437843EA01211F4BC7
:105A10001E781F4B76B11A68207A0F321A60637AAB
:105A200043EA002045180022FFF792FF2B0A237259
:105A300065721DE0174A186812786AB10F30186055
:105A4000E37AA07A43EA002045183246FFF780FF48
:105A50002B0AA372E5720BE00B3018606379207992
:105A600043EA00204518FFF773FF2B0A2371657185
:105A7000A379284623F00203A371FFF7B1FF064A7A
:105A800013880133138070BDF01A00203C370020CA
:105A90000C1B0020021B00202237002070B5214B78
:105AA000214C1E782149224B7EB11A68207A098840
:105AB0000F321A60637A43EA002045180022FFF78C
:105AC00047FF2B0A237265721FE01A4A1868127882
:105AD00072B10F301860E37AA07A098843EA002097
:105AE00045183246FFF734FF2B0AA372E5720CE02B
:105AF0000B30186063792079098843EA0020451843
:105B0000FFF726FF2B0A23716571A379284623F03E
:105B10000203A371FFF764FF074A13880133138060
:105B200070BD00BF3C370020F01A0020FE1A002094
:105B30000C1B0020021B00202237002038B5204B10
:105B4000204C1878204B78B11A68217A0F321A60ED
:105B5000637A43EA01214D0000220846FFF7F8FE70
:105B60002B0A237265721FE0184A1968127872B105
:105B70000F311960E37AA17A43EA01214D00024610
:105B80000846FFF7E5FE2B0AA372E5720CE00B3125
:105B900019606379217943EA01214D000846FFF736
:105BA000D7FE2B0A23716571A379284623F00203DF
:105BB000A371FFF715FF064A13880133138038BD20
:105BC0003C370020F01A00200C1B0020021B002094
:105BD000223700200E4B9A7910F4803F14BF42F018
:105BE000010222F001029A7182B21AB19A7922F06E
:105BF000400202E09A7942F040029A719A790104D7
:105C00004CBF62F07F0202F07F029A71704700BFC2
:105C1000F01A0020F8B5194A194C136807460F33DB
:105C20007E0013602079637914F81710A279013689
:105C300043EA0020A35D43EA0121451802F0010276
:105C40001544FFF785FE14F817006379A25D2179EA
:105C500042EA002243EA01212846FFF7AFFE2B0A61
:105C6000284623716571FFF7B5FFA379054A23F034
:105C70000203A371138801331380F8BD0C1B0020AD
:105C8000F01A002022370020F8B5214A214C136871
:105C900014F81010A7790F334600136001362279EB
:105CA000637943EA0223A25D42EA01215D1AC3F34C
:105CB0000B02C1F30B0307F0010ED31ACEEB030363
:105CC000DB04CEEB050502D5FFF73AFE02E027F034
:105CD0001007A77114F81020A35D217943EA02226E
:105CE0006379D24392B243EA01212846FFF766FE68
:105CF0002B0A284623716571FFF76CFFA379064ACA
:105D000043F00203A371138801331380F8BD00BF71
:105D10000C1B0020F01A00202237002038B50D4A55
:105D200013680A3313600D460446FFF703FB0A4B62
:105D30009A79012303FA05F1114014B1B1FA81F106
:105D40004909064B09B1188038BD1A8801321A80FA
:105D500038BD00BF0C1B0020F01A002022370020A5
:105D600010B50D4B9A79012303FA01F1114010B1DE
:105D7000B1FA81F14909094B094C1A6829B10B3272
:105D80001A60FFF701FB208010BD05321A602388DE
:105D90000133238010BD00BFF01A00200C1B00202F
:105DA0002237002030B5164B164C1D78164B2DB1FE
:105DB000196817311960217A637A07E0134D2D783D
:105DC0005DB1196817311960A17AE37A43EA0123BA
:105DD0001A4492B202800E4B0AE006291A6809D1D1
:105DE0000F321A602279637943EA0223084A03805A
:105DF000D35C02E008321A60635C837030BD00BF80
:105E00003C370020F01A00200C1B0020021B002051
:105E1000643A002010B50B461749098881420246B2
:105E200012D8B0F5B04F05D21449088880B282422A
:105E3000FBD006E0B0F5B64F03D211480178002937
:105E4000FCD110498B5410BD0F4908680C4690B91D
:105E50000E490988B1F5804F01D2042A0BD90C49AB
:105E60000C48098804F004FB0B4B1B68986803F08E
:105E70002DFC0123236010BD283700203E38002070
:105E800024370020643A0020101B00202237002015
:105E90002037002048CE0008BC00002038B5094C4F
:105EA00005462088013880B2290A2080FFF7B2FF1A
:105EB0002088013880B22080E9B2BDE83840FFF781
:105EC000A9BF00BFFE1A002008B5094B1A680B32A3
:105ED0001A60084B13F8102003EB4003587840EA8F
:105EE0000220FFF7DBFF044A13880133138008BD4B
:105EF0000C1B0020F01A00202237002070B50E463F
:105F00000446FFF717FA0F4B9A79012303FA06F1BB
:105F10000546114014B1B1FA81F149090A4B0B4C05
:105F20001A6841B120880130113280B21A60FFF73F
:105F3000B5FF258070BD0A321A60238801332380A3
:105F400070BD00BFF01A00200C1B0020223700207B
:105F500038B5064C064A05462088136801300B33D5
:105F600080B21360FFF79AFF258038BD22370020EA
:105F70000C1B002010B50A4A136807331360094B45
:105F800013F81040D97903EB4000407840EA042030
:105F9000FFF740FF044A13880133138010BD00BF90
:105FA0000C1B0020F01A002022370020062A0B4686
:105FB00003D1C1B21888FFF72DBF014B9854704729
:105FC000F01A002070B50F4B1A6814321A6006469A
:105FD000FFF7B0F90C4B13F8164003EB46030546E8
:105FE0005B7843EA042424B2E1B2FFF713FF681C94
:105FF000C4F3072180B2FFF70DFF044A1388013371
:10600000138070BD0C1B0020F01A002022370020E6
:10601000084A13680C331360074B084A5B78FE2B61
:1060200002BF074B00F0070018701388013313807C
:10603000704700BF0C1B0020F01A00202237002000
:10604000041B0020064B1A5C064B1AB19A7942F0E9
:10605000040202E09A7922F004029A71704700BFAC
:1060600048CD0008F01A00204A40D309064B9A791F
:1060700005D14840010602D542F0040201E022F0B9
:1060800004029A71704700BFF01A0020D243D2B2C6
:10609000FFF7EABF094B9A7910F0FF0F14BF22F007
:1060A000400242F040029A719A7901064CBF62F0B8
:1060B0007F0202F07F029A71704700BFF01A002041
:1060C00010B5214A214C136804331360A379D80614
:1060D00007D4E27902F00F02092A8CBF06220022BF
:1060E00000E00622D90702D4E179992904D9603267
:1060F00043F00103D2B2A371A379144903F0120053
:1061000002280CD01228C87900F00F0002D105280F
:1061100005D801E0092802D943F0100301E023F07B
:1061200010038B71A379E0799B074ABF801A80180E
:1061300080B2E071FFF7AEFFE079FFF783FF044A1A
:1061400013880133138010BD0C1B0020F01A0020AF
:106150002237002070B51B4B1A781B4B04463AB10E
:106160001A6808321A60031F012B10D8043409E0A2
:10617000164A127842B11A6808321A60031F012BBE
:1061800005D80634E4B202E01A6804321A60104DF1
:10619000285D461EB6B200220121FFF7EBFBFE226E
:1061A000295D3046FFF760FF30462E55FFF772FF3E
:1061B000AB79084A43F00203AB71138801331380B3
:1061C00070BD00BF3C3700200C1B0020021B0020CC
:1061D000F01A00202237002038B50C4A0C4C136806
:1061E00061780C33054620781360FFF771FB60552A
:1061F000FFF750FFA37923F00203A371605DFFF75F
:1062000021FF044A13880133138038BD0C1B002082
:10621000F01A00202237002070B51A4B1A781A4B5A
:1062200004463AB11A6808321A60031F012B10D8CD
:10623000043409E0154A127842B11A6808321A602B
:10624000031F012B05D80634E4B202E01A680432B9
:106250001A600F4D285D0022461C0121FFF79CFBB0
:106260000122295D3046FFF7FFFE2E55AB793046FF
:1062700023F00203AB71FFF70DFF064A13880133C9
:10628000138070BD3C3700200C1B0020021B002037
:10629000F01A002022370020F8B5204B204D1A7844
:1062A000204B3AB11A6817321A60FFF761F82C7A5E
:1062B0006B7A09E01C4A12785AB11A6817321A60D0
:1062C000FFF756F8AC7AEB7A43EA0424204484B210
:1062D00006E01A682C790B321A606B7943EA0424C1
:1062E000124B1F5D00227E1C01213846FFF754FB34
:1062F000012239463046FFF7B7FEF1B22046FFF7DC
:1063000089FDAB79304623F00203AB71FFF7C2FE83
:10631000074A138801331380F8BD00BF3C370020C3
:10632000F01A00200C1B0020021B0020643A002001
:1063300022370020F8B5204B204D1A78204B3AB177
:106340001A6817321A60FFF713F82C7A6B7A09E093
:106350001C4A12785AB11A6817321A60FFF708F807
:10636000AC7AEB7A43EA0424204484B206E01A684B
:106370002C790B321A606B7943EA0424124B1F5DAF
:106380007E1EB6B2002201213846FFF7F3FAFE2244
:1063900039463046FFF768FEF1B22046FFF73AFD76
:1063A0003046FFF777FEAB79084A43F00203AB7142
:1063B000138801331380F8BD3C370020F01A002009
:1063C0000C1B0020021B0020643A00202237002012
:1063D0000D4B9A7910F4807F14BF42F0010222F035
:1063E00001029A719A7910F0FF0F14BF22F0400257
:1063F00042F040029A719A7901064CBF62F07F0226
:1064000002F07F029A717047F01A002070B5204B9D
:10641000204C1A78204B3AB11A6813321A60FEF7F2
:10642000A7FF227A637A09E01C4A12785AB11A68E7
:1064300013321A60FEF79CFFA27AE37A43EA022342
:10644000184480B206E01A68207907321A6063792E
:1064500043EA0020124BA2791E5CE07902F00102AF
:10646000851915443146FFF797FA3246E1792846F7
:10647000FFF7FAFD2846E571FFF7AAFFA379094A5D
:1064800023F00203A37113880133138070BD00BF92
:106490003C370020F01A00200C1B0020021B0020BB
:1064A000643A002022370020F8B51F4B1F4C1A78A1
:1064B0001F4B3AB11A6813321A60FEF759FF227A5D
:1064C000637A09E01B4A12785AB11A6813321A60CB
:1064D000FEF74EFFA27AE37A43EA0223184480B221
:1064E00006E01A68207907321A60637943EA0020CF
:1064F000114B1D5CE0794719BEB200222946FFF717
:106500004BFA2A46E1793046FFF7AEFD3046E77197
:10651000FFF75EFFA379094A23F00203A3711388F2
:1065200001331380F8BD00BF3C370020F01A002073
:106530000C1B0020021B0020643A002022370020A0
:10654000F8B51F4B1F4C1A781F4B3AB11A6813321B
:106550001A60FEF70DFF227A637A09E01B4A12786F
:106560005AB11A6813321A60FEF702FFA27AE37A70
:1065700043EA0223184480B206E01A682079073201
:106580001A60637943EA0020114B1D5CE079471BD8
:10659000BEB200222946FFF7EDF92A46E1793046DE
:1065A000FFF774FD3046E771FFF712FFA379094A40
:1065B00043F00203A371138801331380F8BD00BFB9
:1065C0003C370020F01A00200C1B0020021B00208A
:1065D000643A00202237002070B5204B204C1A78F6
:1065E000204B3AB11A6813321A60FEF7C1FE227AC4
:1065F000637A09E01C4A12785AB11A6813321A6099
:10660000FEF7B6FEA27AE37A43EA0223184480B288
:1066100006E01A68207907321A60637943EA00209D
:10662000124BA2791E5CE07902F00102851BAD1AC3
:10663000ADB23146FFF79EF93246E1792846FFF7C1
:1066400025FD2846E571FFF7C3FEA379084A43F00C
:106650000203A37113880133138070BD3C370020FF
:10666000F01A00200C1B0020021B0020643A0020BE
:1066700022370020F7B5954B954C1B78954913B9F7
:10668000954B1A785AB1FEF773FE238801339BB2FB
:106690002380CB5C024603F00705062107E0238830
:1066A00001339BB22380CB5C03F007010D4603F05E
:1066B000F800182871D007D8082844D0102858D0DE
:1066C000002840F0C3802CE028287CD013D8202854
:1066D00040F0BC80814E01A8FFF764FB9DF8067076
:1066E000B37917F0800F14BF43F0010323F00103C7
:1066F000B3717F009DE030287CD0382840F0A68020
:10670000764E01A8FFF74EFB9DF80670B37917F09F
:10671000010F14BF43F0010323F00103B3717F089D
:1067200087E001A8FFF73EFB9DF806606B4F16F06F
:10673000800F4FEA460603D046F00106F6B20FE09E
:1067400006F0FE0610E001A8FFF72CFB9DF806609E
:10675000624F16F0010F4FEA560605D046F080064C
:10676000BB7943F0010302E0BB7923F00103BB7165
:1067700052E05A4F01A8FFF715FBBB799DF8066060
:1067800003F0010343EA460630462A4601A9FFF713
:106790000DFC3046FFF71CFE46E0504E01A8FFF707
:1067A00001FBB3799DF8062013F0010F4FEA520761
:1067B00018BF47F08007D2074CBF43F0010323F016
:1067C0000103B37135E0454F01A8FFF7EBFA9DF8DF
:1067D0000660BB7916F0010F14BF43F0010323F0EC
:1067E000010316F0800FBB714FEA560614D046F035
:1067F000800611E0394F01A8FFF7D4FA9DF8066032
:10680000BB7916F0800F14BF43F0010323F001039E
:106810007600BB7146F0010630462A4601A9FFF713
:10682000C5FB3046FFF736FCBB7923F01203BB7182
:1068300046E02A4601A93846FFF7B8FB3846FFF77D
:1068400029FCB37923F01203B37139E0C3F3C20614
:1068500003F0C003802B1AD0C02B24D0402B32D1A0
:1068600001A8FFF79FFA1D4B9DF806009A79304169
:1068700010F0010F14BF22F0440242F044029A715A
:106880009A7922F0020242F010029A7118E001A8EF
:10689000FFF788FA01209DF80630B0402A4601A98A
:1068A00023EA00000AE001A8FFF77CFA9DF8063011
:1068B0000120B04018432A4601A980B2FFF776FBB9
:1068C00023880133238003B0F0BD00BF3C37002094
:1068D00022370020643A0020021B0020F01A00201A
:1068E0002DE9F74F8E4C8F4D23885A1C92B222808F
:1068F000A95CA1F140027B2A00F24B85DFE812F08F
:106900007C007E00810083008500A6000A01AB00A8
:10691000B500BB00C200C4008500C6004A01CB0020
:10692000D000D200D500DB008500A600DF01E10029
:10693000EB00ED00F000F6008500A6001802FC0058
:1069400001010301060108018500A6000A011A01E0
:106950003E014001430145018500A6004A014F0167
:10696000810196019801CD018500A600DF0149054E
:10697000E401E601E9010D028500A60018024905BF
:106980004905490549054905490549054905490597
:106990004905490549054905490549054905490587
:1069A0004905490549054905490549054905490577
:1069B0004905490549054905490549054905490567
:1069C0001D028602AE02C502490549054905490571
:1069D0004A02E8022E0351034905490549054905C4
:1069E0007803A603E203080449054905490549055A
:1069F00037047604CF04F804002037E04A4B1878B7
:106A00003BE0002052E0002056E0474D474AE9793C
:106A10001368802903F10803136008BFAB79C1F143
:106A200000064FF0000208BF43F00403B6B2104660
:106A300008BFAB71FEF79EFF3046EA790021FFF7F1
:106A400025FB3046EE71FFF7C3FC21E103B0BDE842
:106A5000F04FFEF799BE35490A6809320A60324A9A
:106A6000D179334A117000F08FBC012003B0BDE82A
:106A7000F04FFFF7B1BB2C4B587803B0BDE8F04F97
:106A8000FFF7C6BA00202CE0002030E003B0BDE8DC
:106A9000F04FFEF779BE03B0BDE8F04FFEF74CBEF5
:106AA0000220E3E7204B9878E7E7012003B0BDE838
:106AB000F04FFFF7E9B8012003B0BDE8F04FFFF752
:106AC00081BA1A490A6809320A60194A1178164AC5
:106AD000D17100F059BC0320C8E7134BD878CCE73C
:106AE000012003B0BDE8F04FFFF794B8012003B0D8
:106AF000BDE8F04FFEF7F2BC03B0BDE8F04FFEF783
:106B00001BBE0420B2E7084B1879B6E70220CDE798
:106B10000220D1E703B0BDE8F04FFEF777BC00BF1D
:106B200022370020643A0020F01A00200C1B0020BD
:106B30004A3A0020B24EB34F737930793A6843EA4B
:106B40000020F3792D5C03F00F032909123241EA8A
:106B500003113A60FFF75EF9F07905F00F0320F0BA
:106B60000F001843F071B37910B943F0400301E00E
:106B700023F04003B371FFF765FA3CE1052075E7A8
:106B80009F4B587979E70220ABE703B0BDE8F04F9F
:106B9000FEF7C0BC03B0BDE8F04FFEF737BC984E1F
:106BA00073793079F17943EA0020964B2D5C1A68AD
:106BB00001F00F0141EA05111232C9B21A60FFF764
:106BC00029F9F379B27923F00F0343EA15135BB285
:106BD000D8B2F071314610B942F0400201E022F023
:106BE00040028A71002B8B79B4BF63F07F0303F0FE
:106BF0007F038B71FFF726FA8B7923F012038B71D9
:106C00004AE3804A7E4D1368697828780C33136014
:106C1000FEF75EFE064680B2FFF73CFAAB793046DF
:106C200023F00203AB71FFF70DFA35E3002024E7F0
:106C3000744A734D13687449A8790F880F33136031
:106C40002A796B7943EA0223DE1BC3F30B02C7F3F5
:106C50000B0300F0010ED31ACEEB0303DB04CEEBE3
:106C6000060602D5FEF76CFE02E020F01000A871C7
:106C70000A886B792979D24343EA0121304692B2DE
:106C8000FEF79CFE330A30462B716E71FEF7A2FFB1
:106C9000AB7943F00203AB71FEE2FEF74BFB594ABE
:106CA000136814331360584B1E880546F1B2FFF782
:106CB000B1F8681C310A80B2FFF7ACF8ECE203B01F
:106CC000BDE8F04FFEF790BB0720CFE64C4BD879DC
:106CD000D3E64C4A4A4D13684B4F287939880F3315
:106CE00013606B79AA7943EA0020461802F001028A
:106CF0001644FEF72DFE6B7929793A8843EA012183
:106D00003046FEF75BFE330A30462B716E71FEF79C
:106D100061FFAB7923F00203BDE73A4A13681433ED
:106D20001360FEF707FBFEF7F9FA374B1880B3E262
:106D300003B0BDE8F04FFEF77BBB314E314A7378AC
:106D400096F80090B77896F8048043EA0929F3781A
:106D500043EA0727737943EA0828136815F80810EF
:106D6000103338461360FFF755F809F1FF339BB233
:106D70000137BFB21A0A08F101081FFA88F8327009
:106D80003A0AB2704FEA18227370F770327186F8BF
:106D900005802AE01A4E1B4A737896F8009096F800
:106DA0000280377943EA0929F37843EA082873799E
:106DB00043EA07271368E95D103340461360FFF785
:106DC00029F809F1FF339BB208F1FF381FFA88F860
:106DD0001A0A013FBFB232704FEA1822B2703A0A63
:106DE000737086F8038032717771B279002B6CD0A2
:106DF00042F00402B271B37923F012034BE200BFF8
:106E0000F01A00200C1B0020FE1A0020DFF8F88288
:106E100098F8002098F8013098F8041098F80700C6
:106E200043EA022698F80530B64A43EA0127136878
:106E3000E95D10331360451A0022FEF79BFDADB2E9
:106E400098F8062015F0800F14BF62F07F0202F060
:106E50007F02434688F80620791C60E0A94AAA4DC3
:106E600013682E7969782878103313606B7943EAB8
:106E70000626FEF72DFD01463046FEF7CBFF2A78A9
:106E8000013AD2B22A7001367EE09E499E4E0A68CF
:106E900010320A609C4A1079517941EA00215078F9
:106EA000FE2801BF685C994D00F007002870157836
:106EB0009079013DEDB2157015B940F0400001E048
:106EC00020F04000B07101318AE022F0040291E725
:106ED000DFF8348298F8002098F8013098F8041010
:106EE00098F8070043EA022698F80530854A43EAF5
:106EF00001271368E95D10331360451A0022FEF77D
:106F000039FDADB298F8062015F0800F14BF62F07D
:106F10007F0202F07F02434688F80620791E89B27C
:106F20000A0A1A71721E92B25971110A19707648C2
:106F30005A70997912B921F0040101E041F004017D
:106F400081719A7915B942F0400201E022F04002C5
:106F50009A719A7942F002029A719DE1694A6A4DEA
:106F600013682E7969782878103313606B7943EAB7
:106F70000626FEF7ADFC01463046FEF74BFF2A78A9
:106F8000013AD2B22A70013EB6B2330A2B716E7149
:106F9000AB7912B943F0400301E023F04003AB7139
:106FA00076E65849584E0A6810320A60564A1079F7
:106FB000517941EA00215078FE2801BF685C534DA9
:106FC00000F00700287015789079013DEDB215703A
:106FD00015B940F0400001E020F04000B0710139E7
:106FE00089B2080A51719179107141F00201CAE128
:106FF000454EDFF810B1737896F80080B278377993
:1070000043EA0828F37843EA022973794FF0000A2B
:1070100043EA07271FFA8AF0C3199BB24844E95C88
:1070200080B20AF1010AFEF7F5FE1FFA8AF39845CD
:10703000344805D0DBF800301533CBF80030E9E7F1
:1070400008EB090292B208EB0703BEE02E4EDFF810
:10705000B4A07378377896F8048043EA07277379E9
:1070600043EA0828B37923F04003B371B34615F817
:107070000810F079C1EB00091FFA89F90022FEF728
:1070800079FC08F10108013F19F0800F1FFA88F818
:10709000BFB2B37904D063F07F038BF8063007E00A
:1070A00003F07F038BF80630B9F1000F00F0CF80BA
:1070B000144A002F00F0D880DAF800301533CAF8EF
:1070C0000030D4E7104DDFF83C802E796B7943EA2D
:1070D0000626697828780C4FFEF7FAFB0146304601
:1070E000FEF798FE2B78074A013BDBB201362B7086
:1070F000B6B2002B00F0F180D8F800301533C8F894
:107100000030E6E70C1B0020F01A0020041B0020D2
:10711000A54AA6485179DFF8A0C292F804E00668B3
:10712000019641EA0E2E002692F801B09CF80070FC
:107130001178B046B146E2460EEB060C1FFA8CFC05
:10714000BBF1FE0F08BF15F80C7006F101065FFADF
:1071500086FC04BF07F007074FF001088C4502D0FA
:107160004FF00109E8E70139C9B24D1CEEE08E4E3F
:10717000DFF838B2737896F80080B278377943EA4E
:107180000828F37843EA022973794FF0000A43EAAA
:1071900007271FFA8AF03B1A9BB2C0EB0900E95C93
:1071A00080B20AF1010AFEF735FE1FFA8AF398450C
:1071B0007E4805D0DBF800301533CBF80030E8E727
:1071C000C8EB090292B2C8EB07030168F2701031F4
:1071D0009BB201600021317071707371110A1A0A3B
:1071E000B379B170327123F0160354E06E4EDFF8BC
:1071F000BCA17378377896F8048043EA072773793F
:1072000043EA0828B37923F04003B371B34615F875
:107210000810F079C1EB00091FFA89F90022FEF786
:10722000A9FB08F1FF38013F19F0800F1FFA88F819
:10723000BFB2B37904D063F07F038BF806300BE064
:1072400003F07F038BF80630B9F1000F04D1564AE2
:1072500043F0400393710AE0544A2FB1DAF800304A
:107260001533CAF80030D2E71368103313604FEAC1
:10727000182333713B0A33704B4A86F805807770C8
:10728000B37917B923F0040301E043F004039371C9
:10729000B37943F00203B3712388013375E0424DA3
:1072A000DFF808812E796B7943EA06266978287819
:1072B0003D4FFEF70DFB01463046FEF7ABFD2B7848
:1072C0003A4A013BDBB2013E2B70B6B22BB1D8F883
:1072D00000301533C8F80030E8E713687E711033CA
:1072E0001360330A3B71BB7943F04203BB71D3E7B0
:1072F0002D4A2E485179DFF8C0C092F804E00668A4
:10730000019641EA0E2E002692F801B09CF800701A
:107310001178B046B146E246C6EB0E0C1FFA8CFC63
:10732000BBF1FE0F08BF15F80C7006F101065FFAFD
:1073300086FC04BF07F007074FF00108614502D043
:107340004FF00109E8E70139C9B2CD43019EAE44CF
:1073500015251FFA8EFE15FB0161B9F1000F00D053
:10736000016000211170B8F1000F01D08AF800709F
:10737000016882F805E0103101604FEA1E211171A9
:10738000917941F0420191710233238003B0BDE84D
:10739000F08F074803F06CF8064B1B68986803B041
:1073A000BDE8F04F02F092B9F01A00200C1B00204B
:1073B00083CE0008BC000020041B00202DE9F04F04
:1073C000714A13780133DBB289B0102B137003922A
:1073D00008D16E4A1378B3FA83F35B0913706A4AD3
:1073E000002313706A4E6B4D33782A789A4228D066
:1073F000694A002132F81340009408461F2340F2E6
:107400003F22FDF757FF40F29F131F22202100204B
:107410000094FDF74FFF40F29F1340F23F222021DE
:107420004FF408700094FDF745FF40F2BF1300943D
:1074300040F23F224FF4D0710020FDF73BFF33783C
:107440002B70564B069301221A704FF48047BA10E6
:10745000C7F3022402F0380244EA02037C1104F06C
:10746000C0041C434E4B4F48B9B2CE0019804E4B5E
:107470004E4917F803900D78079106F0F806F308C7
:10748000E20803EB421202F5B042474BA7F58041F8
:107490009B5C65B1455C4D4509D1454D525D9A42B5
:1074A00005D1039A1278002A58D11A0656D513F03E
:1074B000800F00F801904FEAE30803F0070207D0BD
:1074C0003249097821B108F007055FFA82F802E035
:1074D00008F00708D5B25B064FEA440444BF08F140
:1074E000080808354FEA460604F1200444BF5FFA55
:1074F00088F8EDB22036284A631CB9F1000F02D19A
:1075000032F8182004E0B9F1FF0F09D132F8152044
:107510000092214606F10F023046FDF7CBFE1DE03A
:107520004FF0000A4FF0800B04920593049B19EA78
:107530000B0F06EB4A0014BF33F8153033F8183040
:10754000009380B2421C059B21460AF1010AFDF717
:10755000B1FEBAF1080F4FEA5B0BE7D10137B7F57F
:10756000B04F7FF474AF0E4B1249134800244FF410
:1075700040721C8002F09BFB069B079A1C70012343
:10758000137009B0BDE8F08FFC1A002036370020D8
:10759000041B00205100002028CD000824370020C3
:1075A0003E380020201F0020643A00204939002086
:1075B0001CC4FF1F649200201C1C00200D4A0023E5
:1075C0001360536093600C4A1360536093600B4ADE
:1075D00013800B4A13800B4A13800B4A13700B4A1B
:1075E00013700B4A13700B4A13700B4A13700B4A3B
:1075F00013607047F01A00202A370020FE1A00207E
:107600002237002020370020011B00203C370020BB
:10761000021B0020031B0020253700200C1B00202C
:10762000014B00221A70704752000020014B187065
:10763000704700BF50000020020912F0080F00F050
:107640000F004FF0010305D0064A83401078034332
:107650001370704704498340885C20EA03038B540D
:10766000704700BF4839002053000020020912F083
:10767000080F00F00F004FF0010306D0064A8340C8
:10768000107820EA03031370704704498340885C34
:1076900003438B54704700BF48390020530000203B
:1076A000F7B51B4C28B11B4B9879DD7900F0010030
:1076B00003E0A079E57900F00100174B1B68003565
:1076C00018BF0125CBB194F802E0E378277A627AFB
:1076D00012490F4E097843EA0E238DE8210042EA51
:1076E00007220F48FDF7FEFA38B10023B370F3709C
:1076F000B37943F00103B37103E0A37923F00103ED
:10770000A371FDF741FE074B188003B0F0BD00BF29
:10771000F01A00202A37002044380020403800208A
:10772000483800202237002038B5124B124C1B6815
:10773000B3B1E379207AA578E278617AA3F1FF0EFC
:10774000DEF1000343EB0E0341EA002142EA052289
:107750000A48FDF715FD18B1A37943F0010302E0D3
:10776000A37923F00103A371FDF70EFE044B1880EB
:1077700038BD00BF38370020F01A00203D37002008
:1077800022370020044A00231360044A1360044A8D
:107790001370FDF769BD00BF443800201C1F002096
:1077A0004838002038B5044603F05CFB042839D97A
:1077B000FFF7E8FF204603F055FB043825180422A4
:1077C0001949284603F056FB50B9184B18480125B3
:1077D000FF2221461D7003F071FB164B1D6038BD62
:1077E00004221549284603F045FB50B90F4B1048B9
:1077F00002221A702146FF2203F060FB01220D4B8A
:107800000FE004220D49284603F034FB50B9074B22
:10781000074803221A702146FF2203F04FFB084B52
:1078200001221A6038BD00BFB9CA000840380020E4
:107830004838002044380020BECA0008C3CA0008E7
:107840001C1F002010B5044603F00CFB04280AD9C5
:107850002146FF22044803F031FBFDF7D9FFBDE8C4
:107860001040FFF7ABBE10BD4A39002008B50146F5
:10787000034803F008F9034B01221A6008BD00BF5A
:10788000141B0020181C0020034A00231360034A25
:107890001370FDF7F5BC00BF383700203D370020DE
:1078A00010B50446FFF7F0FF204603F0DBFA04288A
:1078B00007D9FF222146034803F000FB024B0122B7
:1078C0001A6010BD3D370020383700202DE9F04FF9
:1078D000DFF878A385B0D146BA4B1A681AB10022F6
:1078E0001A60FFF76BFDB84BB84C1A68002A00F01D
:1078F000D4810026B649B7481E6001F0E7FF05466F
:10790000002800F0C7818DF809608DF80A60FFF744
:1079100055FEB149FDF746FFB0492846FDF742FF45
:10792000AF492846FDF73EFFAE492846FDF73AFF2E
:10793000AD492846FDF736FFAC492846FDF732FF32
:1079400021462846FDF748FFA9492846FDF744FF90
:10795000A8492846FDF726FF0DF10B012846FDF743
:1079600021FF0DF109012846FDF71CFF9DF80930A4
:10797000FF2B04BF01238DF809309DF8093003F077
:10798000200303F0FF064BB101219B4802F070FD7C
:107990009A4B1B68986801F099FE01269DF8093002
:1079A000974A9849C3F3420328461370FDF7FAFE3D
:1079B00095492846FDF7F6FE94492846FDF7F2FE64
:1079C00093492846FDF7EEFE92492846FDF7EAFE68
:1079D00091492846FDF7E6FE90492846FDF7E2FE6C
:1079E0008F492846FDF7DEFE8E492846FDF7DAFE70
:1079F0008D492846FDF7D6FE8C492846FDF7D2FE74
:107A00008B492846FDF7CEFE8A492846FDF7CAFE77
:107A100089492846FDF7C6FE0DF10A012846FDF703
:107A2000C1FE9DF80A20854B02B1012284491A70DB
:107A30002846FDF7B7FE0DF10A012846FDF7B2FE14
:107A40009DF80A307F4A278803F003031370002F44
:107A500040F0FE800DF10E012846FDF7BDFE5B49AA
:107A60002846FDF7B9FEBDF80E30023BADF80E30EA
:107A70003E46BDF80E20B3B29A4206F1010605D982
:107A80000DF10B012846FDF78DFEF2E700238DF87E
:107A90000C308DF80D300DF10E012846FDF79CFEDF
:107AA0000DF10D012846FDF77DFEBDF80E204FF6C5
:107AB000FF739A4205BF4FF48043ADF80E300123A7
:107AC000002300939DF80D30043BDBB2042B9ABFDA
:107AD0005D4A32F813B04FF6FF7B002637460AEBBB
:107AE0000B08BDF80E20BA4257D90DF10A012846FD
:107AF000FDF758FE009B002B40D09DF80A20ED2A90
:107B000037D10DF10A0128460192FDF74BFE9DF891
:107B10000A00019A791CED2889B21BD103A92846D5
:107B2000FDF740FE0DF10A012846FDF73BFE033745
:107B30009DF80C109DF80A00BFB200224FF6FF7EA0
:107B40008A4227DAF3451EBF08F806000136B6B2AE
:107B50000132F5E74FF6FF77BB451AD00AEB06076F
:107B600007F80B20721C92B2023608F80200B6B277
:107B70000FE04FF6FF718B4506D10BE04FF6FF7219
:107B8000934507D09DF80A2008F806200136B6B2C2
:107B900000E00F460137BFB2A3E76B68013B002B43
:107BA0006B6007DA154B2946186802F083FE431C08
:107BB0005ED003E02B685A1C2A601878294603F02F
:107BC0003FFA68E75C3A00201C1F002022370020A3
:107BD000B4CB000848380020F71A0020F61A00201D
:107BE000F11A0020F01A0020F51A0020F41A0020E3
:107BF000FE1A00204A3A0020A5CE0008BC00002052
:107C0000041B0020F31A0020F21A00202B3700205A
:107C10002A3700202D3700202C3700202F37002056
:107C20002E3700203137002030370020FB1A00208B
:107C3000FA1A0020F91A0020F81A0020011B00206F
:107C4000001B002025370020F0CE0008643A0020F9
:107C500076B90DF10A012846FDF7A4FD06F580432B
:107C600001369DF80A2003F80A20B6F5404FF0D1FE
:107C7000274B22881A80274B00261E70264B1E7029
:107C8000264B1E70264B28461E6001F065FC254BD6
:107C90001E7002E0244802F0E3FB1F4E3378002BF5
:107CA00040F015811D4B1A78002A40F010811849C8
:107CB000DFF884B023880B809BF80010F9B11949D4
:107CC0000878E0B10A708BF800201AF80320174DED
:107CD000762A02BF154A013313802088FEF7DEF8AA
:107CE000134B1B78012B02D838232B8007E0022B83
:107CF00005D1104B18780002FDF710FB288023886F
:107D000040F26252934219D10120FFF7C9FC1BE0F7
:107D100020370020031B00203C370020021B0020DE
:107D20000C1B0020263700204A3900202237002073
:107D3000253700204A3A0020011B002040F2C242B1
:107D4000934201D1FFF7F0FC634D2B781BB9FBF791
:107D50004DFA01232B70614B1B68002B00F0B7809C
:107D60005F49604801F0B2FD0546002800F0AC8094
:107D70005D4F5E4B0146F87993F8008001F0E4FD19
:107D80002946B87901F0E0FD2946787801F0DCFD5C
:107D90002946387801F0D8FD2946787901F0D4FDDC
:107DA0002946387901F0D0FD00212846FDF768FD0D
:107DB0004F4B28461988FDF763FD4E4B294618782E
:107DC00001F0C2FD4FEA48082946002001F0BCFD41
:107DD000294608F0FE0001F0B7FDDFF82881F878A9
:107DE000294601F0B1FD2946B87801F0ADFD2946DC
:107DF00098F8010001F0A8FD294698F8000001F06C
:107E0000A3FD294698F8030001F09EFD294698F845
:107E1000020001F099FD294698F8050001F094FD53
:107E2000294698F8040001F08FFD294698F80700CC
:107E300001F08AFD294698F8060001F085FD2946E3
:107E4000F87A01F081FD2946B87A01F07DFD2946D6
:107E5000787A01F079FD2946387A01F075FD2946D6
:107E60009BF8000001F070FD234B2946187801F0C3
:107E70006BFD224B2946187801F066FD3621284615
:107E8000FDF7FEFC21882846FDF7FAFC3427013F68
:107E900029460020BFB201F057FD002FF7D14FF463
:107EA000004204212846FDF7F9FC4FF44042052129
:107EB0002846FDF7F3FC28464FF480420821FDF7E1
:107EC000EDFC284601F048FB044A00231360238898
:107ED0000B4D1AF8031017E052000020181C002068
:107EE00025CD0008141B0020F01A0020041B0020E0
:107EF000FE1A00204A3A0020001B002025370020EF
:107F00000C1B00202A370020FF2901F25382DFE8F2
:107F100011F0000107010C01110116011B012001E4
:107F20002501430158015D01620167016C01710186
:107F300076019401AD01B201B701BC01C101C601D6
:107F4000CB01E701F201F701FC01010206020B027D
:107F50001002310237025F028902C102C602CB025F
:107F6000D002D402DA02DE02E202120317031C037B
:107F7000210330033603420350035B035F036303B3
:107F80008F039D03A303A703B503C003C503CA035F
:107F9000CF03E303E303E303E303E303E303EA03BE
:107FA000E303EF03EF03EF03EF03EF03EF03F60346
:107FB000EF03FB03FB03FB03FB03FB03FB030204D5
:107FC000FB030704070407040704070407040E045F
:107FD00007041304130413041304130413041A04EE
:107FE00013042504250425042504250425042C0454
:107FF00025043104310431043104310431045C04BA
:108000003104610461046104610461046104680471
:1080100061046D046D046D046D046D046D04AE04A3
:108020006D04B204B204B204B204B204B204F404A3
:10803000B204F804F804F804F804F804F804390564
:10804000F8043D053D053D053D053D053D05820521
:108050003D05860586058605860586058605BC05DB
:108060008605F205F205F205F205F205F205210694
:10807000F20555065506550655065506550683065E
:108080005506B606B606B606B606B606B606F70630
:10809000B606330738073C07410748074D07510725
:1080A000750779077E0785078A078D0792079F075F
:1080B000C307C707CC07D007D507E707EC07F007CA
:1080C000140818081D083D0842085108560863089E
:1080D0008E0892089708BB08C008FF080409230906
:1080E0003B093F0944095F096409730978097B0961
:1080F000920996099B09A809AD09B609BB09D109DE
:10810000E809EC09F1090F0A140A1D0A220A280AD3
:108110004D0A2A68013304322A60238001F054B9E1
:108120000020FDF72BFA01F04FB90020FDF722FFE8
:1081300001F04AB90020FDF78DF901F045B90020A2
:10814000FEF76AF801F040B90020FEF703F801F0ED
:108150003BB90020FDF72CFA01F036B92A68043249
:108160002A60B84AD179907911F0800F18BF40F099
:1081700001004FEA41010CBF20F0010041F0010174
:10818000907114BFD171D1719179013321F0120135
:108190009171238001F018B92A68AA4904322A6033
:1081A000A94ACF7992F807E0887981F807E001338E
:1081B00092F806E081F806E0D7719071238001F013
:1081C00003B90020FDF71AFC01F0FEB80020FDF70E
:1081D00097FA01F0F9B80020FDF7E8F801F0F4B8DB
:1081E0000120FEF719F801F0EFB80120FDF7B2FF0A
:1081F00001F0EAB80120FDF7DBF901F0E5B82A68E3
:1082000004322A608F4AD179907911F0010F18BF9A
:1082100040F001004FEA51010CBF20F0010061F075
:108220007F01907114BFD171D1719179013321F027
:1082300012019171238001F0C7B8FDF799F82388E6
:10824000804C82495A1C93B22278013AD2B22270F1
:1082500032B12A6803440D322A600B8001F0B4B8B1
:108260002A680B8008322A6001F0AEB80120FDF7C1
:1082700085F901F0A9B80120FDF77CFE01F0A4B852
:108280000120FDF7E7F801F09FB80220FDF7C4FFD9
:1082900001F09AB80220FDF75DFF01F095B80220C9
:1082A000FDF786F901F090B82A6866480432C17972
:1082B0002A6082794900D70748BF41F00101614F28
:1082C000C171C9054CBF42F0010222F00102BA712E
:1082D0008279013322F012028271238001F074B896
:1082E0002B680C332B60FDF743F8238801331844C7
:1082F000208001F069B80120FDF780FB01F064B82F
:108300000120FDF7FDF901F05FB80120FDF74EF8FF
:1083100001F05AB80320FDF77FFF01F055B80320A4
:10832000FDF718FF01F050B80320FDF741F901F007
:108330004BB82A684348434F817990F807E00432EC
:108340002A60C27911F0010F4FEA520218BF42F0C1
:1083500080021EF0010F14BF41F0010121F0010164
:10836000B971C2718279013322F0120282712380C5
:1083700001F02AB806210120FDF78AF801F024B89F
:10838000337830494BB12B680E332B60FCF7E4FF98
:108390004872FCF7E1FF087215E02D4B1B784BB1DA
:1083A0002B680E332B60FCF7D7FFC872FCF7D4FFA5
:1083B000887208E02B680A332B60FCF7CDFF487108
:1083C000FCF7CAFF087123880133238000F0FCBF4B
:1083D000FCF7B0FF32781B4B074632B12A68597A56
:1083E00093F8088014322A600FE0194A127832B1EB
:1083F0002A68D97A93F80A8014322A6005E02A683C
:10840000597993F8048010322A603846FDF702FD4E
:10841000781C414680B2FDF7FDFC238801332380A0
:1084200000F0D2BF3178074AA1B12968107A0A3129
:108430002960517A41EA0021013189B2080A10729B
:10844000517223E0F01A00202A3700202237002042
:10845000021B0020BE49097861B12968907A0A316F
:108460002960D17A41EA0021013189B2080A90726B
:10847000D1720BE02968107906312960517941EAFF
:108480000021013189B2080A107151710133238032
:1084900000F09ABF0420FDF7BFFE00F095BF042056
:1084A000FDF758FE00F090BF0420FDF781F800F0C2
:1084B0008BBFFDF705FE00F087BF06210020FCF70B
:1084C000E7FF00F081BFFDF739FB00F07DBFFDF74E
:1084D00021F800F079BF31789E4A61B12968107A9D
:1084E0000A312960517A41EA0021013989B2080A2A
:1084F000107251721BE09649097861B12968907A2F
:108500000A312960D17A41EA0021013989B2080A89
:108510009072D1720BE02968107906312960517987
:1085200041EA0021013989B2080A10715171013301
:10853000238000F049BF0520FDF76EFE00F044BF28
:108540000520FDF707FE00F03FBF0520FDF730F8DE
:1085500000F03ABF2A6804322A607E4AD179C943C2
:10856000D1719179013341F012019171238000F0B2
:108570002BBF00210120FCF78BFF00F025BF2B68EB
:108580000A332B60FCF7D6FE734B18802388013327
:10859000238000F019BF2B680D332B60FCF7CAFE57
:1085A0006C4BD979FDF736FC23880133238000F02A
:1085B0000BBF2A68684906322A600A8801330132F3
:1085C0000A80238000F000BFFDF766FE00F0FCBECD
:1085D000FDF7B0FE00F0F8BE33785E493BB12B6882
:1085E00013332B60FCF7C4FE0F7A4B7A09E0584B2B
:1085F0001B785BB12B6813332B60FCF7B9FE8F7AC5
:10860000CB7A43EA0727384487B206E02B680F7914
:108610000A332B604B7943EA0727FCF79DFEC1B272
:108620003846FDF7F7FB23880133238000F0CCBEEA
:108630002A68484904322A608A7922F0120242F0FC
:10864000010201338A71238000F0BEBE002108467A
:10865000FCF71EFF00F0B8BEFDF720FA00F0B4BE34
:108660002B680D332B60FCF765FE3A4B19F80020A0
:10867000DA7123880133238000F0A6BE2A683649C8
:1086800006322A600A880133013A0A80238000F00A
:108690009BBE0720FDF7C0FD00F096BE0720FDF74A
:1086A00059FD00F091BE0720FCF782FF00F08CBE60
:1086B0002A68284904322A608A79D0074CBF22F000
:1086C000010242F001028A718A79013322F002022A
:1086D0008A71238000F078BE01F007010020FCF7CA
:1086E00099FF00F071BE0020FCF7D0FF00F06CBED7
:1086F00001F007010120FCF78DFF00F065BE0120AD
:10870000FCF7C4FF00F060BE01F007010220FCF797
:1087100081FF00F059BE0220FCF7B8FF00F054BE04
:1087200001F007010320FCF775FF00F04DBE0320A8
:10873000FCF7ACFF00F048BE01F007010420FCF795
:1087400069FF00F041BE0420FCF7A0FF00F03CBE32
:10875000021B0020F01A0020FE1A002001F0070181
:108760000520FCF757FF00F02FBE0520FCF78EFF19
:1087700000F02ABE3378B04F01F007013BB12B68FF
:1087800013332B60FCF7F4FD3A7A7B7A09E0AB4BAC
:108790001B785BB12B6813332B60FCF7E9FDBA7AC9
:1087A000FB7A43EA0223184480B206E02B6838794A
:1087B00007332B607B7943EA0020795CFDF72AFBC5
:1087C00023880133238000F0FFBD2B6804332B6026
:1087D00000F0FABD01F007010720FCF71BFF00F0D5
:1087E000F3BD0720FCF752FF00F0EEBD337801F037
:1087F00007073BB12B6808332B603B1F012B11D8B7
:1088000004370FE08D4B1B784BB12B6808332B607E
:108810003B1FDBB2012B05D8B91DCFB202E02B689C
:1088200004332B60DFF8108298F8070018F807105F
:1088300043181FFA83FB00220093FDF7ADF818F8E8
:10884000072098F807105846FDF70EFC009B88F8A3
:1088500007305846FDF7BCFD98F8063023F00203B8
:1088600088F8063023880133238000F0ADBDFDF782
:108870001BFE00F0A9BD337801F007073BB12B6860
:1088800008332B603B1F012B11D804370FE06B4BD3
:108890001B784BB12B6808332B603B1FDBB2012BDD
:1088A00005D8B91DCFB202E02B6804332B60DFF886
:1088B000888198F8070018F8071098F8062000EB50
:1088C000010B02F001029344FDF766F818F8072047
:1088D00098F807105846FDF7C7FB584688F807B0C8
:1088E000FDF776FD98F8063023F0020388F806308D
:1088F00023880133238000F067BDFDF787FD00F07A
:1089000063BD337801F007073BB12B6808332B6058
:108910003B1F012B11D804370FE0484B1B784BB19C
:108920002B6808332B603B1FDBB2012B05D8B91D28
:10893000CFB202E02B6804332B60DFF8FC8098F89C
:10894000070018F80710431A1FFA83FB0022009350
:10895000FDF710F818F8072098F807105846FDF7AB
:1089600095FB009B88F807305846FDF731FD98F8D5
:10897000063043F0020388F8063023880133238051
:1089800000F022BDFDF7DCFD00F01EBD337801F0E4
:1089900007073BB12B6808332B603B1F012B11D815
:1089A00004370FE0254B1B784BB12B6808332B6045
:1089B0003B1FDBB2012B05D8B91DCFB202E02B68FB
:1089C00004332B60DFF8708098F8070018F8071060
:1089D00098F80620C1EB000B02F00102C2EB0B0B72
:1089E0001FFA8BFBFCF7C6FF18F8072098F8071052
:1089F0005846FDF74BFB584688F807B0FDF7E8FCF2
:108A000098F8063043F0020388F8063023880133D3
:108A1000238000F0D9BCFDF7DFFD00F0D5BC337832
:108A200001F0070163B12B6808332B600B1F012B8A
:108A300016D8043114E000BFF01A0020021B0020F9
:108A40009B4B1B784BB12B6808332B600B1FDBB2A1
:108A5000012B05D80631C9B202E02B6804332B6024
:108A6000944F7B5CF8791840F871FDF713FBBB79E4
:108A7000F87923F0030343F01003BB71FDF7E2FA2A
:108A800023880133238000F09FBC3378894F3BB1AA
:108A90002B6813332B60FCF76BFC3A7A7B7A09E086
:108AA000834B1B785BB12B6813332B60FCF760FCA6
:108AB000BA7AFB7A43EA0223184480B206E02B68B4
:108AC000387907332B607B7943EA0020FB7919F86A
:108AD00000001840F871FDF7DDFABB79F87923F052
:108AE000030343F01003BB71FDF7ACFA2388013395
:108AF000238000F069BC337801F007013BB12B689B
:108B000008332B600B1F012B11D804310FE0684B89
:108B10001B784BB12B6808332B600B1FDBB2012B8A
:108B200005D80631C9B202E02B6804332B60614FCF
:108B30007B5CF8795840F871FDF7ACFABB79F879AD
:108B400023F01303BB71FDF77DFA238801332380E3
:108B500000F03ABC3378574F3BB12B6813332B608E
:108B6000FCF706FC3A7A7B7A09E0514B1B785BB143
:108B70002B6813332B60FCF7FBFBBA7AFB7A43EAD2
:108B80000223184480B206E02B68387907332B6043
:108B90007B7943EA0020FB7919F800005840F8710E
:108BA000FDF778FABB79F87923F01303BB71FDF771
:108BB00049FA23880133238000F006BC337801F0A2
:108BC00007013BB12B6808332B600B1F012B11D819
:108BD00004310FE0364B1B784BB12B6808332B6008
:108BE0000B1FDBB2012B05D80631C9B202E02B689E
:108BF00004332B602F4F7B5CF8791843F871FDF735
:108C000049FABB79F87923F01303BB71FDF71AFA1F
:108C1000238801332380D7E33378264F3BB12B6879
:108C200013332B60FCF7A4FB3A7A7B7A09E0204BE4
:108C30001B785BB12B6813332B60FCF799FBBA7A76
:108C4000FB7A43EA0223184480B206E02B683879A5
:108C500007332B607B7943EA0020FB7919F8000089
:108C60001843F871FDF716FABB79F87923F013036E
:108C7000BB71FDF7E7F9238801332380A4E3337840
:108C800001F007073BB12B6808332B603B1F012B1A
:108C900015D8043713E0064B1B786BB12B680833EB
:108CA0002B603B1FDBB2012B09D8B91DCFB206E008
:108CB000021B0020F01A00202B6804332B60DFF821
:108CC000088398F8070018F80710C1EB000B1FFA8B
:108CD0008BFB0022FCF74EFE18F8072098F80710CF
:108CE0005846FDF7D3F95846FDF772FB98F8063061
:108CF00043F0020388F8063023880133238063E3BE
:108D00003378B14F3BB12B6813332B60FCF730FB4A
:108D10003A7A7B7A09E0AD4B1B785BB12B68133351
:108D20002B60FCF725FBBA7AFB7A43EA022318444E
:108D300080B206E02B68387907332B607B7943EAF1
:108D4000002019F80080F879C8EB000B1FFA8BFBA4
:108D500000224146FCF70EFE4246F9795846FDF7DF
:108D600095F95846FDF734FBBB7943F00203BB711C
:108D700023880133238027E306210120FCF7F0FF3D
:108D800022E30020FCF7E6FC1EE306210120FCF7AD
:108D9000C5FF19E32B680A332B60FCF7CBFA208060
:108DA00012E306210120FDF7A9F80DE30020FDF7ED
:108DB0008BF809E32B68844F07332B60FCF7CCFA60
:108DC0005FFA80F8F87900EB08031FFA83FB0022B2
:108DD00041460093FCF7E0FD4246F9795846FDF71D
:108DE00043F9009BFB715846FDF7F2FABB7923F07B
:108DF0000203BB71238801332380E5E20020FDF7E5
:108E0000A7F8E1E206210020FCF7AAFFDCE22B68CC
:108E10000A332B60FCF7B8FA2080D5E20621002047
:108E2000FCF77CFFD0E2FDF725FCCDE20621002017
:108E3000FDF764F8C8E22B6811332B60FCF77AFA6F
:108E400007462088013080B2FDF728F82780BBE272
:108E50002B685D4F07332B60FCF77EFABA795FFA17
:108E600080F8F87902F0010208EB000B93444146C8
:108E7000FCF792FD4246F9795846FDF7F5F8584659
:108E800087F807B0FDF7A4FABB7923F00203BB71A2
:108E900023880133238097E20820FDF759F893E2F5
:108EA00000210120FCF75CFF8EE20120FCF752FC60
:108EB0008AE200210120FCF731FF85E22B680B33A9
:108EC0002B60FCF749FAC0B2FE2805D13E4B404A60
:108ED000DB7903F00703137023880133238073E2E7
:108EE00000210120FDF70AF86EE20120FCF7ECFFFB
:108EF0006AE22B68344F07332B60FCF72DFA5FFAD8
:108F000080F8F879C8EB00031FFA83FB0022414682
:108F10000093FCF72FFD4246F9795846FDF7B6F865
:108F2000009BFB715846FDF753FABB7943F00203EF
:108F3000BB7123880133238046E21020FDF708F837
:108F400042E200210846FCF70BFF3DE22A681E4979
:108F500004322A601F4A087817780F70107057780B
:108F6000487850704F70887897788F709070D77865
:108F7000C878D070CF70087917790F711071577950
:108F80004879507101334F7123801DE2002108465A
:108F9000FCF7C4FE18E22B680B4F0B332B60FCF779
:108FA000DBF9C1B2F879FCF793FC2388F87101333F
:108FB000238009E200210846FCF7A0FF04E2012219
:108FC000134432702380FFE1F01A0020021B0020BE
:108FD000041B00202A3700202B68DFF8C8820733E3
:108FE0002B60FCF7B9F998F806205FFA80FB98F837
:108FF000070002F00102CBEB0007BF1ABFB25946CF
:10900000FCF7B8FC5A4698F807103846FDF73EF8CA
:10901000384688F80770FDF7DBF998F8063043F01A
:10902000020388F80630238801332380CCE118201E
:10903000FCF78EFFC8E102210120FCF791FEC3E19D
:109040003378984F43B12B680E332B60FCF79CF9B3
:10905000030A3B72787213E0934B1B7843B12B6881
:109060000E332B60FCF790F9030ABB72F87207E02D
:109070002B680A332B60FCF787F9030A3B71787180
:109080002388013323809FE102210120FCF746FE63
:109090009AE13378834F2BB12B68797A3A7A173378
:1090A0002B600DE0804B1B782BB12B68F97ABA7AD4
:1090B00017332B6004E02B6879793A7913332B60EE
:1090C0007A4B0192188800F101081FFA88F819F804
:1090D0000030009319F808B0FCF79CFE019A404656
:1090E0001146FCF797FE3278009B1AB17B7287F825
:1090F00008B009E06C4A12781AB1FB7287F80AB01E
:1091000002E07B7187F804B02388013323805BE1A0
:1091100002210120FCF7F2FE56E13278614B2AB1C0
:109120002A68187A5B7A0F322A600DE05E4A12785C
:109130002AB12A68987ADB7A0F322A6004E02A681A
:1091400018795B790B322A6043EA0020FCF7A6FE0F
:1091500023880133238037E12B68524F07332B607C
:10916000FCF7FAF8FB791840F871FCF793FFBB792C
:10917000F87923F0030343F01003BB71FCF762FF9F
:109180002388013323801FE12020FCF7E1FE1BE14F
:1091900002210020FCF7E4FD16E13378414A2BB1AF
:1091A0002B68117A08332B60537A0DE03E4B1B7805
:1091B0002BB12B68917A08332B60D37A04E02B68AB
:1091C000117904332B60537943EA01232380FBE0B8
:1091D00002210020FCF7A2FDF6E02A6804322A6092
:1091E000304AD778507911795771013397781771D0
:1091F000D07091702380E7E002210020FCF77EFE12
:10920000E2E0FDF76DFBDFE02B68264F07332B60B4
:10921000FCF7A2F8FB79584080B2F871FCF73AFFEE
:10922000BB79F87923F01303BB71FCF70BFF23889C
:1092300001332380C8E02820FCF78AFEC4E0072120
:109240000120FCF78DFDBFE02B680A332B60FCF793
:109250009BF8144B020ADA7198712388013323803A
:10926000B2E007210120FCF759FDADE02A68043285
:109270002A600F4A0021013311702380A4E00721E6
:109280000120FCF73BFE9FE02B680B332B60054B66
:10929000D8799B7943EA0020FCF700FE238801334C
:1092A000238091E0F01A0020021B0020FE1A00200B
:1092B000011B00202B685D4F07332B60FCF74CF837
:1092C000FB79184380B2F871FCF7E4FEBB79F879BA
:1092D00023F01303BB71FCF7B5FE23880133238011
:1092E00072E03020FCF734FE6EE007210020FCF72E
:1092F00037FD69E031784D4A4D4829B129680A3176
:109300002960117A527A0DE04A49097829B1296811
:109310000A312960917AD27A04E0296806312960FD
:109320001179527942EA01220133028023804BE015
:1093300007210020FCF7F2FC46E02A6804320121F4
:109340002A603D4A0B44117023803DE00721002034
:10935000FCF7D4FD38E00121364A0B44117023801C
:1093600032E02B68DFF8C48007332B60FBF7F4FF93
:10937000C7B298F80700C7EB000B1FFA8BFB00225F
:109380003946FCF7F7FA3A4698F807105846FCF7C2
:109390007DFE5846FDF71CF898F8063043F00203AE
:1093A00088F806302388013323800DE03820FCF74D
:1093B000CFFD09E0214B22481A8801F059F8214BD2
:1093C0001B68986800F082F9337813B9194B1B7841
:1093D0004BB11D4B1A7822B11649002232700A7027
:1093E00000E001221A702B6848F2373293427EF671
:1093F00073AA164A1648A3F50343373B1360154A70
:109400001368643301688B42FCD8114B1B681360EE
:10941000114A13680133022B13607EF45DAA002306
:1094200013600E4B01221A70FEF756BAF01A002094
:10943000FE1A0020021B0020011B00202037002004
:10944000C4CE0008BC000020031B00200C1B002021
:10945000603A0020141C0020081B00202637002042
:1094600008B5FF220449054801F028FDFCF7D0F9B2
:10947000FEF7A4F8FEF72AFAE9CE00084A390020E0
:10948000014B1868704700BFBC00002008B5074BAF
:10949000044613B10021AFF30080054B1868836ABE
:1094A00003B19847204602F0C7F900BF0000000052
:1094B00060CF000870B505460C4609B9002070BDA4
:1094C00018B183690BB900F053F9204B9C4201D1CC
:1094D0006C6808E01E4B9C4201D1AC6803E01D4B58
:1094E0009C4208BFEC68B4F90C30002BE6D0214652
:1094F000284600F039F8236B064633B1216A284626
:1095000098470028B8BF4FF0FF36A3891B0603D544
:109510002169284600F0DEFB616B41B104F1440390
:10952000994202D0284600F0D5FB00236363A16C6A
:1095300021B1284600F0CEFB0023A36400F084F99B
:109540000023A38100F081F9304670BDFCCE0008F5
:109550001CCF00083CCF0008024B01461868FFF7FB
:10956000A9BF00BFBC0000208A892DE9F041054653
:1095700010070C4659D44B68002B02DC0B6C002BF7
:1095800017DDE66AAEB102F48052002392B22F6872
:109590002B600AB1606D15E0216A01232846B047AF
:1095A000411C0FD12B686BB11D2B01D0162B03D1A1
:1095B0002F600020BDE8F081A38943F04003A38120
:1095C000BDE8F081A3895A0705D56368C01A636BAB
:1095D0000BB1236CC01A00230246E66A216A2846B2
:1095E000B047431CA38906D129681D293AD8214ACE
:1095F000CA40D60736D500226260D90422692260AB
:1096000004D5421C01D12B6803B96065616B2F60E2
:109610000029CED004F14403994202D0284600F03C
:1096200059FB00206063BDE8F0810F69002FC0D0B6
:1096300093070E6808BF4B690F6018BF0023C7EB84
:1096400006088B6002E00744C0EB0808B8F1000F81
:10965000AFDD43463A46216AA66A2846B04700284D
:10966000F1DCA38943F04003A3814FF0FF30BDE854
:10967000F08100BF0100402038B50B6905460C465B
:10968000DBB118B183690BB900F072F80C4B9C4246
:1096900001D16C6808E00B4B9C4201D1AC6803E03F
:1096A000094B9C4208BFEC68B4F90C302BB1214641
:1096B0002846BDE83840FFF757BF002038BD00BF3F
:1096C000FCCE00081CCF00083CCF0008014620B9A2
:1096D000044B0549186800F037BA044B1868FFF7C7
:1096E000CBBF00BF60CF000879960008BC00002007
:1096F000014900F029BA00BF79960008002310B58F
:10970000044603604360836081814366C2810361D4
:1097100043618361194608225C3000F0D3FA054B9F
:109720006362054BA362054BE362054B246223632E
:1097300010BD00BF91A90008B3A90008EBA900085B
:109740000FAA000870B568234D1E5D430E4605F153
:10975000740100F00DFB044640B1002180E8420096
:109760000C30A06005F1680200F0ACFA204670BD34
:10977000836910B5044633BB8364C3640365124B2D
:10978000124A1B688262984204BF0123836100F081
:109790001FF86060204600F01BF8A060204600F033
:1097A00017F80022E06004216068FFF7A7FF01229C
:1097B0000921A068FFF7A2FF02221221E068FFF74B
:1097C0009DFF0123A36110BD60CF0008F196000842
:1097D000F8B51C4B1E68B369074613B93046FFF74E
:1097E000C7FF4836B4687368013B04D4B4F90C5021
:1097F0007DB16834F8E733680BB13668F2E70421CD
:109800003846FFF79FFF30600028F6D10C233B60FD
:10981000F8BD4FF6FF73E3810123A38165662560E0
:10982000A560656025616561A5610822294604F18E
:109830005C0000F047FA6563A563A564E564204613
:10984000F8BD00BF60CF000870477047F7B50F46FE
:10985000114601AA054601F0DFFC064608B90020C2
:1098600029E02846FFF7B4FF04460028F7D04FF45C
:10987000DB73019A3946284600F0BAFD002806DA63
:109880000025FFF7E1FFA581FFF7DFFFE7E70B4BBF
:1098900063620B4BA3620B4BE3620B4B2363F30539
:1098A000E081A681246205D50223002221462846B4
:1098B00000F0A0F8204603B0F0BD00BF91A9000859
:1098C000B3A90008EBA900080FAA0008024B0A463A
:1098D00001461868FFF7BABFBC0000200EB403B5FC
:1098E000014603AB054853F8042B0068019300F0D0
:1098F000C7FA02B05DF804EB03B07047BC0000206B
:1099000070B50E461446054618B183690BB9FFF7CA
:109910002FFF0A4B9C4201D16C6808E0084B9C4227
:1099200001D1AC6803E0074B9C4208BFEC682246BB
:1099300031462846BDE8704000F0B2BDFCCE0008BC
:109940001CCF00083CCF0008024B0A4601461868AD
:10995000FFF7D6BFBC00002070B50E461446054682
:1099600018B183690BB9FFF703FF1B4B9C4201D170
:109970006C6808E0194B9C4201D1AC6803E0184BBD
:109980009C4208BFEC68A3891B0701D523693BB93A
:109990002146284601F0C2FB10B14FF0FF3070BDE8
:1099A000013E16F8011FA9B1A368013B002BA3607B
:1099B00004DAA269934206DB0A2904D023685A1C00
:1099C00022601970EDE72246284601F041FB013084
:1099D000E7D1E2E7084670BDFCCE00081CCF0008C6
:1099E0003CCF0008024B0A4601461868FFF7B4BF97
:1099F000BC00002000F000B82DE9F8430C4690466A
:109A00001E46054618B183690BB9FFF7B1FE3D4B01
:109A10009C4201D16C6808E03B4B9C4201D1AC6890
:109A200003E03A4B9C4208BFEC68A38903F48473BB
:109A3000B3F5847F03D121462846FFF71DFEE76A70
:109A40000FB91D232BE0012E04D0022E2BD056B3CC
:109A5000162324E021462846FFF70EFEA28902F4D1
:109A6000805292B20AB1606D05E0216A3346284601
:109A7000B847411C14D0A3895A0706D56368C01A99
:109A8000636B4BB1236CC01A06E01B0704D5236837
:109A900013B122699B1A18448044002603E02B600E
:109AA0004FF0FF392BE023691BB92146284600F00F
:109AB000B3F821462846FFF7DFFD81460028EFD1A5
:109AC00033464246216A2846B8470130E8D0616BE8
:109AD00041B104F14403994202D0284600F0FAF85B
:109AE0000023636323692360A389002123F40263B5
:109AF0006160A381082204F15C0000F0E3F84846AD
:109B0000BDE8F883FCCE00081CCF00083CCF00085D
:109B10002DE9F041884600F1480400268CB1A56883
:109B20006768013F0BD4AB89012B06D9B5F90E301C
:109B3000013302D02846C04706436835F1E7246860
:109B4000ECE73046BDE8F0812DE9F84380468946D0
:109B500000F14804002694B1A5686768013F0CD461
:109B6000AB89012B07D9B5F90E30013303D0294653
:109B70004046C84706436835F0E72468EBE73046BF
:109B8000BDE8F88370B50E4B0E4CE41AA410002506
:109B90001E46A54204D056F8253098470135F8E70F
:109BA00001F04CFE084C094BE41AA41000251E4697
:109BB000A54204D056F8253098470135F8E770BD26
:109BC000C4000020C4000020C8000020C400002001
:109BD00070B50E46B1F90E10002990B014461D461E
:109BE00006DA00232B60B3891A060ED540230EE057
:109BF00001AA01F049FB0028F3DB029A02F470424B
:109C0000A2F500535A425A412A604FF48063002063
:109C1000236010B070BD00008B8973B59E070546A8
:109C20000C4610D401AB6A46FFF7D2FF00990646F6
:109C3000284600F09DF868B9B4F90C309A0522D492
:109C400043F00203A38104F147032360236101234E
:109C5000636118E00D4BAB62A389206043F0800381
:109C6000A381009B6361019B20614BB1B4F90E108D
:109C7000284601F01BFB18B1A38943F00103A3811F
:109C8000A0893043A08102B070BD00BFF1960008EA
:109C900010B501390244904207D010F8013B11F889
:109CA000014FA342F7D0181B10BD002010BD10B506
:109CB000431E0A44914204D011F8014B03F8014FAE
:109CC000F8E710BD02440346934202D003F8011B9B
:109CD000FAE7704738B50546002946D051F8043CEC
:109CE0000C1F002BB8BFE41801F06DFB1F4A13686E
:109CF000114613B96360146032E0A3420ED92268A2
:109D0000A018834204BF18685B68636004BF121820
:109D100022600C6024E0A24203D813465A68002A4D
:109D2000F9D118681918A1420BD1216801445818BB
:109D30008242196014D1106852685A600144196057
:109D40000EE002D90C232B600AE0216860188242E1
:109D500004BF10685268626004BF091821605C602B
:109D60002846BDE8384001F02FBB38BD503A0020EE
:109D700070B5CD1C25F0030508350C2D38BF0C251A
:109D8000002D064601DBA94202D90C23336046E0D0
:109D900001F019FB234B1C681A462146A1B10B6840
:109DA0005B1B0ED40B2B03D90B60CC18CD501EE0DF
:109DB0008C420DBF63684B686360136018BF0C462C
:109DC00015E00C464968E9E7174C23681BB9304693
:109DD00000F09CFD20602946304600F097FD431CB2
:109DE00018D0C41C24F00304A0420DD125603046D5
:109DF00001F0EAFA04F10B00231D20F00700C31A5A
:109E00000ED05A42E25070BD211A304600F07EFD5D
:109E10000130EBD10C233360304601F0D5FA00203D
:109E200070BD00BF503A00204C3A00209368013BBF
:109E3000002B10B4936009DA9469A34202DBCBB221
:109E40000A2B03D15DF8044B01F002B91368581CCA
:109E500010601970C8B25DF8044B7047F8B506463B
:109E60000F461446D518AC4208D03A4614F8011BE8
:109E70003046FFF7DBFF431CF5D100E00020F8BDC2
:109E80002DE9F04F9DB00C4617460393064618B1D6
:109E900083690BB9FFF76CFC7F4B9C4201D174685E
:109EA00008E07E4B9C4201D1B46803E07C4B9C42AD
:109EB00008BFF468A38918070CD5236953B10023A0
:109EC000099320238DF8293030238DF82A30DFF8CC
:109ED000D4B144E02146304601F020F90028EED00C
:109EE0004FF0FF30D5E0039A111D12680391002A4C
:109EF00080F28C80524243F002000792049098F85E
:109F000000302E2B00F08480032298F80010654862
:109F100001F0EEF948B14023CBEB000003FA00F06A
:109F2000049B1843049008F1010898F800105E485B
:109F30008DF82810062208F1010701F0D9F9002850
:109F400000F09580594B002B40F08880039B07332D
:109F500023F0070308330393099B53440993B8463E
:109F6000454615F8013B1BB9B8EB07090FD003E0D4
:109F7000252BF9D0A846F3E74B463A462146304612
:109F8000FFF76CFF01307FD0099B4B44099398F891
:109F90000030002B78D000234FF0FF32049307935A
:109FA000059206938DF853301A93012705222978DC
:109FB0003F4801F09DF905F10108049B38B13C4A86
:109FC000801A07FA00F0184304904546EEE7D906D8
:109FD00044BF20228DF853201A0744BF2B228DF84E
:109FE00053202A782A2A3FF47EAF079A00210A20BC
:109FF000A846013598F80030303B092B03D800FB08
:10A0000002320121F4E700293FF479AF079276E7A5
:10A0100098F801302A2B0BD1039B1A1D1B68039261
:10A02000002BB8BF4FF0FF3308F1020805936BE730
:10A030000023059308F1010019460A2580460130E6
:10A0400098F80020303A092A03D805FB01210123A2
:10A05000F4E7002B3FF458AF059155E703AB0093AD
:10A060002246144B04A93046AFF3008007E003AB4F
:10A07000009322460F4B04A9304600F093F8B0F14C
:10A08000FF3F82467FF468AFA3895B063FF528AFA8
:10A0900009981DB0BDE8F08FFCCE00081CCF000869
:10A0A0003CCF00086ACF00086ECF00080000000017
:10A0B00064CF00085D9E00082DE9F04791461F46D9
:10A0C0000A698B68DDF820809342B8BF1346C9F84F
:10A0D000003091F8432006460C4612B10133C9F80E
:10A0E00000302368990642BFD9F800300233C9F81E
:10A0F0000030256815F0060510D104F1190A07E0B3
:10A100000123524639463046C04701301AD0013546
:10A11000E368D9F800209B1A9D42F1DB94F84330A4
:10A120002268003318BF012392060FD5E1185A1C8C
:10A13000302081F84300224494F8451082F84310FF
:10A14000023303E04FF0FF30BDE8F08704F1430233
:10A1500039463046C0470130F4D02268D9F8005063
:10A16000E36802F00602042A08BF5D1B2269A368A7
:10A170000CBF25EAE57500259342C4BF9B1AED1874
:10A180004FF000091A344D4509D0012322463946C3
:10A190003046C0470130D5D009F10109F3E700206E
:10A1A000BDE8F0872DE9F04317460A7E85B06E2A98
:10A1B000984606460C460C9B01F1430E00F0AE801B
:10A1C00011D8632A22D009D8002A00F0BB80582A6F
:10A1D00040F0CA8081F84520834955E0642A1ED0AA
:10A1E000692A1CD0C0E0732A00F0B08009D86F2A19
:10A1F0002ED0702A40F0B8800A6842F020020A602F
:10A200003EE0752A24D0782A3AD0ADE01A6801F1F0
:10A210004205111D1960136884F84230A8E02168D6
:10A220001A6811F0800F02D0111D196008E011F0BA
:10A23000400F02F10401196002D0B2F9003000E0D1
:10A240001368002B3CDA2D225B4284F8432037E070
:10A2500021681A6811F0800F02D0111D196007E003
:10A2600011F0400F02F10401196001D0138800E0E1
:10A270001368227E5C496F2A14BF0A2208221BE061
:10A2800078225A4984F845202268186812F0800F15
:10A2900000F104051D6003D1550601D5038800E0D7
:10A2A0000368D00744BF42F0200222601BB9226835
:10A2B00022F0200222601022002084F8430001E0F6
:10A2C00049490A226568A560002D08DB206820F056
:10A2D000040020602BB9002D7DD175460CE0002BC9
:10A2E00079D07546B3FBF2F002FB1033CB5C05F876
:10A2F000013D03460028F5D1082A0BD12368DA076F
:10A3000008D5236962689A42DEBF302305F8013C14
:10A3100005F1FF35C5EB0E0323612EE008681A68CE
:10A32000496910F0800F03D0101D1860136808E011
:10A3300010F0400F02F104001860136801D019807A
:10A3400000E0196000232361754616E01A68111DAC
:10A350001960156862680021284600F0C9FF08B13D
:10A36000401B6060636804E004F1420584F8422009
:10A3700001232361002384F84330CDF800803B465D
:10A3800003AA21463046FFF797FE013002D14FF075
:10A39000FF3026E023692A4639463046C04701305F
:10A3A000F5D023689B0710D5002504F1190907E0B3
:10A3B00001234A4639463046C0470130E7D00135CF
:10A3C000E368039A9B1A9D42F2DBE068039B984284
:10A3D000B8BF184605E00B7884F8423004F1420516
:10A3E0008AE705B0BDE8F08375CF000886CF000886
:10A3F00038B5074C054608461146002222601A4629
:10A40000F8F7B0F8431C02D1236803B12B6038BDC4
:10A41000643A012037B50D46044618B183690BB97B
:10A42000FFF7A6F94DB12B783BB1E1682846FFF75D
:10A43000D9FAE1680948FFF7D5FA01AB0122216892
:10A44000204600F029FB10B1E168FFF7CBFAE16884
:10A450000A20FFF779FA03B030BD00BF23C500081A
:10A46000024B01461868FFF7D5BF00BFBC000020B3
:10A470000FB40A4B13B51C6824B1A36913B9204665
:10A48000FFF776F905AB049AA16801932046FFF720
:10A49000F7FC02B0BDE8104004B07047BC000020DB
:10A4A00070B50D461446064618B183690BB9FFF71F
:10A4B0005FF9134B9C4201D1746808E0114B9C4238
:10A4C00001D1B46803E0104B9C4208BFF468A36854
:10A4D000013B002BA3600CDAA269934202DBEBB2D2
:10A4E0000A2B06D1224629463046BDE8704000F0CE
:10A4F000AFBD23685A1C22601D70E8B270BD00BF5A
:10A50000FCCE00081CCF00083CCF000870B50E46FA
:10A51000054618B183690BB9FFF72AF9AB69AC6836
:10A5200013B92846FFF724F9224B9C4201D16C68ED
:10A5300008E0214B9C4201D1AC6803E01F4B9C42D8
:10A5400008BFEC68A3891B0701D523693BB92146E5
:10A55000284600F0E3FD10B14FF0FF3070BD013E22
:10A56000A36816F8011F013BA36091B1002B04DA28
:10A57000A269934206DB0A2904D023685A1C226090
:10A580001970EDE72246284600F062FD0130E7D160
:10A59000E2E7002B08DA22460A21284600F058FD9F
:10A5A0000130D9D00A2070BD23680A205A1C2260CD
:10A5B000187070BDFCCE00081CCF00083CCF00080E
:10A5C000024B01461868FFF7A1BF00BFBC00002086
:10A5D000012B30B50ADC9208013A03680C6840F898
:10A5E000044B002A41F8043BF6DC30BD03460D78ED
:10A5F0001C7803F8015B01F8014BD41A0444002CC9
:10A60000F5DC30BDF8B50F46144606461D469847A2
:10A610000028214638460BDAA847002801DA3846D8
:10A62000F8BD21463046A847002809DB3046F8BD72
:10A63000A8470028F3DC21463046A8470028F5DB70
:10A640002046F8BD2DE9F04F85B006468B461446EE
:10A650000093B20707D1A30705D1B4F1040818BFCE
:10A660004FF0010801E04FF002083319BBF1060F6B
:10A67000019326D81F4604FB0B65AF4280F016817C
:10A68000B9464E4501D32744F7E7C4EB090A4946CA
:10A690005046009B98470028F5DDB8F1000F08D11F
:10A6A000D9F80030DAF80020C9F80020CAF80030E4
:10A6B00005E04346224651464846FFF789FFD1460A
:10A6C000DFE74FEA5B050BF1FF33BBF1070F04FB3C
:10A6D0000565019326D0BBF1280F04FB036919D946
:10A6E0004FEADB076743F119CA19009B3046FFF7B1
:10A6F00089FFEA192946009B8246E81BFFF782FF83
:10A700000546A9EB47004A46009BC119FFF77AFFAF
:10A71000814600E0B2462946009B4A465046FFF774
:10A7200071FF0546B8F1000F04D133682A68326022
:10A730002B6005E04346224629463046FFF748FF96
:10A74000019B371904FB03653B190293A946019746
:10A750000023029AC4EB020A554555D303933146B0
:10A76000009B504698470028039B24DC15D1B8F184
:10A77000000F08D1019B01991B68DAF800200A60DC
:10A78000CAF8003005E04346224651460198FFF7DB
:10A790001FFF019B234401930123029A224402924A
:10A7A000D7E703933146009B284698470028039B30
:10A7B00018DB03D02D1B5545F3D225E0B8F1000F6F
:10A7C00006D12B68D9F800202A60C9F8003005E0CE
:10A7D0004346224649462846FFF7FAFEC4EB0909DC
:10A7E0000123E7E7B8F1000F06D1DAF800302A6854
:10A7F000CAF800202B6005E0434622462946504611
:10A80000FFF7E6FE2D1BC7E704FB0BFB63B3019BC1
:10A8100006EB0B079A1BC3EB0A0B5A45A8BF5A4617
:10A820002AB14346C2EB0A013046FFF7D1FEC9EB1D
:10A830000702C5EB0905121BAA4228BF2A4622B10E
:10A840004346B91A5046FFF7C3FE5C4506D2BBFB30
:10A85000F4F1009B22463046FFF7F4FEAC4225D2CD
:10A86000B5FBF4FB7E1BF4E6B3445F451ED23D46C8
:10A87000AE4201D32744F8E7C4EB05092946484610
:10A88000009B98470028F5DDB8F1000F06D12B6832
:10A89000D9F800202A60C9F8003005E04346224676
:10A8A00049462846FFF794FE4D46E1E705B0BDE86E
:10A8B000F08F000038B50C46054618B183690BB916
:10A8C000FEF756FF0E4B9C4201D16C6808E00D4B21
:10A8D0009C4201D1AC6803E00B4B9C4208BFEC6882
:10A8E0002146284600F000FF38B96368013B6360E9
:10A8F00023685A1C2260187838BD4FF0FF3038BDED
:10A90000FCCE00081CCF00083CCF000838B5064C30
:10A91000002305460846236000F080FF431C02D157
:10A92000236803B12B6038BD643A01200CB430B504
:10A93000164B0C1E9DB01D6804DA8B232B604FF064
:10A94000FF301EE04FF40273ADF8143014BF04F171
:10A95000FF332346049307934FF6FF73029006904C
:10A96000ADF81630209A21AB02A92846019300F0D9
:10A97000ABFD431CBCBF8B232B6014B1029B002298
:10A980001A701DB0BDE8304002B07047BC00002016
:10A9900010B50C46B1F90E1000F08AFE0028ABBFCE
:10A9A000636DA3891B1823F48053ACBF6365A38137
:10A9B00010BD2DE9F0411F468B89DB0505460C468D
:10A9C000164605D502230022B1F90E1000F07EFCD8
:10A9D000A389B4F90E1023F48053A38132463B4679
:10A9E0002846BDE8F04100F087BB10B50C46B1F930
:10A9F0000E1000F06BFC431CA38915BF606523F4A7
:10AA0000805343F48053A38118BFA38110BDB1F9D3
:10AA10000E1000F0F1BB00000D4B30B51D6810F8B2
:10AA2000013BEA18527802F00302012A11F8012BC7
:10AA300005EB020408BF2033647804F00304012C02
:10AA400008BF20329B1A01D1002AE8D1184630BD38
:10AA5000C000002010B50246134601321C78002CBD
:10AA6000FAD1013B11F8012B03F8012F002AF9D18B
:10AA700010BD10F8012B11F8013B012A28BF9A42A2
:10AA8000F7D0D01A7047034611F8012B03F8012BB9
:10AA9000002AF9D17047000010B504460846114657
:10AAA0008E2800F22F81DFE810F038018F0091002E
:10AAB00093009500970099009B009D00A100A300C2
:10AAC000A700A900AB00AD002D01AF00B100B3009D
:10AAD000B500B700BD00BF00C500C700C900CB006E
:10AAE000CD00D100D500D700D900DB00DD00DF00AC
:10AAF000E100E3002D012D012D012D012D012D017E
:10AB00002D012D01E700EB002D012D012D012D015F
:10AB10002D012D012D012D012D012D012D012D01C5
:10AB20002D01ED000701EF00F1002D012D012D0198
:10AB3000F3002D012D012D01F5002D012D01F9004E
:10AB40002D012D01FB002D012D012D012D012D01C8
:10AB50002D012D012D012D012D01FD002D01FF00E5
:10AB6000010103012D012D0125012D012D012D01D3
:10AB70002D012D012D012D012D01130105010901CB
:10AB80000B010D010F012D01110115011901E90042
:10AB9000C1002B01B900CF00BB009F00A500290117
:10ABA000F7002D011701C3001D011B012D012D010F
:10ABB0002D012D012D01D3002D012D012D01E500C9
:10ABC00027011F0121012301554810BD554810BD23
:10ABD000554810BD554810BD554810BD554810BDCD
:10ABE000554810BD554810BD554810BD554810BDBD
:10ABF000554810BD554810BD554810BD554810BDAD
:10AC0000554810BD554810BD554810BD554810BD9C
:10AC1000554810BD554810BD554810BD554810BD8C
:10AC2000554810BD554810BD554810BD554810BD7C
:10AC3000554810BD554810BD554810BD554810BD6C
:10AC4000554810BD554810BD554810BD554810BD5C
:10AC5000554810BD554810BD554810BD554810BD4C
:10AC6000554810BD554810BD554810BD554810BD3C
:10AC7000554810BD554810BD554810BD554810BD2C
:10AC8000554810BD554810BD554810BD554810BD1C
:10AC9000554810BD554810BD554810BD554810BD0C
:10ACA000554810BD554810BD554810BD554810BDFC
:10ACB000554810BD554810BD554810BD554810BDEC
:10ACC000554810BD554810BD554810BD554810BDDC
:10ACD000554810BD554810BD554810BD554810BDCC
:10ACE000554810BD554810BD554810BD554810BDBC
:10ACF000554810BD554810BD554810BD554810BDAC
:10AD0000554810BD002B14BF1A46224600F0E9F842
:10AD1000524B002808BF184610BD514810BD00BF57
:10AD20009FCF0008A9CF0008C3CF0008D3CF0008E9
:10AD3000EBCF0008F5CF00080FD0000821D00008A5
:10AD400033D000084CD000085CD0000868D0000860
:10AD500085D0000897D00008A8D00008BAD0000815
:10AD6000C6D00008DED00008EAD00008FCD00008F9
:10AD70000BD100081BD1000828D1000847D10008DA
:10AD800056D1000867D100088BD10008A9D100086E
:10AD9000C7D10008E7D10008FED100080DD2000895
:10ADA0001CD2000830D2000848D2000856D2000851
:10ADB00063D2000879D2000888D2000894D2000833
:10ADC000C3D20008D4D20008EFD2000802D3000892
:10ADD00018D3000821D3000838D3000840D3000856
:10ADE0004DD3000862D3000876D300088ED3000844
:10ADF0009DD30008AED30008C1D30008CDD300080E
:10AE0000E6D30008FAD3000815D400082DD40008B2
:10AE100047D400084FD400087FD400089ED400080F
:10AE2000BDD40008D4D40008E7D4000800D5000839
:10AE300017D500082DD500084ED5000866D50008A6
:10AE400082D5000895D50008ABD50008BFD500080D
:10AE5000E1D5000807D6000818D600086FCA000818
:10AE600097CF0008034613F8012B002AFBD1181ACC
:10AE700001387047104B70B51E680A44914217D0D4
:10AE800010F8013BF418647804F00304012C11F865
:10AE9000014B06EB040508BF20336D7805F0030570
:10AEA000012D08BF20341B1B03D1002CE6D100E08C
:10AEB0000023184670BD00BFC000002010B5034637
:10AEC00042B111F8014B03F8014B013A002CF7D1C4
:10AED0001A4400E010BD934202D003F8014BFAE798
:10AEE00010BD002070472DE9F0410C46496B04F17C
:10AEF000440399421CD14FF48061FEF739FF18B921
:10AF00004FF0FF30BDE8F0814FF48063A36394F805
:10AF10004630606380F8FF3394F8453080F8FE33A4
:10AF200094F8443080F8FD3300F2FD30206012E0E8
:10AF3000A66B77003A4600F048FA05460028DFD0B5
:10AF400000EB0608014632464046FEF7B0FEC4F864
:10AF500000806563A7630020BDE8F081F8B54D1C53
:10AF600006460F46144602D14FF0FF30F8BD18B127
:10AF700083690BB9FEF7FCFB2E4B9C4201D1746830
:10AF800008E02D4B9C4201D1B46803E02B4B9C425E
:10AF900008BFF468B4F90C3023F02003A3819BB2FE
:10AFA000590713D4DA06DFD51B070BD521463046E7
:10AFB000FEF762FB0028D7D1A389A06023F0080325
:10AFC000A381A061A38943F00403A381636B62683A
:10AFD000FDB28BB1A36B9A4207DA23685A1E226036
:10AFE00003F8017C6368013320E021463046FFF717
:10AFF0007AFF0028F1D0B7E72169236851B199425F
:10B0000008D213F8011C8D4204D1013B01322360A8
:10B0100062600CE0E36304F1440363630323A3630E
:10B020002346226403F8467F236001236360284699
:10B03000F8BD00BFFCCE00081CCF00083CCF0008C4
:10B04000024B0A4601461868FFF788BFBC00002083
:10B05000F8B50F461446064618B183690BB9FEF7DA
:10B0600087FB224B9C4201D1746808E0204B9C4234
:10B0700001D1B46803E01F4B9C4208BFF468A36988
:10B08000A360A3891A0709D523693BB12368206906
:10B09000181A63699842FDB20FDB08E0214630467A
:10B0A00000F03CF80028F1D04FF0FF30F8BD214609
:10B0B0003046FEF7E1FA0028F6D1A368013BA36011
:10B0C00023685A1C22601F706269431C934204D09B
:10B0D000A389DB0707D50A2D05D121463046FEF7A7
:10B0E000CBFA0028E0D12846F8BD00BFFCCE00080E
:10B0F0001CCF00083CCF000838B5074C0546084671
:10B100001146002222601A46F7F7ECFA431C02D1DE
:10B11000236803B12B6038BD643A0120324B70B50F
:10B120001D6806460C4625B1AB6913B92846FEF7E3
:10B130001FFB2E4B9C4201D16C6808E02C4B9C42BB
:10B1400001D1AC6803E02B4B9C4208BFEC68B4F91A
:10B150000C309AB215071DD4D00602D409223260F1
:10B160003AE0510712D5616B41B104F144039942B1
:10B1700002D03046FEF7AEFD00236363A38923F0BF
:10B180002403A3810023636023692360A38943F020
:10B190000803A38123694BB9A38903F42073B3F592
:10B1A000007F03D021463046FEF736FDA28912F01B
:10B1B000010305D00023A36063695B42A36103E040
:10B1C000920758BF6369A36023695BB9B4F90C3077
:10B1D00003F0800080B230B143F04003A3814FF010
:10B1E000FF3070BD002070BDBC000020FCCE000808
:10B1F0001CCF00083CCF000838B5064C002305469C
:10B2000008462360F7F70AFA431C02D1236803B10A
:10B210002B6038BD643A01200B78722B30B50ED00C
:10B22000772B07D0612B0ED14FF4027401234FF41A
:10B2300084701AE04FF4C0640123082015E0002454
:10B240002346042011E016230360002030BD622D48
:10B2500010D0782D11D02B2D07D120F01C0023F019
:10B26000030340F0100043F0020311F8015F002DCA
:10B27000EDD105E043F48033F7E743F40063F4E7EE
:10B280002343136030BD000038B5074C002305464A
:10B2900008461146236000F0B9FA431C02D1236826
:10B2A00003B12B6038BD00BF643A012038B5064CAD
:10B2B0000023054608462360F7F7C2FA431C02D173
:10B2C000236803B12B6038BD643A012038B5074CC0
:10B2D000054608461146002222601A46F7F788FA0A
:10B2E000431C02D1236803B12B6038BD643A0120AE
:10B2F00001F0FF01102A2BDB10F0070F08D010F827
:10B30000013B013A8B422DD010F0070F42B3F6D12A
:10B31000F0B441EA012141EA014122F007047FF043
:10B3200000070023F0E80256083C85EA010586EA9A
:10B33000010685FA47F5A3FA87F586FA47F6A5FAD6
:10B3400087F68EB9EED1F0BC01F0FF0102F00702E2
:10B3500032B110F8013B013A83EA010313B1F8D18D
:10B360000020704701387047002D06BF354603386E
:10B37000073815F0010F07D1013015F4807F02BFA7
:10B38000013015F4C03F0130F0BC0138704700BFF8
:10B39000884210B501EB020301D8421E0BE098422F
:10B3A000FBD28118D21AD34204D013F8014D01F810
:10B3B000014DF8E710BD994204D011F8014B02F895
:10B3C000014FF8E710BD70477047F8B507461546BE
:10B3D0000E4621B91146BDE8F840FEF7C9BC1AB9BE
:10B3E000FEF778FC2846F8BD00F006FA85420ED933
:10B3F00029463846FEF7BCFC044650B131462A4681
:10B40000FEF755FC31463846FEF764FC01E0304655
:10B41000F8BD2046F8BD2DE9F0478E689E42824671
:10B420000C46914698463ED88A8912F4906F3AD0DD
:10B43000256809696F1A6569022305EB450595FBC7
:10B44000F3F57B1C43449D4238BF1D4653050FD581
:10B450002946FEF78DFC064698B13A462169FEF76B
:10B4600026FCA38923F4906343F08003A38113E0B7
:10B470002A46FFF7AAFF064670B921695046FEF733
:10B4800029FC0C23CAF80030A38943F04003A381B0
:10B490004FF0FF30BDE8F087266165613E44ED1B4B
:10B4A0002660A5604646464528BF46463246494680
:10B4B0002068FFF76DFFA3689B1BA36023681E44F1
:10B4C00026600020BDE8F0872DE9F04F9DB0804652
:10B4D00003938B891C060D4616460DD50B695BB987
:10B4E0004021FEF745FC2860286118B90C23C8F8F4
:10B4F0000030CDE040236B610023099320238DF8B9
:10B500002930DFF89CB130238DF82A3037463C468D
:10B5100014F8013B1BB9B7EB060910D003E0252B4B
:10B52000F9D02746F3E74B46324629464046FFF717
:10B5300072FF013000F0A780099B4B4409933B78D0
:10B54000002B00F0A08000234FF0FF3204930793FC
:10B55000059206938DF853301A930126052221781F
:10B560004E48FFF7C5FE671C049B38B14B4A801A52
:10B5700006FA00F0184304903C46EFE7D90644BFB2
:10B5800020228DF853201A0744BF2B228DF8532018
:10B5900022782A2A03D0079A00210A200BE0039A76
:10B5A000111D12680391002A10DA524243F0020082
:10B5B000079204900BE0274601343B78303B092B7F
:10B5C00003D800FB02320121F5E701B107923B7875
:10B5D0002E2B1ED17B782A2B0AD1039B1A1D1B68A8
:10B5E0000392002BB8BF4FF0FF330237059310E0F2
:10B5F00000230593781C19460A24074601303A783F
:10B60000303A092A03D804FB01210123F5E703B1ED
:10B610000591032239782248FFF76AFE40B14023A2
:10B62000CBEB000003FA00F0049B184304900137B1
:10B6300039781C488DF8281006227E1CFFF758FE2A
:10B6400088B1194B33B9039B073323F00703083341
:10B65000039314E003AB00932A46144B04A940461D
:10B66000AFF3008007E003AB00932A460F4B04A919
:10B670004046FEF797FDB0F1FF3F824603D0099B9D
:10B680005344099342E7AB895B0601D4099801E072
:10B690004FF0FF301DB0BDE8F08F00BF64CF000851
:10B6A0006ACF00086ECF00080000000017B4000841
:10B6B00038B5074C054608461146002222601A4656
:10B6C000F6F7D0FF431C02D1236803B12B6038BDCD
:10B6D000643A0120838903F00903092B01D1FDF7A6
:10B6E000F5BF002070470000F8B50C46054618B1BC
:10B6F00083690BB9FEF73CF83A4B9C4201D16C6868
:10B7000008E0394B9C4201D1AC6803E0374B9C42C6
:10B7100008BFEC68B4F90C200023636093B29E0666
:10B720005BD458071AD4D90605D4092342F0400245
:10B730002B60A28151E01A070BD521462846FDF760
:10B740009BFF002849D1A389A06023F00803A381AF
:10B75000A061A38943F00403A38110E0616B71B180
:10B7600004F14403994202D02846FEF7B3FA236C51
:10B7700063600020606313B1E36B2360F8BD23694D
:10B780001BB921462846FEF747FAB4F90C70BEB241
:10B79000B3070FD00123A381154B1649186806F093
:10B7A0000906FEF7B5F9092EA78103D121462846DF
:10B7B000FDF7DAFE22692260666A6369216A28461B
:10B7C000B047002860600BDCA38917BF002243F05C
:10B7D000200343F040036260A3814FF0FF30F8BDC7
:10B7E0000020F8BDFCCE00081CCF00083CCF0008AC
:10B7F00060CF0008D5B6000851F8040C0028BEBF81
:10B80000091851F8043CC01804387047024B5822FC
:10B810001A604FF0FF307047643A0120044B1968FA
:10B82000024609B903491960186802441A60704752
:10B83000543A0020683A0120FEE70000F8B500BF46
:10B84000F8BC08BC9E467047F8B500BFF8BC08BC01
:10B850009E46704746415400464154333200222AE6
:10B860002B2C3A3B3C3D3E3F5B5D7C7F00EBFE90EA
:10B870004D53444F53352E30004E4F204E414D45D1
:10B88000202020204641543332202020004E4F20DB
:10B890004E414D452020202046415420202020208C
:10B8A0000043554541414141434545454949494189
:10B8B000414592924F4F4F5555594F554F9C4F9E72
:10B8C0009F41494F55A5A5A6A7A8A9AAABACADAE67
:10B8D000AFB0B1B2B3B4414141B8B9BABBBCBDBE5F
:10B8E000BFC0C1C2C3C4C54141C8C9CACBCCCDCEFB
:10B8F000CFD1D145454549494949D9DADBDCDD4954
:10B90000DF4FE14F4F4F4FE6E8E85555555959EE97
:10B91000EFF0F1F2F3F4F5F6F7F8F9FAFBFCFDFEBF
:10B92000FF00000000000000000000000000000018
:10B930000000000000000000000000000000000007
:10B9400000000000000000000000000000000000F7
:10B9500000000000000000000000000000000000E7
:10B9600000000000000000000000000000000000D7
:10B9700000000000000000000000000000000000C7
:10B9800000000000000000000000000000000000B7
:10B9900000000000000000000000000000000000A7
:10B9A0000000000000000000000000000000000097
:10B9B0000000000000000000000000000000000087
:10B9C0000000000000000000000000000000000077
:10B9D0000000000000000000000000000000000067
:10B9E0000000000000000000000000000000000057
:10B9F0000000000000000000000000000000000047
:10BA00000000000000000000000000000000000036
:10BA10000000000000000000000000000000000026
:10BA20000000000000000000000000000000000016
:10BA30000000000000000000000000000000000006
:10BA400000000000000000000000000000000000F6
:10BA500000000000000000000000000000000000E6
:10BA600000000000000000000000000000000000D6
:10BA700000000000000000000000000000000000C6
:10BA800000000000000000000000000000000000B6
:10BA900000000000000000000000000000000000A6
:10BAA00000000000000000000000000000003078EE
:10BAB0007878303000303000000066666624000080
:10BAC0000000000000006C6CFE6C6C6CFE6C6C0086
:10BAD0000030307CC0C0780C0CF830300000000022
:10BAE000C4CC183060CC8C00000070D8D870FADE5E
:10BAF000CCDC760000003030306000000000000038
:10BB000000000C183060606030180C0000006030DD
:10BB1000180C0C0C1830600000000000663CFF3C64
:10BB2000660000000000000018187E1818000000D1
:10BB30000000000000000000003838600000000035
:10BB40000000FE00000000000000000000000000F7
:10BB50000038380000000002060C183060C0800079
:10BB600000007CC6CEDED6F6E6C67C0000001030B3
:10BB7000F03030303030FC00000078CCCC0C183085
:10BB800060CCFC00000078CC0C0C380C0CCC78009D
:10BB900000000C1C3C6CCCFE0C0C1E000000FCC019
:10BBA000C0C0F80C0CCC780000003860C0C0F8CCE5
:10BBB000CCCC78000000FEC6C6060C183030300031
:10BBC000000078CCCCCC78CCCCCC7800000078CC01
:10BBD000CCCC7C1818307000000000003838000011
:10BBE00038380000000000003838000038381830BD
:10BBF00000000C183060C06030180C00000000001D
:10BC0000007E007E0000000000006030180C060C72
:10BC100018306000000078CC0C1830300030300054
:10BC200000007CC6C6DEDEDEC0C07C0000003078CE
:10BC3000CCCCCCFCCCCCCC000000FC6666667C6630
:10BC40006666FC0000003C66C6C0C0C0C6663C001C
:10BC50000000F86C66666666666CF8000000FE62BE
:10BC600060647C646062FE000000FE6662647C6466
:10BC70006060F00000003C66C6C0C0CEC6663E00F4
:10BC80000000CCCCCCCCFCCCCCCCCC0000007830B0
:10BC9000303030303030780000001E0C0C0C0CCCF2
:10BCA000CCCC78000000E6666C6C786C6C66E600C4
:10BCB0000000F060606060626666FE000000C6EE34
:10BCC000FEFED6C6C6C6C6000000C6C6E6F6FEDE46
:10BCD000CEC6C6000000386CC6C6C6C6C66C3800E4
:10BCE0000000FC6666667C606060F0000000386CF6
:10BCF000C6C6C6CEDE7C0C1E0000FC6666667C6C8A
:10BD00006666E600000078CCCCC07018CCCC780019
:10BD10000000FCB430303030303078000000CCCC43
:10BD2000CCCCCCCCCCCC78000000CCCCCCCCCCCC0B
:10BD3000CC7830000000C6C6C6C6D6D66C6C6C0087
:10BD40000000CCCCCC783078CCCCCC000000CCCC73
:10BD5000CCCC7830303078000000FECE98183060BF
:10BD600062C6FE0000003C303030303030303C00E5
:10BD700000000080C06030180C06020000003C0C7F
:10BD80000C0C0C0C0C0C3C000010386CC6000000B5
:10BD9000000000000000000000000000000000FFA4
:10BDA000003030180000000000000000000000001B
:10BDB00000780C7CCCCC76000000E060607C66668D
:10BDC0006666DC00000000000078CCC0C0CC7800C3
:10BDD00000001C0C0C7CCCCCCCCC7600000000000D
:10BDE0000078CCFCC0CC78000000386C6060F86053
:10BDF0006060F000000000000076CCCCCC7C0CCC65
:10BE00007800E060606C76666666E60000001818F0
:10BE10000078181818187E0000000C0C003C0C0C60
:10BE20000C0CCCCC7800E06060666C786C66E60048
:10BE3000000078181818181818187E000000000064
:10BE400000FCD6D6D6D6C6000000000000F8CCCC48
:10BE5000CCCCCC00000000000078CCCCCCCC78005E
:10BE60000000000000DC666666667C60F000000092
:10BE70000076CCCCCCCC7C0C1E00000000EC6E76A6
:10BE80006060F000000000000078CC6018CC780002
:10BE90000000002060FC6060606C38000000000062
:10BEA00000CCCCCCCCCC76000000000000CCCCCCBC
:10BEB000CC7830000000000000C6C6D6D66C6C00FE
:10BEC0000000000000C66C38386CC600000000009E
:10BED00000666666663C0C18F000000000FC8C18DA
:10BEE00060C4FC0000001C303060C06030301C00BA
:10BEF0000000181818180018181818000000E03072
:10BF000030180C183030E000000073DACE0000006A
:10BF1000000000000000000010386CC6C6FE0000E3
:10BF2000000010387CFEFE7C38100000002492498E
:10BF30002492492492492492490000000000000004
:10BF400000000000000000000000000000000000F1
:10BF500000000000000000000000000000000000E1
:10BF600000000000000000000000000000000000D1
:10BF700000000000000000000000000000000000C1
:10BF800000000000000000000000000000000000B1
:10BF90000000000000000000001818181818F80031
:10BFA00000000000000000000000F8181818181821
:10BFB0001800000000001F18181818181818181872
:10BFC00018181F0000000000001818181818FF1893
:10BFD00018181818180000000000000000000000E9
:10BFE0000000000000000000000000000000000051
:10BFF0000000FF0000000000000000000000000042
:10C000000000000000000000000000000000000030
:10C010000018181818181F181818181818181818B1
:10C020001818F81818181818180000000000000058
:10C0300000000000000000000000FF181818181889
:10C0400018181818181818181818181818000000B8
:10C0500000000000000000000000000000000000E0
:10C0600000000000000000000000000000000000D0
:10C0700000000000000000000000000000000000C0
:10C0800000000000000000000000000000000000B0
:10C0900000000000000000000000000000000000A0
:10C0A0000000000000000000000000000000303030
:10C0B00000303078787830000000303078CCC0C064
:10C0C000CC783030003C66606060FC6060C0FE0090
:10C0D000000000000000C67C6C7CC60000CCCCCC0C
:10C0E000CC78FC30FC30300000001818181800180C
:10C0F0001818180000007E63303C66663C0CC67E53
:10C100000000CC00000000000000000000003844E7
:10C11000BAA2A2A2BA443800000078CCCC7E00FEBD
:10C120000000000000000000003366CCCC66330045
:10C13000000000000000FC0C0C0C000000000000DF
:10C140000000FC000000000000003844BAAABAB2A7
:10C15000AA4438000000FC000000000000000000BD
:10C1600000003C6666663C000000000000000030F5
:10C1700030FC303000FC00000000780C18307C00EF
:10C18000000000000000780C380C7800000000006F
:10C19000000C18300000000000000000000000004B
:10C1A0000066666666667B60C0007FDBDBDB7B1B50
:10C1B0001B1B1B0000000000000018000000000016
:10C1C000000000000000000000000030700030702F
:10C1D0003030780000000000000078CCCC7800FE01
:10C1E000000000000000000000CC66333366CC0085
:10C1F000000063E66C78376FDBB33F03000062E654
:10C200006C78306EC3860C1F00E033663CF8376FE5
:10C21000DBB33F0300003030003060C0C0CC78009A
:10C22000006030003078CCCCFCCCCC00000C180086
:10C230003078CCCCFCCCCC000078CC003078CCCCA6
:10C24000FCCCCC000076DC003078CCCCFCCCCC0034
:10C250000000CC003078CCCCFCCCCC000078CCCC2E
:10C260007878CCCCFCCCCC0000003E78D8D8FED876
:10C27000D8D8DE00000078CCCCC0C0C0CCCC7830A0
:10C2800060603000FCC4C0F8C0C4FC00000C1800A2
:10C29000FCC4C0F8C0C4FC000078CC00FCC4C0F8EA
:10C2A000C0C4FC000000CC00FCC4C0F8C0C4FC004A
:10C2B00000603000783030303030780000183000C6
:10C2C00078303030303078000078CC007830303042
:10C2D000303078000000CC007830303030307800DA
:10C2E0000000F86C6666F666666CF8000076DC00A6
:10C2F000C6E6F6DECEC6C6000060300078CCCCCCF8
:10C30000CCCC78000018300078CCCCCCCCCC7800E9
:10C310000078CC0078CCCCCCCCCC78000076DC009B
:10C3200078CCCCCCCCCC78000000CC0078CCCCCC79
:10C33000CCCC7800000000000000C66C386CC60051
:10C3400000003A6CCED6D6D6E66CB800006030005D
:10C35000CCCCCCCCCCCC780000183000CCCCCCCC25
:10C36000CCCC78000078CC00CCCCCCCCCCCC780039
:10C3700000CC00CCCCCCCCCCCCCC7800001830009D
:10C38000CCCCCC78303078000000F0607C666666FB
:10C390007C60F000000078CCCCD8CCCCCCF8C0606D
:10C3A00000C0603000780C7CCCCC7600000C1830DB
:10C3B00000780C7CCCCC7600003078CC00780C7CFB
:10C3C000CCCC7600000076DC00780C7CCCCC7600FF
:10C3D0000000CCCC00780C7CCCCC760000386C6CA7
:10C3E00038F80C7CCCCC76000000000000FE1B7FEF
:10C3F000D8D8EF00000000000078CCC0C0CC783066
:10C4000060C060300078CCFCC0C07C00000C1830EC
:10C410000078CCFCC0CC7800003078CC0078CCFC24
:10C42000C0C07C000000CCCC0078CCFCC0C07C003C
:10C43000006030180078181818187E00000C1830AA
:10C440000078181818187E000010386C007818183A
:10C4500018187E0000006C6C0078181818187E0000
:10C4600000CC30D80C067EC6C6C67C00000076DC48
:10C4700000F8CCCCCCCCCC0000C060300078CCCC68
:10C48000CCCC7800000C18300078CCCCCCCC780028
:10C49000003078CC0078CCCCCCCC7800000076DCB6
:10C4A0000078CCCCCCCC78000000CCCC0078CCCCC4
:10C4B000CCCC7800000000303000FC0030300000B0
:10C4C000000000000078CCDCECCC780000C06030CC
:10C4D00000CCCCCCCCCC7600000C183000CCCCCC32
:10C4E000CCCC7600003078CC00CCCCCCCCCC760058
:10C4F0000000CCCC00CCCCCCCCCC760000060C1808
:10C5000000666666663C0C18F00000E0607C6666BB
:10C510007C60F0000000666600666666663C0C188B
:10C52000F025733A20007375636365656465640A7A
:10C5300000612068617264206572726F72206F639F
:10C5400063757272656420696E20746865206C6F13
:10C5500077206C6576656C206469736B20492F4F7A
:10C56000206C617965720A00617373657274696F1A
:10C570006E206661696C65640A007068797369632E
:10C58000616C2064726976652063616E6E6F7420E1
:10C59000776F726B0A006E6F20737563682066692F
:10C5A0006C650A006E6F20737563682066696C6540
:10C5B000206F72206469726563746F72790A00700B
:10C5C000617468206E616D6520666F726D617420A4
:10C5D000697320696E76616C69640A0061636365E2
:10C5E00073732064656E6965642064756520746F7B
:10C5F0002070726F68696269746564206163636545
:10C600007373206F72206469726563746F7279202E
:10C6100066756C6C0A006163636573732064656E94
:10C620006965642064756520746F2070726F686935
:10C630006269746564206163636573730A00666987
:10C640006C652F6469726563746F7279206F626ABA
:10C6500065637420697320696E76616C69640A0091
:10C66000706879736963616C2064726976652069AA
:10C67000732077726974652070726F746563746576
:10C68000640A006C6F676963616C20647269766527
:10C69000206E756D62657220697320696E76616CBB
:10C6A00069640A00766F6C756D6520686173206E31
:10C6B0006F20776F726B20617265610A0074686524
:10C6C0007265206973206E6F2076616C6964204604
:10C6D000415420766F6C756D650A00665F6D6B6600
:10C6E0007328292061626F72746564206475652007
:10C6F000746F20616E792070726F626C656D0A00D4
:10C70000636F756C64206E6F7420676574206120A0
:10C710006772616E7420746F206163636573732048
:10C7200074686520766F6C756D65207769746869CB
:10C730006E20646566696E656420706572696F64F9
:10C740000A006F7065726174696F6E206973207280
:10C75000656A6563746564206163636F7264696EA2
:10C760006720746F207468652066696C6520736843
:10C770006172696E6720706F6C6963790A006C463C
:10C780004E20776F726B696E6720627566666572A0
:10C7900020636F756C64206E6F7420626520616C1D
:10C7A0006C6F63617465640A006E756D62657220FA
:10C7B0006F66206F70656E2066696C6573203E2021
:10C7C00046465F46535F4C4F434B0A0067697665A8
:10C7D0006E20706172616D65746572206973206985
:10C7E0006E76616C69640A00756E6B6E6F776E2091
:10C7F0006572726F720A006572726F723A206664B7
:10C80000202564206E6F7420636C6F7365640A006A
:10C8100000FF00FF00FF00FF00FF00FF00FF00FF20
:10C8200000FF00FF00FF00FF00FF00FF00FF00FF10
:10C8300000FF00FF000000FF01710120023000FF37
:10C8400000FF00FF0154011101100121025000FFFF
:10C8500000FF01030102011201220233003200FF36
:10C8600000FF01700104011301240123023400FFC1
:10C8700000FF01730174016401140101024400FF0F
:10C8800000FF00FF0172016301530204024200FF36
:10C8900000FF02510162015201510261024100FF99
:10C8A00000FF02010240016100FF0050020300FF8F
:10C8B00000FF00FF00FF00FF00FF00FF00FF00FF80
:10C8C00000FF00FF0060027400FF024300FF00FF52
:10C8D00000FF022400FF00FF00FF00FF014000FFF7
:10C8E00000FF00FF00FF00FF00FF00FF00FF00FF50
:10C8F00000FF00FF00FF00FF00FF00FF017000FFCE
:10C9000000FF00FF00FF00FF00FF00FF00FF00FF2F
:10C91000437572736F72204A6F79737469636B0029
:10C9200053696E636C616972204A6F7973746963CD
:10C930006B20310053696E636C616972204A6F79B4
:10C94000737469636B2032004B656D7073746F6E26
:10C95000204A6F79737469636B0000FF00FF00FF6A
:10C9600000FF00FF00FF00FF00FF00FF00FF00FFCF
:10C9700000FF00FF00FF00FF00FF00FF00FF0000BE
:10C9800000FF00710020003000FF00FF00FF0001E9
:10C99000001100100021003100FF00FF0003000221
:10C9A000001200220033003200FF00FF007000047C
:10C9B000001300240023003400FF00FF0073007404
:10C9C000006400140054004400FF00FF00FF0072E8
:10C9D000006300530043004200FF00FF0273006247
:10C9E000005200510040004100FF00FF027202634C
:10C9F000006100FF005000FF00FF00FF00FF00FF8C
:10CA000000FF00FF00FF00FF00FF00FF00FF0060CD
:10CA1000026200FF023200FF00FF00FF022300FF5E
:10CA200000FF00FF00FF014000FF00FF00FF00FFCC
:10CA300000FF00FF00FF00FF00FF00FF00FF00FFFE
:10CA400000FF00FF00FF017000FF00FF00FF00FF7C
:10CA500000FF00FF00FF00FF00FF0D0A57656C6339
:10CA60006F6D6520746F205354454343590D0A0080
:10CA70005344206361726420616C72656164792043
:10CA80006D6F756E74656400534420636172642039
:10CA90006D6F756E7465642C207265747279206395
:10CAA0006F756E74203D2025640A006D6F756E747D
:10CAB00000252D323073002F002E746170002E740B
:10CAC0007A78002E7A383000524553455400524F40
:10CAD0004D004C4F41440053746F70205265636F9A
:10CAE0007264005341564500534E415053484F54D1
:10CAF00000536E617073686F743A005361766520FD
:10CB0000746F2066696C653A004175746F73746167
:10CB100072743A204E6F004175746F737461727451
:10CB20003A2059657300000009CB000817CB0008B4
:10CB3000747A785F6765745F776F72643A20756E98
:10CB4000657870656374656420454F460A00747AA1
:10CB5000785F6765745F627974653A20756E657891
:10CB600070656374656420454F460A00747A785F87
:10CB7000726561645F626C6F636B5F7461703A20B1
:10CB8000756E657870656374656420454F460A006C
:10CB9000747A785F726561645F626C6F636B5F74F7
:10CBA00061703A20636865636B73756D206572729E
:10CBB0006F720A00726200747A785F726561645FF6
:10CBC0006865616465723A20756E65787065637436
:10CBD000656420454F460A005A585461706521002B
:10CBE000696E76616C696420545A58207369676E67
:10CBF00061747572650A0077726F6E6720456E64A6
:10CC0000206F6620746578742066696C65206D619C
:10CC1000726B65723A203078253032580A00747A87
:10CC2000785F726561645F626C6F636B5F31303A2D
:10CC300020756E657870656374656420454F460A9B
:10CC400000747A785F726561645F626C6F636B5FBA
:10CC500031323A20756E657870656374656420457D
:10CC60004F460A00747A785F726561645F626C6F28
:10CC7000636B5F31343A20756E65787065637465F7
:10CC80006420454F460A007061757365203D20257C
:10CC9000640A00537472696E67206C656E6774680D
:10CCA000203D2025640A00747A785F626C6F636BA4
:10CCB0005F33303A20756E65787065637465642003
:10CCC000454F460A00746170655F6C6F61643A207D
:10CCD000756E6B6E6F776E20626C6F636B2069642C
:10CCE0003A203078253032580A00746170655F6CE4
:10CCF0006F61643A20454F462072656163686564E0
:10CD00000A00747A785F726561645F626C6F636B4E
:10CD10005F31313A20756E657870656374656420A3
:10CD2000454F460A0077620000001E0000F01EF02A
:10CD300080079E0780F79EF700001F0000F81FF88D
:10CD4000E007FF07E0FFFFFF010000010001010015
:10CD500000010100010000010001010001000001CB
:10CD600001000001000101000001010001000001BB
:10CD700001000001000101000100000100010100AB
:10CD8000000101000100000100010100010000019B
:10CD9000010000010001010001000001000101008B
:10CDA000000101000100000101000001000101007B
:10CDB000000101000100000100010100010000016B
:10CDC000010000010001010000010100010000015B
:10CDD000010000010001010001000001000101004B
:10CDE000000101000100000101000001000101003B
:10CDF000000101000100000100010100010000012B
:10CE0000010000010001010001000001000101001A
:10CE1000000101000100000100010100010000010A
:10CE200001000001000101000001010001000001FA
:10CE300001000001000101000100000100010100EA
:10CE400000010100010000010D0A57726974696E4A
:10CE50006720696E746F20524F4D2C207063203D07
:10CE600020253034582061646472203D2025303400
:10CE700058682C2076616C7565203D20253032582D
:10CE8000680A007A38305F657874643A20696E7693
:10CE9000616C6964206F70636F64653A2030782537
:10CEA0003032580A0076657273696F6E20313A200D
:10CEB000646174615F636F6D707265737365643D07
:10CEC00025640A007A38303A20556E68616E646CC9
:10CED0006564206F70636F64653A20253032582096
:10CEE00050433D253034580A0034382E726F6D009F
:10CEF000008000C0FFFFFFFF0040000000000000B6
:10CF00000000000000000000000000000000000021
:10CF10000000000000000000000000000000000011
:10CF20000000000000000000000000000000000001
:10CF300000000000000000000000000000000000F1
:10CF400000000000000000000000000000000000E1
:10CF5000000000000000000000000000430000008E
:10CF60005C000020232D302B2000686C4C0065668F
:10CF7000674546470030313233343536373839412A
:10CF80004243444546003031323334353637383940
:10CF90006162636465660053756363657373004E15
:10CFA0006F74206F776E6572004E6F2073756368C3
:10CFB0002066696C65206F72206469726563746FA6
:10CFC0007279004E6F20737563682070726F6365AD
:10CFD000737300496E746572727570746564207342
:10CFE000797374656D2063616C6C00492F4F206507
:10CFF00072726F72004E6F2073756368206465767D
:10D00000696365206F7220616464726573730041A7
:10D010007267206C69737420746F6F206C6F6E6719
:10D02000004578656320666F726D61742065727269
:10D030006F7200536F636B657420616C726561641D
:10D040007920636F6E6E656374656400426164206D
:10D0500066696C65206E756D626572004E6F206347
:10D0600068696C6472656E0044657374696E61749E
:10D07000696F6E2061646472657373207265717587
:10D0800069726564004E6F206D6F72652070726FFB
:10D09000636573736573004E6F7420656E6F75679B
:10D0A00068207370616365005065726D69737369A0
:10D0B0006F6E2064656E696564004261642061641E
:10D0C000647265737300446576696365206F7220CE
:10D0D0007265736F75726365206275737900466956
:10D0E0006C65206578697374730043726F73732D78
:10D0F000646576696365206C696E6B004E6F2073A2
:10D1000075636820646576696365004E6F7420619D
:10D11000206469726563746F727900486F7374205C
:10D12000697320646F776E00436F6E6E6563746918
:10D130006F6E20616C726561647920696E20707217
:10D140006F6772657373004973206120646972654B
:10D1500063746F727900496E76616C6964206172E4
:10D1600067756D656E74004E6574776F726B2069BC
:10D170006E74657266616365206973206E6F7420DA
:10D18000636F6E6669677572656400436F6E6E6586
:10D190006374696F6E2061626F7274656420627976
:10D1A000206E6574776F726B00546F6F206D616EC7
:10D1B00079206F70656E2066696C657320696E20DA
:10D1C00073797374656D0046696C6520646573637B
:10D1D000726970746F722076616C756520746F6F00
:10D1E000206C61726765004E6F7420612063686116
:10D1F0007261637465722064657669636500546565
:10D2000078742066696C6520627573790046696C74
:10D210006520746F6F206C6172676500486F73746E
:10D2200020697320756E726561636861626C650068
:10D230004E6F207370616365206C656674206F6E3D
:10D2400020646576696365004E6F74207375707035
:10D250006F7274656400496C6C6567616C207365FE
:10D26000656B00526561642D6F6E6C792066696C28
:10D27000652073797374656D00546F6F206D616EF6
:10D2800079206C696E6B730042726F6B656E2070F3
:10D29000697065004D617468656D617469637320C0
:10D2A000617267756D656E74206F7574206F66208E
:10D2B000646F6D61696E206F662066756E63746958
:10D2C0006F6E00526573756C7420746F6F206C61A3
:10D2D000726765004E6F206D657373616765206FBF
:10D2E00066206465736972656420747970650049AD
:10D2F00064656E7469666965722072656D6F7665C6
:10D300006400496C6C6567616C2062797465207398
:10D31000657175656E636500446561646C6F636B10
:10D32000004E6574776F726B20697320756E72653D
:10D3300061636861626C65004E6F206C6F636B00A7
:10D340004E6F7420612073747265616D0053747246
:10D3500065616D20696F63746C2074696D656F75AC
:10D3600074004E6F2073747265616D207265736F07
:10D370007572636573005669727475616C206369B8
:10D38000726375697420697320676F6E65005072EF
:10D390006F746F636F6C206572726F7200556E6B85
:10D3A0006E6F776E2070726F746F636F6C004D7567
:10D3B0006C7469686F7020617474656D70746564F5
:10D3C00000426164206D6573736167650046756E28
:10D3D0006374696F6E206E6F7420696D706C656D1B
:10D3E000656E746564004469726563746F72792058
:10D3F0006E6F7420656D7074790046696C65206F7E
:10D40000722070617468206E616D6520746F6F208A
:10D410006C6F6E6700546F6F206D616E7920737949
:10D420006D626F6C6963206C696E6B73004E6F2068
:10D4300062756666657220737061636520617661EE
:10D44000696C61626C65004E6F20646174610041BB
:10D450006464726573732066616D696C79206E6FA8
:10D460007420737570706F727465642062792070B7
:10D47000726F746F636F6C2066616D696C790050B8
:10D48000726F746F636F6C2077726F6E6720747940
:10D49000706520666F7220736F636B657400536FE5
:10D4A000636B6574206F7065726174696F6E206F55
:10D4B0006E206E6F6E2D736F636B65740050726FAC
:10D4C000746F636F6C206E6F7420617661696C613C
:10D4D000626C6500436F6E6E656374696F6E207277
:10D4E00065667573656400436F6E6E656374696F1E
:10D4F0006E207265736574206279207065657200B4
:10D500004164647265737320616C72656164792033
:10D51000696E207573650041646472657373206E73
:10D520006F7420617661696C61626C6500536F662F
:10D5300074776172652063617573656420636F6ED3
:10D540006E656374696F6E2061626F727400536FF1
:10D55000636B6574206973206E6F7420636F6E6EE9
:10D56000656374656400536F636B65742069732031
:10D57000616C726561647920636F6E6E656374655A
:10D5800064004F7065726174696F6E2063616E63D1
:10D59000656C6564005374617465206E6F742072ED
:10D5A00065636F76657261626C650050726576695D
:10D5B0006F7573206F776E65722064696564004FC4
:10D5C0007065726174696F6E206E6F742073757010
:10D5D000706F72746564206F6E20736F636B657417
:10D5E0000056616C756520746F6F206C61726765A1
:10D5F00020666F7220646566696E6564206461747C
:10D60000612074797065004D65737361676520747E
:10D610006F6F206C6F6E6700436F6E6E6563746929
:10D620006F6E2074696D6564206F75740000202032
:10D6300020202020202020282828282820202020C2
:10D640002020202020202020202020202020881082
:10D6500010101010101010101010101010100404E2
:10D6600004040404040404041010101010101041E9
:10D67000414141414101010101010101010101015A
:10D6800001010101010101010110101010101042EF
:10D69000424242424202020202020202020202022A
:10D6A0000202020202020202021010101020000008
:10D6B000000000000000000000000000000000006A
:10D6C000000000000000000000000000000000005A
:10D6D000000000000000000000000000000000004A
:10D6E000000000000000000000000000000000003A
:10D6F000000000000000000000000000000000002A
:10D700000000000000000000000000000000000019
:10D710000000000000000000000000000000000009
:10D7200000000000000000000000000000000000F9
:04D7300000000000F5
:08D73400B02AFF7F0100000094
:10D73C0000000000010203040102030406070809AB
:10D74C00010000000A00000064000000FFFFFFFF62
:10D75C00FFFFFFFF0100000010C9000820C90008EE
:10D76C0034C9000848C9000803000000000000008C
:10D77C00000000000102030406070809007A030AEE
:10D78C0001FF01FFFFFFFFFFFFFFFF000000000094
:10D79C00FCCE00081CCF00083CCF000800000000A5
:10D7AC000000000000000000000000005CCF00083A
:10D7BC00000000000000000000000000000000005D
:10D7CC00000000000000000000000000000000004D
:10D7DC00000000000000000000000000000000003D
:10D7EC000000000000000000000000005C000020B1
:0CD7FC002DD60008AD01000889010008CE
:0400000508000000EF
:00000001FF
